:100000000C9451340C9482340C9482340C948234C9
:100010000C9482340C9496AF0C9482340C9429A3E3
:100020000C9421AF0C9482340C9482340C9482345E
:100030000C9407640C9482340C94EBCA0C94BB6F40
:100040000C9482340C9437A40C9482340C94823433
:100050000C9482340C9482340C9482340C94FE8779
:100060000C9482340C94676A0C9482340C9482341D
:100070000C9482340C9482340C9482340C94823428
:100080000C9482340C9482340C9482340C94823418
:100090000C94236A0C9482340C9482340C94823431
:1000A0000C9482340C9482340C94D96E0C94823467
:1000B0000C9482340C94BB6E0C9482340C94823475
:1000C0000C9482340C9482340C9482340C94416EDF
:1000D0000C9482340C9482340C9482340C948234C8
:1000E0000C9482341A8828883688438855885C881E
:1000F0007E8894888CD990DB60DB55DB4ADB3FDB64
:1001000034DBB3DBA3DB0DDBDFDAC3DAC9E087E086
:10011000C9E0CCE03BE168E1C9E0C9E07FE162EE23
:1001200065EE54EE58EE5EEE9CEE69EE6DEE73EE0B
:1001300077EE7BEE81EE85EE89EE9CEE8FEE93EE10
:1001400097EE39F23EF243F24DF257F2D0F261F2FD
:1001500069F271F27BF285F28FF29EF2A8F2D0F290
:10016000B2F2BCF2C6F287019D01C701C901F301D9
:100170005F01A701B1010D02E901A701EF01FF0134
:100180008101930113028F019101ED014901AF013A
:10019000B901CD01DF01B501C301A501D701D70127
:1001A0008D01D7018D01170207021102C1016901FA
:1001B0004B01AB01D1018901730159015B01EB01D5
:1001C0000502B701084AD73B3BCE016E84BCBFFD98
:1001D000C12F3D6C74319ABD56833DDA3D00C77F17
:1001E00011BED9E4BB4C3E916BAAAABE00000080B0
:1001F0003F05A84CCDB2D44EB93836A9020C50B93F
:10020000918688083CA6AAAA2ABE000000803F0763
:10021000634236B79BD8A71A39685618AEBAAB55A1
:100220008C1D3CB7CC5763BD6DEDFD753EF6177266
:1002300031BF000000803F08000000BE9224491238
:100240003EABAAAA2ABECDCCCC4C3E00000080BE5C
:10025000ABAAAAAA3E00000000BF000000803F0039
:1002600000000000084178D3BB4387D1133D190E2D
:100270003CC3BD4282AD2B3E68EC8276BED98FE195
:10028000A93E4C80EFFFBE01C4FF7F3F000000008D
:1002900000000D9412470D946E790D94E7180D949B
:1002A000E8200D94354D0D9420150D94D9690D94C9
:1002B00016000D94A0790D94A9790D94A9140D94AC
:1002C0002A040D94876B0D944B690D9494500D94F2
:1002D000F94F0D946B790D942A520D9467140D9477
:1002E0005C140D94074D0D9497790D94574F0D9410
:1002F000E94B0D9438520D94E1690D94A84F0D947B
:10030000EA210D9485040D949A500D945C4F0D9440
:10031000B5030D948E790D94D0690D94C8510D9448
:10032000C8470D946D470D9497040D9465100D9476
:100330003C4B0D9484690D941A180D94D1030D94BF
:10034000DB680D9458100D94D5680D94234A0D94D4
:100350009F030D94DC6A0D9488790D943F520D949F
:100360006F4A0D9440040D9490010D94E1490D9451
:10037000C9790D94FD470D949B100D943A140D947A
:10038000324B0D945E790D94FB490D9492150D94AA
:10039000E3030D94F0030D9412690D9411490D942B
:1003A00047140D948B790D9423520D9475500D9430
:1003B000BA510D942E500D948D4B0D9439190D9406
:1003C00096490D943E4C0D942F150D94AD100D943F
:1003D000784C0D944E040D94BD790D943C470D94CA
:1003E00054040D948D6A0D94FA030D94E9660D94EE
:1003F000D34A0D94079F0D9431520D94BB4B0D942D
:1004000071040D94494B0D94E4040D94C0790D943E
:10041000CE510D9402190D94789F0D9452040D94B1
:100420001C520D9455790D94BF470D94966B0D9405
:10043000CB510D942E4D6E616E00696E66004E417B
:100440004E494E495459494E46CDCCCC3D0AD7234E
:100450003C17B7D13877CC2B329595E6241FB14F96
:100460000A000020410000C84200401C4620BCBEDB
:100470004CCA1B0E5AAEC59D7400407A10F35A0048
:10048000A0724E18090010A5D4E80000E8764817BD
:100490000000E40B54020000CA9A3B000000E1F5A2
:1004A00005000080969800000040420F000000A068
:1004B0008601000000102700000000E80300000093
:1004C000006400000000000A0000000000010000BD
:1004D0000000002C76D888DC674F0823DFC1DFAE30
:1004E00059E1B1B796E5E3E453C63AE651997696F9
:1004F000E8E6C28426EB898C9B62ED407C6FFCEFC2
:10050000BC9C9F40F2BAA56FA5F490055A2AF75CEF
:10051000936B6CF9676DC11BFCE0E40D47FEF520A1
:10052000E6B500D0ED902E03009435770500808469
:100530001E080000204E0A000000C80C333333337D
:100540000F986E12831141EF8D2114893BE65516E9
:10055000CFFEE6DB18D1844B381BF77C1D901DA421
:10056000BBE424203284725E228100C9F124ECA114
:10057000E53D276364696E6F70737578585B00643E
:10058000756D7020636C65617265640A006E6F2022
:1005900064756D7020617661696C61626C650A00DA
:1005A000443231202D20726561642063726173686A
:1005B0002064756D700A006E6F2064756D70206127
:1005C0007661696C61626C650A0064756D702063A8
:1005D0006F6D706C6574656420696E20256C756D37
:1005E000730A0058464C41534800454550524F4D00
:1005F000005352414D00442D31202D20456E646C36
:10060000657373206C6F6F700A00534420707269B9
:100610006E74696E67206279746520004163746945
:1006200076652045787472756465723A2000496E6B
:1006300076616C6964206578747275646572005ABD
:10064000204F666673657400556E6B6E6F776E2013
:10065000636F6D6D616E643A2022004D3230302040
:10066000496E76616C696420657874727564657230
:1006700020007A5F6D61783A20007A5F6D696E3A8A
:100680002000795F6D61783A2000795F6D696E3A7C
:100690002000785F6D61783A20006F70656E0054BD
:1006A000524947474552454400785F6D696E3A208C
:1006B000005265706F7274696E6720656E64737442
:1006C0006F70207374617475730053494C454E54B8
:1006D000004E4F524D414C002553204D4F44453A5A
:1006E0002050657263656E7420646F6E653A2025D4
:1006F0006868643B207072696E742074696D65204F
:1007000072656D61696E696E6720696E206D696ED4
:10071000733A2025643B204368616E676520696EEB
:10072000206D696E733A2025640A00456E64206668
:10073000696C65206C69737400426567696E206638
:10074000696C65206C69737400556E6B6E6F776EA3
:1007500020256320636F64653A2025730A000A50E0
:10076000494E44412074656D70657261747572659F
:100770003A20252E3166205A207368696674202835
:100780006D6D293A20252E3366000A537465703A40
:100790002025642F360A000A537465703A202564B8
:1007A0002F362028736B6970706564290A50494E92
:1007B00044412074656D70657261747572653A208C
:1007C0002564205A20736869667420286D6D293A63
:1007D000300A000A5A45524F3A20252E33660A0045
:1007E00073746172742074656D7065726174757272
:1007F000653A20252E31660A0025642020252E32F8
:100800006600255320583A20252E356620593A2077
:10081000252E3566205A3A20252E35660A00536C5F
:100820006565702E2E2E0045303A25642052504DBD
:100830000A50524E303A25642052504D0A00257518
:1008400000416476616E6365204B3D004B206F75FF
:1008500074206F6620616C6C6F7765642072616EC6
:1008600067652100200A200A20004D3232302053D3
:10087000256900255346696C616D656E742073654A
:100880007474696E67733A2044697361626C65645D
:100890000A00255346696C616D656E74207365743A
:1008A00074696E67733A0A25532020204D32303028
:1008B0002044252E32660A00255352657472616306
:1008C000743A20533D4C656E67746820286D6D291D
:1008D00020463A537065656420286D6D2F6D292080
:1008E0005A3A205A4C69667420286D6D290A25539E
:1008F0002020204D3230372053252E3266204625C9
:100900002E3266205A252E32660A25535265636FB1
:100910007665723A20533D4578747261206C656E3D
:1009200067746820286D6D2920463A5370656564A8
:1009300020286D6D2F6D290A25532020204D32303F
:10094000382053252E32662046252E32660A25533E
:100950004175746F2D526574726163743A20533D12
:100960003020746F2064697361626C652C203120C3
:10097000746F20696E746572707265742065787426
:10098000727564652D6F6E6C79206D6F766573205E
:100990006173207265747261637473206F72207268
:1009A00065636F7665726965730A25532020204D53
:1009B000323039205325640A0025535049442068B9
:1009C0006561746265642073657474696E67733AF7
:1009D0000A25532020204D3330342050252E3266F6
:1009E0002049252E32662044252E32660A002553E2
:1009F0005049442073657474696E67733A0A2553CD
:100A00002020204D3330312050252E3266204925BC
:100A10002E32662044252E32660A00255353746513
:100A200070732070657220756E69743A0A255320C0
:100A3000204D39322058252E32662059252E326617
:100A4000205A252E32662045252E32660A2553551A
:100A500053746570207265736F6C7574696F6E3A4C
:100A6000200A2553204D3335302058256420592540
:100A700064205A2564204525640A25534D61786910
:100A80006D756D20666565647261746573202D20D7
:100A90006E6F726D616C20286D6D2F73293A0A2577
:100AA0005320204D3230332058252E3266205925D0
:100AB0002E3266205A252E32662045252E32660AB1
:100AC00025534D6178696D756D2066656564726149
:100AD000746573202D20737465616C746820286DB3
:100AE0006D2F73293A0A255320204D323033205878
:100AF000252E32662059252E3266205A252E326642
:100B00002045252E32660A25534D6178696D756D35
:100B100020616363656C65726174696F6E202D205E
:100B20006E6F726D616C20286D6D2F7332293A0AD9
:100B3000255320204D3230312058256C7520592501
:100B40006C75205A256C752045256C750A25534D0A
:100B50006178696D756D20616363656C6572617440
:100B6000696F6E202D20737465616C746820286D28
:100B70006D2F7332293A0A255320204D323031200F
:100B800058256C752059256C75205A256C752045A3
:100B9000256C750A2553416363656C6572617469E0
:100BA0006F6E3A20503D7072696E742C20523D7207
:100BB0006574726163742C20543D74726176656C47
:100BC0000A255320204D3230342050252E32662005
:100BD00052252E32662054252E32660A2553416452
:100BE00076616E636564207661726961626C6573BB
:100BF0003A20533D4D696E20666565647261746587
:100C000020286D6D2F73292C20543D4D696E207462
:100C1000726176656C206665656472617465202812
:100C20006D6D2F73292C20423D6D696E696D756D58
:100C3000207365676D656E742074696D6520286D1D
:100C400073292C20583D6D6178696D756D20585958
:100C5000206A65726B20286D6D2F73292C20205A15
:100C60003D6D6178696D756D205A206A65726B20E3
:100C7000286D6D2F73292C2020453D6D6178696D9D
:100C8000756D2045206A65726B20286D6D2F732964
:100C90000A255320204D3230352053252E32662030
:100CA00054252E32662042252E32662058252E32BB
:100CB000662059252E3266205A252E32662045257B
:100CC0002E32660A2553486F6D65206F6666736520
:100CD0007420286D6D293A0A255320204D32303674
:100CE0002058252E32662059252E3266205A252E70
:100CF00032660A004625642025640A004D4D5520C1
:100D00003C3D2027462564202564270A0043617066
:100D10003A25533A25630A0050525553415F4D4DD1
:100D2000553200455854454E4445445F4D323000DD
:100D30004155544F5245504F52545F504F534954B0
:100D4000494F4E004155544F5245504F52545F4603
:100D5000414E53004155544F5245504F52545F54E9
:100D6000454D5000005A30005A3100593000593179
:100D700000583000583100456E642073746F7073F2
:100D800020646961670044656C6574696F6E2066F4
:100D900061696C65642C2046696C653A200046697F
:100DA0006C652064656C657465643A004E6F7420F0
:100DB0005344207072696E74696E67005072696E78
:100DC00074207361766564005344207072696E7498
:100DD00020706175736564004F4B004241440052BE
:100DE000414D426F2046414E200043524153485FDF
:100DF00043414E43454C0043524153485F524543A3
:100E00004F5645520043524153485F5245434F5657
:100E100045520022283229004475706C6963617460
:100E20006520542D636F64652069676E6F72656419
:100E30002E00496E76616C6964205420636F64658E
:100E40002E002C204D39303720452069676E6F7297
:100E50006564006E6F2076616C696420636F6D6DF0
:100E6000616E64002C20002C20002C20006E2F616D
:100E7000002C20002C20002C20006E2F6100503A06
:100E8000005761697420666F722050494E444120BA
:100E90007461726765742074656D706572617475D4
:100EA00072653A004155544F004C414E472053451E
:100EB0004C20464F5243454400256925250A00250C
:100EC0006925250A002228312900303030303030A1
:100ED00030302D303030302D303030302D3030301B
:100EE000302D303030303030303030303030002045
:100EF000555549443A00310020455854525544450F
:100F0000525F434F554E543A0050727573612069D9
:100F100033204D4B335300204D414348494E455FEC
:100F2000545950453A00312E300020626173656497
:100F3000206F6E204D61726C696E204649524D578C
:100F40004152455F55524C3A68747470733A2F2F72
:100F50006769746875622E636F6D2F707275736147
:100F600033642F50727573612D4669726D776172AB
:100F7000652050524F544F434F4C5F564552534992
:100F80004F4E3A004649524D574152455F4E414DF2
:100F9000453A50727573612D4669726D776172655D
:100FA00020004D31313320530020423A0020453A91
:100FB00000543A006F6B20006E2F61003F546F7336
:100FC0006869626120466C61736841697220476597
:100FD000744950206661696C65640A00000125311E
:100FE0001D0C4024301C0B45232F1B0A17FF040641
:100FF000222B1A03373735382569206D696E2C206E
:1010000025692073656300496E76616C6964204DC3
:1010100020636F64653A2025730A004D657368206C
:10102000626564206C6576656C696E67206E6F74AE
:10103000206163746976652E002020000A4D656189
:10104000737572656420706F696E74733A000A5A22
:1010500020736561726368206865696768743A2007
:10106000004E756D20582C593A200050494E44418D
:101070002070726F62652063616C6962726174696D
:101080006F6E2073746172740047323820573000DD
:101090004E6F2050494E444120746865726D6973EB
:1010A000746F7200736574006E6F7A7A6C65004DB0
:1010B000424C004652004C7A004C616E670052650B
:1010C000760046697200534E20696E76616C6964E1
:1010D00000534E005245534554004D4D5552455313
:1010E000004D32340075766C6F00746878004641AC
:1010F0004E0046414E50494E5453540050524E00FB
:1011000050696E67005052555341005345545F4338
:10111000484F505F005345545F535445505F005350
:1011200045545F574156455F00544D435F0043525D
:101130004153485F43414E43454C0043524153485D
:101140005F5245434F5645520043524153485F4416
:10115000455445435445440043524153485F004D74
:101160003120004D30004D31313700472D636F6421
:101170006520736C6963656420666F72206120640A
:101180006966666572656E74206C6576656C2E2086
:10119000436F6E74696E75653F00472D636F6465BC
:1011A00020736C6963656420666F722061206469D6
:1011B00066666572656E74206C6576656C2E20506F
:1011C0006C656173652072652D736C69636520744D
:1011D0006865206D6F64656C20616761696E2E20A3
:1011E0005072696E742063616E63656C6C65642E09
:1011F00000472D636F646520736C696365642066C6
:101200006F722061206E65776572206669726D77F6
:101210006172652E20506C65617365207570646124
:10122000746520746865206669726D776172652ED9
:10123000205072696E742063616E63656C6C6564C6
:101240002E00472D636F646520736C6963656420AD
:10125000666F722061206E65776572206669726DB7
:10126000776172652E20436F6E74696E75653F00FD
:10127000472D636F646520736C6963656420666FD6
:1012800072206120646966666572656E7420707292
:10129000696E74657220747970652E20436F6E7468
:1012A000696E75653F00472D636F646520736C69D7
:1012B00063656420666F722061206469666665728A
:1012C000656E74207072696E7465722074797065D1
:1012D0002E20506C656173652072652D736C696397
:1012E0006520746865206D6F64656C206167616955
:1012F0006E2E205072696E742063616E63656C6C33
:1013000065642E00507265737320746865206B6E7F
:101310006F6220746F2070726568656174206E6FF3
:101320007A7A6C6520616E6420636F6E74696E7585
:10133000652E00506C656173652070726573732053
:10134000746865206B6E6F6220746F20756E6C6FB1
:1013500061642066696C616D656E740052656D6FC5
:101360007665206F6C642066696C616D656E7420B3
:10137000616E6420707265737320746865206B6E93
:101380006F6220746F207374617274206C6F61647B
:10139000696E67206E65772066696C616D656E7435
:1013A0002E00616E6420707265737320746865200E
:1013B0006B6E6F6200496E736572742066696C6152
:1013C0006D656E7400436F6C6F72206E6F74206376
:1013D0006F72726563740046696C616D656E74202E
:1013E0006E6F74206C6F61646564004368616E6742
:1013F000656420636F72726563746C793F004C6F33
:101400006164696E6720636F6C6F72004368616E20
:10141000676520737563636573732100506C656144
:101420007365206F70656E2069646C657220616EF3
:10143000642072656D6F76652066696C616D656E9E
:1014400074206D616E75616C6C792E00576173202C
:1014500066696C616D656E7420756E6C6F61642079
:101460007375636365737366756C3F00506C65617B
:10147000736520757067726164652E004E65772014
:101480006669726D776172652076657273696F6ED9
:1014900020617661696C61626C653A0057616974BC
:1014A000696E6720666F722050494E444120707209
:1014B0006F626520636F6F6C696E670043686F6F62
:1014C00073652065787472756465723A0043686F5D
:1014D0006F73652066696C616D656E743A004E6F5E
:1014E000206D6F76652E00537461626C6520616DAE
:1014F0006269656E742074656D7065726174757271
:10150000652032312D323643206973206E65656463
:1015100065642061207269676964207374616E6418
:101520002069732072657175697265642E00506C54
:10153000656173652072756E2058595A2063616C1D
:101540006962726174696F6E2066697273742E00CD
:101550005761697420666F7220757365722E2E2E26
:1015600000435A5058003B53006164635F696E69E1
:1015700074000A204F726967696E616C2050727541
:1015800073612069330A20202050727573612052E4
:101590006573656172636800200A200A200A2000D2
:1015A000416C6C20446174610053657276696365B7
:1015B0002070726570005368697070696E67207082
:1015C0007265700053746174697374696373004C5D
:1015D000616E67756167650045524153494E47200A
:1015E000616C6C206461746100466163746F727930
:1015F0002052455345540044495341424C45440010
:10160000454E41424C454400202873656E736F720D
:1016100020626F617264207265766973696F6E3AD9
:101620002553290A004653656E736F7220255300B7
:10163000494E5434004D4B33534D4D553253004EAB
:101640004F4D4B3353002E014E4F435455410041F3
:101650004C5446414E0046656220313720323032CC
:101660003200436F6D70696C65643A2000286E6FBC
:101670006E652C2064656661756C7420636F6E66A0
:1016800069672900466562203137203230323220C6
:1016900032323A30363A35370020332E31302E315F
:1016A0002D3436393700737461727400534E2075CF
:1016B0007064617465206661696C656400534E20D6
:1016C0007570646174656400435A50580043524118
:1016D00053485F4445544543544544585900435288
:1016E0004153485F4445544543544544590043528F
:1016F0004153485F444554454354454458004D3296
:10170000390045787465726E616C205350492066CB
:101710006C6173680A58464C415348206973206EC7
:101720006F74207265732D0A706F6E64696E672E18
:10173000204C616E67756167650A737769746368C9
:1017400020756E617661696C61626C652E002F2F69
:1017500020616374696F6E3A64756D705F61766164
:10176000696C61626C650050727573612069332029
:101770004D4B3353204F4B2E0043726173684465C9
:10178000746563742044495341424C45440043729C
:1017900061736844657465637420454E41424C45ED
:1017A00044210045787472756465722066616E200C
:1017B000747970653A200058464C415348206E6F4A
:1017C0007420726573706F6E64696E672E002020DE
:1017D000506C616E6E6572427566666572427974B0
:1017E00065733A20002046726565204D656D6F7205
:1017F000793A2000207C20417574686F723A20008D
:10180000204C61737420557064617465643A2000E3
:1018100020536F667477617265205265736574003A
:10182000205761746368646F672052657365740044
:101830002042726F776E206F7574205265736574E5
:10184000002045787465726E616C20526573657412
:1018500000506F7765725570006572726F722077F5
:10186000726974696E6720746F2066696C650044E4
:101870006F6E6520736176696E672066696C652E90
:10188000006F6B004D4B3353206669726D77617248
:1018900065206465746563746564206F6E204D4BCC
:1018A00033207072696E74657200465720637261EE
:1018B00073682064657465637465642120596F756D
:1018C0002063616E20636F6E74696E75652070723F
:1018D000696E74696E672E20446562756720646165
:1018E000746120617661696C61626C6520666F72FB
:1018F00020616E616C797369732E20436F6E746121
:10190000637420737570706F727420746F207375B8
:10191000626D69742064657461696C732E00426C39
:1019200061636B6F7574206F636375727265642E8B
:10193000205265636F766572207072696E743F0025
:1019400053656C66746573742077696C6C2062658E
:101950002072756E20746F2063616C6962726174AD
:10196000652061636375726174652073656E736F62
:10197000726C657373207265686F6D696E672E0097
:101980005468657265206973207374696C6C20619A
:10199000206E65656420746F206D616B65205A2030
:1019A00063616C6962726174696F6E2E20506C6540
:1019B00061736520666F6C6C6F7720746865206D4D
:1019C000616E75616C2C206368617074657220466D
:1019D000697273742073746570732C2073656374FB
:1019E000696F6E2043616C6962726174696F6E2009
:1019F000666C6F772E005072696E74657220686134
:101A000073206E6F74206265656E2063616C69621D
:101A10007261746564207965742E20506C65617301
:101A20006520666F6C6C6F7720746865206D616EE1
:101A300075616C2C206368617074657220466972F0
:101A400073742073746570732C2073656374696F8D
:101A50006E2043616C6962726174696F6E20666C9E
:101A60006F772E004F6C642073657474696E6773B2
:101A700020666F756E642E2044656661756C7420F7
:101A80005049442C20457374657073206574632E2F
:101A90002077696C6C206265207365742E00576135
:101AA000726E696E673A20626F7468207072696E38
:101AB000746572207479706520616E64206D6F7436
:101AC000686572626F617264207479706520636802
:101AD000616E6765642E005761726E696E673A20A9
:101AE0007072696E746572207479706520636861C4
:101AF0006E6765642E005761726E696E673A206D7D
:101B00006F74686572626F617264207479706520A9
:101B10006368616E6765642E0055534152543220EC
:101B200072782046756C6C212121005365747469AC
:101B30006E67732053746F7265640053746F7265BF
:101B4000642073657474696E67732072657472695A
:101B5000657665640048617264636F6465642044FF
:101B6000656661756C742053657474696E67732063
:101B70004C6F6164656400563200000000C842008A
:101B800000C8420000C84300008C430000484300E6
:101B9000004843000040410000F042E8030000E834
:101BA000030000C80000008813000000409C4400AF
:101BB000409C440000000000000000204E00000097
:101BC00000204100002041CDCCCC3E0000904000E0
:101BD0000000000000000000000000CDCCCC3E3D25
:101BE0000A8141FF08433EB099AB438F42FC42E675
:101BF0005A343F4C62B045000000000040400000F5
:101C0000344200000000000000000000004100001D
:101C100000E03F0000C8420000C842000040410010
:101C200000F042C0030000C0030000C800000088AC
:101C30001300001010102000409C44627573793A24
:101C40002070617573656420666F7220696E7075AF
:101C50007400627573793A207061757365642066EB
:101C60006F72207573657200627573793A207072B5
:101C70006F63657373696E670000007F4300805473
:101C8000430000524300000000000080C09A9919F0
:101C90003E00000000000080C09A99193E0000A09C
:101CA000400000A0400000004025336420737465AC
:101CB000703D253264206D73636E743D2534640A73
:101CC0000000007F43008058439AD95143FFFFFF33
:101CD000256C7520627974657320777269747465F8
:101CE0006E20746F202553206174206164647265D6
:101CF00073732030782530346C780A0044256420D2
:101D00002D20526561642F57726974652025530A2E
:101D10000043726173682064657465637465642E42
:101D20000058595A2063616C6962726174696F6E00
:101D300020616C6C2072696768742E20536B657724
:101D40002077696C6C20626520636F7272656374C2
:101D50006564206175746F6D61746963616C6C7921
:101D60002E0058595A2063616C6962726174696F00
:101D70006E20616C6C2072696768742E20582F5930
:101D800020617865732061726520736C696768747F
:101D90006C7920736B657765642E20476F6F6420C4
:101DA0006A6F62210058595A2063616C69627261DE
:101DB00074696F6E206F6B2E20582F5920617865E3
:101DC00073206172652070657270656E64696375F9
:101DD0006C61722E20436F6E67726174756C6174F2
:101DE000696F6E73210058595A2063616C69627281
:101DF0006174696F6E206661696C65642E2052693A
:101E00006768742066726F6E742063616C696272B9
:101E10006174696F6E20706F696E74206E6F7420CC
:101E2000726561636861626C652E0058595A20635F
:101E3000616C6962726174696F6E206661696C655C
:101E4000642E2046726F6E742063616C69627261E9
:101E500074696F6E20706F696E7473206E6F74207A
:101E6000726561636861626C652E0058595A20631F
:101E7000616C6962726174696F6E206661696C651C
:101E8000642E20506C6561736520636F6E73756C92
:101E90007420746865206D616E75616C2E005859F0
:101EA0005A2063616C6962726174696F6E20636F3E
:101EB0006D70726F6D697365642E20526967687406
:101EC0002066726F6E742063616C696272617469FE
:101ED0006F6E20706F696E74206E6F742072656112
:101EE000636861626C652E0058595A2063616C69A1
:101EF00062726174696F6E20636F6D70726F6D696D
:101F00007365642E2046726F6E742063616C696223
:101F1000726174696F6E20706F696E7473206E6F7A
:101F20007420726561636861626C652E0058595A4D
:101F30002063616C6962726174696F6E20666169A9
:101F40006C65642E204265642063616C6962726115
:101F500074696F6E20706F696E7420776173206E84
:101F60006F7420666F756E642E00506C65617365CA
:101F700020706C61636520737465656C207368659F
:101F80006574206F6E20686561746265642E00441C
:101F9000697374616E6365206265747765656E2030
:101FA000746970206F6620746865206E6F7A7A6C31
:101FB0006520616E642074686520626564207375B5
:101FC000726661636520686173206E6F742062655C
:101FD000656E20736574207965742E20506C656180
:101FE000736520666F6C6C6F7720746865206D6117
:101FF0006E75616C2C20636861707465722046692F
:102000007273742073746570732C207365637469C4
:102010006F6E204669727374206C617965722063FB
:10202000616C6962726174696F6E2E00506C6163DD
:10203000652061207368656574206F66207061702B
:10204000657220756E64657220746865206E6F7AA3
:102050007A6C6520647572696E67207468652063A8
:10206000616C6962726174696F6E206F6620666967
:10207000727374203420706F696E74732E204966F9
:1020800020746865206E6F7A7A6C65206361746372
:10209000686573207468652070617065722C2070AB
:1020A0006F776572206F666620746865207072694C
:1020B0006E74657220696D6D6564696174656C79B3
:1020C0002E00506C656173652072656D6F766520BA
:1020D000737465656C2073686565742066726F6DD6
:1020E00020686561746265642E00497320737465AD
:1020F000656C207368656574206F6E206865617417
:102100006265643F00536561726368696E6720624F
:1021100065642063616C6962726174696F6E2070BE
:102120006F696E74004D6561737572696E672072B8
:1021300065666572656E63652068656967687420A9
:102140006F662063616C6962726174696F6E207082
:102150006F696E7400506C6561736520636C6561B6
:102160006E20746865206E6F7A7A6C6520666F7277
:102170002063616C6962726174696F6E2E20436CBA
:1021800069636B207768656E20646F6E652E004111
:1021900075746F20686F6D65004D6561737572654C
:1021A0006420736B6577733A2025662025660A00E4
:1021B00046697474696E67206661696C6564203D68
:1021C0003E2063616C6962726174696F6E20666142
:1021D000696C65642E0A0043616C6962726174699E
:1021E0006F6E20737563636573732E0A00416C6CA8
:1021F00020342063616C6962726174696F6E207053
:102200006F696E747320666F756E642E0A00312FCD
:102210003400312F3400312F390078797A63616CC2
:102220005F6D656173737572655F656E7465720A63
:102230000078797A63616C5F73706972616C3820C1
:1022400063783D25642063793D2564207A303D25FF
:102250006420647A3D2564207261646975733D254C
:10226000642061643D25640A0078797A63616C5F5B
:102270007365617263685A206E6F207369676E615F
:102280006C0A20783D256C6420793D256C64207AA9
:102290003D256C640A00204F4E2D5349474E414C5A
:1022A00020617420783D256420793D2564207A3DA5
:1022B00025642061643D25640A0078797A63616C45
:1022C0005F7365617263685A20783D256C6420797C
:1022D0003D256C64207A3D256C640A0025640A0063
:1022E0005363616E20636F756E74646F776E3A200E
:1022F000000A002530327800205B25662025665DC7
:10230000206D6D207061747465726E2063656E74EB
:1023100065720A00205B25662025665D5B25665D8B
:10232000206D6D20646976657267656E63650A006D
:102330000000F000F801FC03FE07FE07FE07FE07A1
:10234000FC03F801F000000000000000F000F801BC
:10235000FC03FC03FC03FC03F801F0000000000098
:1023600078797A63616C5F6D656173737572655FAF
:102370006C656176650A00203C20005741524E4949
:102380004E473A2046726F6E7420706F696E7420EB
:102390006E6F7420726561636861626C652E20598E
:1023A00020636F6F7264696E6174653A00000000AB
:1023B00040410000C04000005C430000C0400000FD
:1023C0005C43000046430000404100004643256452
:1023D0002F3400497465726174696F6E3A2000434E
:1023E000616C6962726174696F6E206661696C65A7
:1023F000642120436865636B20746865206178659B
:102400007320616E642072756E20616761696E2E43
:102410000022206661696C65643A204275666665D3
:10242000722066756C6C21002200256920686F752A
:102430007273202569206D696E7574657300544947
:102440004D454F55543A004D3131300046756C6C56
:102450002052582042756666657200437573746F2A
:102460006D00536174696E20005465787475720054
:10247000536D6F6F74680047312059252D2E3266D9
:102480002045252D2E3366004731205825642059DC
:10249000252D2E32662045252D2E33660066736568
:1024A0006E736F725F636865636B706F696E745F84
:1024B0007072696E74006673656E736F7220763029
:1024C0002E3420696E206661756C742072616E67AF
:1024D0006520342E362D3556202D20756E636F6E97
:1024E0006E6563746564006673656E736F722069F0
:1024F0006E20666F7262696464656E2072616E67D9
:102500006520312E352D3356202D20636865636B91
:102510002073656E736F7200312E3000312E3500DE
:10252000554E4B4E4F574E004C413130433A204CA4
:10253000696E65617220416476616E6365206D6FBE
:1025400064653A20004C413130433A2041646A7559
:102550007374656420452D4A65726B3A2000656E80
:10256000717565696E67202200446F6E6520707218
:10257000696E74696E672066696C65004D31313231
:102580002063616C6C65642E20456D657267656EB5
:1025900063792053746F702E005072696E74657287
:1025A0002073746F707065642064756520746F208B
:1025B0006572726F72732E20466978207468652088
:1025C0006572726F7220616E6420757365204D397B
:1025D000393920746F20726573746172742E2028EB
:1025E00054656D70657261747572652069732072CF
:1025F000657365742E205365742069742061667458
:1026000065722072657374617274696E6729004E19
:102610006F204C696E65204E756D6265722077691A
:10262000746820636865636B73756D2C204C6173EF
:1026300074204C696E653A20004E6F2043686563D4
:102640006B73756D2077697468206C696E65206E98
:10265000756D6265722C204C617374204C696E65D7
:102660003A2000636865636B73756D206D69736DE7
:10267000617463682C204C617374204C696E653AF8
:1026800020004C696E65204E756D6265722069731D
:10269000206E6F74204C617374204C696E65204EFF
:1026A000756D6265722B312C204C617374204C69FE
:1026B0006E653A200053544F505045442E00756EBD
:1026C0006B6E6F776E2073746174650020302E34EA
:1026D000206F72206E657765720020302E33206F78
:1026E00072206F6C64657200000E1315110E0000ED
:1026F0000004120912040000001C1F11111F000029
:102700000006191803130C00040E1F041C0000001F
:10271000040A0A0A0A11110E0C12120C0000000021
:10272000001F1511151F0000000103161C080000F2
:102730000000110A04110A042563252D31382E31B9
:1027400038532563005B25735D2563005B25535D6E
:102750002563002563252D31382E31385300252E71
:1027600031305320002563252D31382E3138732523
:1027700063002563252D2E31365320002563252E39
:102780003135533A257325336400252D32302E32EE
:1027900030530A00457872656D65207370616E2054
:1027A0006F6620746865205A2076616C75657321A8
:1027B0000025642F3900426564206C6576656C697C
:1027C0006E67206661696C65642E2053656E736F59
:1027D00072206469646E2774207472696767657219
:1027E0002E20446562726973206F6E206E6F7A7A54
:1027F0006C653F2057616974696E6720666F72204F
:1028000072657365742E00312F390024F4D4305072
:10281000C38E20C2A24017828B7011127A910D8153
:102820006CD90AA861E108C7586607615143061EC2
:102830004B5D05C145A7041A411104093D98037178
:102840003931034036DB0265339102D430540280C3
:102850002E1D02632CEE01752AC501B028A00110BF
:102860002781018F2564012B244B01E0223401AC28
:10287000211F018D200D01801FFC00841EED00979B
:102880001DDF00B81CD200E61BC600201BBC006484
:102890001AB200B219A8000A19A0006A189900D14A
:1028A00017910040178B00B516840031167E00B3D7
:1028B0001579003A157300C7146F0058146A00EEBA
:1028C0001366008813630025135E00C7125B006C5B
:1028D00012570015125400C111510070114F002100
:1028E000114B00D61049008D1047004610440002DD
:1028F000104200C00F4000800F3E00420F3C000617
:102900000F3B00CB0E3800930E37005C0E350027CE
:102910000E3400F30D3200C10D3100900D30006017
:102920000D2E00320D2D00050D2C00D90C2B00AE04
:102930000C2900850C29005C0C2700350C27000EA3
:102940000C2600E80B2400C40B2400A00B23007D00
:102950000B23005A0B2100390B2100180B2000F823
:102960000A1F00D90A1E00BB0A1E009D0A1D008016
:102970000A1D00630A1C00470A1B002C0A1B0011D9
:102980000A1A00F7091A00DD091900C4091900AB79
:10299000091900920917007B091800630917004CF8
:1029A00009160036091600200916000A091500F557
:1029B000081500E0081400CC081400B8081400A49E
:1029C000081400900813007D0812006B08130058CB
:1029D00008120046081200340811002308110012E2
:1029E00008110001081100F0071000E0071000D0E6
:1029F000071000C0071000B0070F00A107100091DA
:102A0000070E0083070F0074070F0065070E0057BD
:102A1000070E0049070E003B070D002E070E002091
:102A2000070D0013070D0006070D00F9060C00ED59
:102A3000060D00E0060C00D4060C00C8060C00BC15
:102A4000060C00B0060C00A4060B0099060C008DC5
:102A5000060B0082060B0077060B006C060B00616C
:102A6000060A0057060B004C060A0042060A003808
:102A7000060A002E060A0024060A001A060A00109A
:102A800006090007060A00FD050900F4050900EB28
:102A9000050900E2050900D9050900D0050900C7AC
:102AA000050900BE050900B5050800AD050800A52B
:102AB0000509009C050800940508008C05080084A1
:102AC0000508007C050800740508006C0507006512
:102AD0000508005D050700560508004E050700477C
:102AE0000507004005080038050700310507002AE2
:102AF000050700230507001C050600160507000F43
:102B00000507000805060002050700FB040600F59E
:102B1000040700EE040600E8040600E2040700DBF8
:102B2000040600D5040600CF040600C9040600C34D
:102B3000040600BD040600B7040600B1040500AC9D
:102B4000040600A6040600A00405009B04060095E8
:102B5000040500900406008A040500850405008031
:102B60000406007A04050075040500700405006B76
:102B700004050066040500610405005C04050057B7
:102B8000040500520405004D0405004804050043F7
:102B90000405003E0404003A040500350405003035
:102BA0000404002C04050027040400230405001E6F
:102BB0000404001A04040016040500110404000DA6
:102BC000040400090405000404040000040400FCDB
:102BD000030400F8030400F4030400F0030400EC11
:102BE000030400E8030400E4030400E0030400DC41
:102BF000030400D8030400D4030400D0030400CC71
:102C0000030400C8030300C503030024F404D9200F
:102C10001BC40C5C0E9804C4095F0265077101F4C3
:102C200005F900FB04B30048048700C1036900589C
:102C300003550003034500BE023A008402310053ED
:102C4000022A002902250004022000E4011C00C819
:102C5000011900AF011700980114008401130071DD
:102C60000110006101100051010E0043010D0036FA
:102C7000010B002B010B0020010B00150109000CBA
:102C800001090003010800FB000800F3000800EB45
:102C9000000700E4000600DE000600D8000600D2AF
:102CA000000600CC000500C7000500C2000500BDFD
:102CB000000400B9000400B5000400B1000400AD38
:102CC000000400A9000400A5000300A20003009F67
:102CD0000004009B0003009800030095000200938D
:102CE000000300900003008D0002008B00030088A9
:102CF0000002008600020084000300810002007FC1
:102D00000002007D0002007B0002007900020077D3
:102D100000010076000200740002007200010071E0
:102D20000002006F0002006D0001006C0002006AEA
:102D300000010069000200670001006600010065F3
:102D400000010064000200620001006100010060F7
:102D50000001005F0002005D0001005C0001005BFB
:102D60000001005A000100590001005800010057FD
:102D700000010056000100550001005400010053FD
:102D800000000053000100520001005100010050FA
:102D90000001004F0001004E0000004E0001004DF8
:102DA0000001004C0001004B0000004B0001004AF4
:102DB00000010049000100480000004800010047F0
:102DC00000010046000000460001004500000045EB
:102DD00000010044000100430000004300010042E4
:102DE00000000042000100410000004100010040DD
:102DF0000001003F0000003F0001003E0000003ED7
:102E00000001003D0000003D0001003C0000003CCE
:102E10000000003C0001003B0000003B0001003AC4
:102E20000000003A000100390000003900010038BC
:102E300000000038000000380001003700000037B3
:102E400000010036000000360000003600010035A9
:102E5000000000350000003500010034000000349F
:102E60000000003400010033000000330000003394
:102E70000001003200000032000000320001003189
:102E8000000000310000003100010030000000307F
:102E9000000000300001002F0000002F0000002F74
:102EA0000000002F0001002E0000002E0000002E68
:102EB0000001002D0000002D0000002D0000002D5D
:102EC0000001002C0000002C0000002C0000002C51
:102ED0000001002B0000002B0000002B0000002B45
:102EE0000001002A0000002A0000002A0000002A39
:102EF000000100290000002900000029000000292D
:102F0000000000290001002800000028000000281F
:102F10000000002800000028000100270000002712
:102F20000000002700000027000000270001002605
:102F300000000026000000260000002600000026F9
:102F400000010025000000250000002500000025EC
:102F500000000025000000250001002400000024DE
:102F600000000024000000240000002400010023D1
:102F700000000023000000230000002300000023C5
:102F800000000023000000230001002200000022B6
:102F900000000022000000220000002200000022A9
:102FA000000100210000002100000021000000219C
:102FB000000000210000002100000021000100208D
:102FC0000000002000000020000000200000002081
:102FD0000000002000000020000000200001001F71
:102FE0000000001F0000001F0000001F0000001F65
:102FF0000000001F0000001F0001001E0000001E56
:103000000000001E0000001E000000504944204146
:1030100075746F74756E652066696E697368656432
:10302000212050757420746865206C617374204B86
:10303000702C204B6920616E64204B6420636F6E9E
:103040007374616E74732066726F6D2061626F7647
:103050006520696E746F20436F6E66696775726173
:1030600074696F6E2E6800504944204175746F7406
:10307000756E65206661696C6564212074696D6593
:103080006F75740020403A00543A00423A005049AB
:1030900044204175746F74756E65206661696C6556
:1030A00064212054656D7065726174757265207459
:1030B0006F6F206869676800204B643A2000204BDE
:1030C000693A2000204B703A200020436C617373F2
:1030D00069632050494420002054753A2000204B59
:1030E000753A2000206D61783A2000206D696E3AB3
:1030F000200020643A200020626961733A20004D6C
:10310000363030006673656E736F725F7570646120
:103110007465202D204D3630300049522073656E85
:10312000736F72206E6F7420726573706F6E646956
:103130006E672028256429210A0020573A0020457F
:103140003A00543A005A206C6976652061646A75C9
:103150007374206F7574206F662072616E67652EC0
:103160002053657474696E6720746F20302E20437D
:103170006C69636B20746F20636F6E74696E756524
:103180002E005A206C6976652061646A757374201C
:103190006F7574206F662072616E67652E205365AF
:1031A0007474696E6720746F20300020423A0020EA
:1031B000453A00543A00494E5434004865617469F8
:1031C0006E672064697361626C6564206279207344
:1031D00061666574792074696D65722E00465320AE
:1031E00076302E33206F72206F6C64657200465308
:1031F0002076302E34206F72206E6577657200491C
:103200006E61637469766974792053687574646F4C
:10321000776E004B494C4C45442E20005072696E2D
:103220007465722068616C7465642E206B696C6CC7
:1032300028292063616C6C656421004B494C4C3A31
:103240002025640A004D32323120496E76616C6966
:103250006420657874727564657220004D3231386F
:1032600020496E76616C6964206578747275646556
:103270007220004D31303920496E76616C696420CE
:10328000657874727564657220004D31303520495F
:103290006E76616C696420657874727564657220FD
:1032A000004D31303420496E76616C696420657858
:1032B0007472756465722000504F5745522050411A
:1032C0004E49432044455445435445440055564CCB
:1032D0004F202D20656E642025640A0055564C4F02
:1032E0005F54494E59202D20656E642025640A00E4
:1032F000436F6F6C646F776E0050726568656174C0
:1033000020746865206E6F7A7A6C65210045525290
:103310004F523A0046696C616D656E742065787431
:10332000727564696E672026207769746820636F00
:10333000727265637420636F6C6F723F00417574C5
:103340006F6C6F6164696E672066696C616D656E34
:1033500074206973206163746976652C206A7573C3
:103360007420707265737320746865206B6E6F6271
:1033700020616E6420696E736572742066696C6189
:103380006D656E742E2E2E005072696E74207469F5
:103390006D650046696C616D656E7420757365645A
:1033A00000546F74616C207072696E742074696D62
:1033B0006500546F74616C2066696C616D656E7434
:1033C000005269676874004C65667400592064692E
:1033D0007374616E63652066726F6D206D696E0037
:1033E00053657665726520736B657700536C69670A
:1033F000687420736B6577004D65617375726564E1
:1034000020736B6577005B303B305D20706F696EB9
:1034100074206F66667365740041646A75737469BD
:103420006E67205A3A0052656172207369646520A4
:103430005B756D5D0046726F6E7420736964655BC9
:10344000756D5D00526967687420736964655B75AA
:103450006D5D004C6566742073696465205B756DF5
:103460005D005365742074656D706572617475726A
:10347000653A00464C4558202D20203234302F35F7
:10348000300050502020202D20203235342F313074
:10349000300048495053202D20203232302F313017
:1034A000300041425320202D20203235352F31303D
:1034B000300050564220202D20203231352F373514
:1034C0000050432020202D20203237352F3131303D
:1034D0000041534120202D20203236302F3130350D
:1034E0000050455420202D20203233302F38350015
:1034F000504C4120202D20203231352F3630006EA7
:103500006F7A7A6C65202D20203235302F3000669E
:1035100061726D2020202D20203235302F38300070
:10352000252D31322E313253252B382E3166004570
:10353000787472756465723A006D6D0059005800B8
:10354000583A00593A005A3A002563252D31332E56
:10355000313353252B352E33660025533A0A253156
:10356000382E32666D200A25533A0A2531306C64B4
:103570006820253032646D20253032647300255375
:103580003A0A2531382E32666D200A25533A0A252B
:1035900031306C6464202530326468202530326418
:1035A0006D0025362E32666D6D0025530A25530AAF
:1035B00025533A0A25533A0025332E326601002559
:1035C0002D31342E3134533A0A25530A252D313406
:1035D0002E3134533A25332E3266010A252D3134EB
:1035E0002E3134533A25332E326601001000C902C1
:1035F00010012C014001220170011801B0010E01DF
:10360000F00104015002FA00B002F0003003E600BD
:10361000D003DC009004D2007005C800A006BE00F4
:103620000008B400B009AA00D00BA000600E9600FC
:1036300060118C000015820020197800C01D6E00FA
:10364000A0226400B0275A00902C500000314600A0
:10365000E0343C0010383200903A2800603C1E00F4
:10366000A03D1400803E0A00203F0000457874729F
:10367000756465722066616E20737065656420698B
:1036800073206C6F776572207468616E2065787046
:103690006563746564005072696E742066616E20A3
:1036A0007370656564206973206C6F776572207430
:1036B00068616E206578706563746564004D494E7D
:1036C00054454D5020414D42004D415854454D50B8
:1036D000004D415854454D5020424544004D4158FD
:1036E00054454D5020414D4200202D20496E7661B9
:1036F0006C6964206578747275646572206E756D8E
:1037000062657220210070012C0190012701B00137
:103710002201C0011D01F001180110021301300245
:103720000E016002090190020401C002FF000003C3
:10373000FA004003F5008003F000D003EB00200402
:10374000E6007004E100E004DC004005D700C0059D
:10375000D2004006CD00D006C8008007C300300864
:10376000BE00F008B900C009B400B00AAF00B00B49
:10377000AA00D00CA500000EA000500F9B00C010A6
:1037800096005012910000148C00C0158700B017ED
:103790008200B0197D00D01B7800001E730040200D
:1037A0006E0090226900F024640040275F00902999
:1037B0005A00E02B5500102E500020304B001032E4
:1037C0004600E033410090353C0010373700703838
:1037D0003200A0392D00B03A2800A03B2300603C05
:1037E0001E00103D1900903D1400103E0F00703E69
:1037F0000A00C03E0500003F000090137D00B01598
:103800007800F0177300601A6E00F01C6900A01FAA
:10381000640050225F0020255A00E0275500902ABE
:103820005000202D4B00A02F4600F03141001034F5
:103830003C00F0353700A037320020392D00603AC7
:103840002800703B2300603C1E00203D1900C03D55
:103850001400403E0F00A03E0A00F03E0500403F2D
:103860000000703FFBFF903FF6FFB03FF1FFC03F0D
:10387000ECFFD03FE7FFE03FE2FFF03FDDFFF03F2E
:10388000D8FF20484F54454E4420544845524D419E
:103890004C2052554E415741590020484541544211
:1038A000454420544845524D414C2052554E4157B5
:1038B000415900544845524D414C2052554E4157B4
:1038C00041590042454420544845524D414C2052F4
:1038D000554E415741590020544845524D414C20C6
:1038E00052554E4157415920285052454845415460
:1038F00020484F54454E44290020544845524D41DC
:103900004C2052554E415741592028505245484568
:1039100041542048454154424544290050524548AD
:10392000454154204552524F520042454420505286
:103930004548454154204552524F52004572723A13
:1039400020002074726967676572656421004865AC
:103950006174657273207377697463686564206F3E
:1039600066662E20003A2000506C656173652072F7
:103970006573746172740047312058352E302045CC
:10398000342E302046313030302E30004731205A2E
:10399000302E32302046313030302E30004731204A
:1039A0005835352E30204532352046313430302ED2
:1039B0003000473120592D322E3020463130303002
:1039C0002E3000473120583234302E3020453235E9
:1039D0002E30202046323230302E3000473932200F
:1039E00045302E30004731205A302E3320463130BA
:1039F00030302E30004731205835352E30204538B4
:103A00002E302046323030302E30004731205835AD
:103A10002E30204533322E302046313830302E3093
:103A2000004731205835352E30204533322E302096
:103A300046313037332E3000473120463430303075
:103A4000004D323034205331303030004731205A6D
:103A5000352046373230302E303030004731204567
:103A60002D312E35303030302046323130302E304E
:103A700030303030004D3833004739300047323174
:103A8000004739322045302E30004731205835303C
:103A9000205935352045332E3632373733004731FC
:103AA0002058323030205935352045302E343933C6
:103AB00038360047312058323030205937352045CC
:103AC000332E3632373733004731205835302059BE
:103AD00037352045302E34393338360047312058B9
:103AE0003530205939352045332E363237373300BB
:103AF00047312058323030205939352045302E3466
:103B0000393338360047312058323030205931317E
:103B1000352045332E36323737330047312058357C
:103B20003020593131352045302E34393338360084
:103B300047312058353020593133352045332E3622
:103B40003237373300473120583230302059313343
:103B5000352045302E363631373400473120583243
:103B6000303020593135352045322E363237373313
:103B70000047312058313030205931353520453219
:103B80000047312058373520593135352045322E00
:103B900035004731204631303830004731205A3027
:103BA0002E3135302046373230302E30303000471D
:103BB00031205835302059313535004739322045CC
:103BC000302E3000473238004D313039004D313918
:103BD00030004D31303700726573756C742076613A
:103BE0006C75653A2025640A0020693D2532642001
:103BF000636E743D2532642076616C3D2532640A23
:103C000000636C7573746572733A0020693D2532E8
:103C10006420737465703D2532640A00736F72749A
:103C200065642073616D706C65733A00252D377380
:103C3000003A200025642F3600252D323053002015
:103C40003A2000252D32307300542564004731207E
:103C50005A302E342046313030302E30004731205B
:103C6000592D332E302046313030302E30004D3833
:103C70003300473120583130302E30204531322E3C
:103C8000352046313030302E300047312058363024
:103C90002E302045392E302046313030302E300045
:103CA000213A0B3AF539E539DC39C339B2399D3956
:103CB0008C397739813A7D3A793A753A5C3A4C3A9F
:103CC000413A383A4731205835302059333520456C
:103CD000252D2E336600AF3B9B3B923B813B713BD6
:103CE0005B3B453B303B1B3B053BF03ADC3AC83A7B
:103CF000B33A9E3A8A3A496E76616C6964205049BB
:103D0000442063616C2E20726573756C74732E2071
:103D10004E6F742073746F72656420746F20454514
:103D200050524F4D2E004D353030004731205A3122
:103D30003520463135303000473931004731205881
:103D40003530205931393020453020463730303039
:103D500000473930004D3834004D373032204300B1
:103D600047312058313020593138302046343030F6
:103D700030004731205A31302046313330302E3038
:103D80003030004D313430205330004D313034204C
:103D9000533000473120452D302E3037353030201C
:103DA00046323130302E3030303030004D31303707
:103DB000004D313137204669727374206C6179652A
:103DC000722063616C2E00526573756D696E672099
:103DD0007072696E740050494E44412048656174A8
:103DE000696E670043616C6962726174696F6E200D
:103DF000646F6E650043616C6962726174696E67BD
:103E0000205A0042656420646F6E6500426564203C
:103E100048656174696E670048656174696E672002
:103E2000646F6E652E0048656174696E6700504965
:103E3000442063616C2E2066696E69736865640056
:103E40005049442063616C2E005072696E7420707A
:103E500061757365640025632533642F25642563CC
:103E6000005A25362E32662563005A2020202D2D3B
:103E70002D200025632533642525002D2D2D0025BB
:103E800033640025335325337325250055534200F1
:103E900020202000205344002025753E2575002059
:103EA0003F3E257500204625750020463F002046F0
:103EB000524D200025632D2D3A2D2D202000256305
:103EC0002533756820256325630025632530327509
:103ED0003A253032752563256300257500593A204F
:103EE0002575202D3E202E2E2E00257500583A20B7
:103EF0002575202D3E202E2E2E004D656173757286
:103F000065642066696C616D656E742073656E739F
:103F10006F72206C6F77206C6576656C3A20253463
:103F20002E3266560A004D656173757265642066AF
:103F3000696C616D656E742073656E736F72206855
:103F4000696768206C6576656C3A2025342E326688
:103F5000560A00457874722066616E20737065653C
:103F6000643A2025640A005072696E742066616E9E
:103F70002073706565643A2025640A005465737483
:103F800020323A00457874722066616E2073706545
:103F900065643A2025640A005072696E7420666177
:103FA0006E2073706565643A2025640A0054657359
:103FB0007420313A004D383400256320415849536C
:103FC000205347313D25640A00486F74656E6400D4
:103FD000426564005A00590058002D2D2D2D2D2DBD
:103FE0002D2D2D2D2D2D2D2D2D2D2D2D2D2D004F0C
:103FF0004B00496E73657274207468652066696C45
:10400000616D656E742028646F206E6F74206C6F14
:1040100061642069742920696E746F20746865205A
:10402000657874727564657220616E642074686569
:104030006E20707265737320746865206B6E6F629A
:104040002E00566572696669636174696F6E2066D9
:1040500061696C65642C2072656D6F76652074688B
:10406000652066696C616D656E7420616E64207494
:10407000727920616761696E2E0053656E736F728D
:104080002076657269666965642C2072656D6F764D
:1040900065207468652066696C616D656E74206E5C
:1040A0006F772E00506C6561736520636865636B84
:1040B000207468652049522073656E736F722063A7
:1040C0006F6E6E656374696F6E2C20756E6C6F61B8
:1040D000642066696C616D656E742069662070721B
:1040E0006573656E742E00506C6561736520756E26
:1040F0006C6F6164207468652066696C616D656EC3
:10410000742066697273742C207468656E20726501
:1041100070656174207468697320616374696F6E7F
:104120002E0057616974696E6720666F72206E6F2A
:104130007A7A6C6520616E642062656420636F6FBB
:104140006C696E670053656C662074657374204FEC
:104150004B0053656C6620746573742073746172D0
:1041600074005072696E742066616E3A004578740E
:1041700072756465722066616E3A0043616C6962B3
:10418000726174696E6720686F6D6500416C6C20A8
:10419000636F727265637400436865636B696E6711
:1041A0002073656E736F727300436865636B696E2D
:1041B0006720686F74656E6400436865636B696E41
:1041C000672062656400436865636B696E67205AA7
:1041D000206178697300436865636B696E67205975
:1041E000206178697300436865636B696E67205866
:1041F000206178697300436865636B696E67206549
:104200006E6473746F70730041786973206C656EAF
:1042100067746820646966666572656E63653A25D1
:104220002E33660A004D656173757265642061788E
:104230006973206C656E6774683A252E33660A00D0
:104240004C434420737461747573206368616E67B6
:10425000656400534420636172642072656C65611B
:1042600073656400452D636F6F6C206D6F6465002E
:10427000414C5446414E206465742E004361726483
:104280002072656D6F766564004F6E004F66660044
:104290004261636B005072696E746572206E6F7A52
:1042A0007A6C65206469616D657465722064696605
:1042B000666572732066726F6D2074686520472D85
:1042C000636F64652E20506C65617365206368655B
:1042D000636B207468652076616C756520696E205B
:1042E00073657474696E67732E205072696E7420E2
:1042F00063616E63656C6C65642E005072696E74E8
:104300006572206E6F7A7A6C65206469616D657480
:10431000657220646966666572732066726F6D20CF
:1043200074686520472D636F64652E20436F6E743B
:10433000696E75653F006265746100616C706861EB
:10434000006465760003000A0001005912505255BE
:104350005341334446570000002100240027002A1F
:10436000002D003000330001010000040107010AA4
:104370000100002200250028002B002E003100340F
:104380000002010000050108010B010000200023CC
:1043900000260029002C002F00320000010000033D
:1043A00001060109010505050507050808080802B9
:1043B0000202020A0A0808040404040101010101BE
:1043C0000101010303030303030303040707070CAD
:1043D0000C0C0C0C0C0C0C02020202060606060663
:1043E0000606060B0B0B0B0B0B0B0B07070A0A0A37
:1043F0000A0A0A0505050404040808010210202021
:104400000808102040102040800201020108040228
:10441000010102040810204080804020100804029E
:1044200001800402018040201008040201080402F7
:1044300001010204081020408001020408102040FD
:1044400080100804088010204004408010204004A0
:104450008000000A0B02090C0D0E0807030401007E
:10446000000000000000000000000000000000004C
:104470000000000000000000000000000012111009
:10448000000000000000000000000000000000002C
:10449000000000000000000000000000000000001C
:1044A0000000000000000054656D70657261747555
:1044B00072652063616C6962726174696F6E2066F7
:1044C00061696C65640054656D70657261747572C4
:1044D000652063616C6962726174696F6E206973D3
:1044E0002066696E697368656420616E642061632B
:1044F000746976652E2054656D702E2063616C6939
:1045000062726174696F6E2063616E2062652064FF
:10451000697361626C656420696E206D656E7520DB
:1045200053657474696E67732D3E54656D702E20EB
:1045300063616C2E0046696C2E2073656E736F721A
:10454000004578747275646572004D6F7665205A07
:10455000004D6F76652059004D6F766520580043F9
:104560007261736820646574656374696F6E20633B
:10457000616E0A6265207475726E6564206F6E20CC
:104580006F6E6C7920696E0A4E6F726D616C206D72
:104590006F6465005741524E494E473A0A43726173
:1045A000736820646574656374696F6E0A64697307
:1045B00061626C656420696E0A537465616C74682D
:1045C000206D6F6465004175746F6C6F6164696E16
:1045D000672066696C616D656E7420617661696CD7
:1045E00061626C65206F6E6C79207768656E2066FD
:1045F000696C616D656E742073656E736F7220698E
:1046000073207475726E6564206F6E2E2E2E0045B9
:1046100052524F523A2046696C616D656E74207338
:10462000656E736F72206973206E6F74207265738C
:10463000706F6E64696E672C20706C6561736520A5
:10464000636865636B20636F6E6E656374696F6E1C
:104650002E004D6F6465206368616E676520696E2A
:104660002070726F67726573732E2E2E0043616C1B
:1046700069627261746500536865657420252E3720
:10468000730A5A206F66667365743A20252B312EA3
:104690003366206D6D0A2563436F6E74696E7565B0
:1046A0000A256353746172742066726F6D207A6597
:1046B000726F00506C65617365206C6F6164206679
:1046C000696C616D656E742066697273742E003E4C
:1046D00043616E63656C0046696C616D656E740064
:1046E00053656C6563742066696C616D656E743AC0
:1046F0000054656D70657261747572652063616CDC
:104700006962726174696F6E206661696C65642E9E
:1047100020436F6E74696E756520776974682070C8
:1047200072657373696E6720746865206B6E6F6263
:104730002E0054656D7065726174757265206361D9
:104740006C6962726174696F6E20646F6E652E2091
:10475000436F6E74696E7565207769746820707236
:10476000657373696E6720746865206B6E6F622E67
:10477000007B5B4552523A00332E31302E31005DC2
:104780005B4657523A005D5B54494D3A005D5B46CB
:104790004E4D3A005D5B46454D3A005D5B504344EB
:1047A0003A005B5446553A007B5B50524E3A3939D9
:1047B0005D007B5B50524E3A355D007B5B50524E44
:1047C0003A305D007B5B50524E3A395D007B5B5066
:1047D000524E3A385D007B5B5245533A305D5B4642
:1047E000494C3A007B5B5245533A315D5B46494C3C
:1047F0003A005B50524E3A005B50464E3A305D00F4
:104800005B4449413A005D5B4154423A005D5B4183
:1048100054303A005D5B5354423A005B5354303A93
:1048200000473830004D3435004D3435205A0047AC
:10483000373600202030002020310046494E4441C8
:104840000050494E44410052756E6E696E672057A4
:10485000697A6172642077696C6C2064656C657438
:10486000652063757272656E742063616C69627233
:104870006174696F6E20726573756C747320616EFC
:10488000642073746172742066726F6D2074686541
:1048900020626567696E6E696E672E20436F6E7465
:1048A000696E75653F0050726568656174696E6711
:1048B000206E6F7A7A6C652E20506C65617365206E
:1048C000776169742E004C6F6164696E6720666958
:1048D0006C616D656E7400506C6561736520696E06
:1048E000736572742066696C616D656E7420696EA3
:1048F000746F207468652065787472756465722CB5
:10490000207468656E20707265737320746865200A
:104910006B6E6F6220746F206C6F61642069742EFF
:1049200000506C6561736520696E736572742066F2
:10493000696C616D656E7420696E746F2074686552
:104940002066697273742074756265206F662074C6
:104950006865204D4D552C207468656E2070726519
:10496000737320746865206B6E6F6220746F206CA7
:104970006F61642069742E00546865207072696EDE
:104980007465722077696C6C207374617274207026
:1049900072696E74696E672061207A69672D7A6129
:1049A00067206C696E652E20526F74617465207487
:1049B0006865206B6E6F6220756E74696C20796F0C
:1049C0007520726561636820746865206F70746912
:1049D0006D616C206865696768742E204368656343
:1049E0006B207468652070696374757265732069E3
:1049F0006E207468652068616E64626F6F6B20283A
:104A000043616C6962726174696F6E206368617082
:104A1000746572292E0053656C6563742074656D2E
:104A20007065726174757265207768696368206D5E
:104A300061746368657320796F7572206D61746548
:104A40007269616C2E0043686F6F73652061206628
:104A5000696C616D656E7420666F72207468652084
:104A60004669727374204C617965722043616C6988
:104A700062726174696F6E20616E642073656C652B
:104A8000637420697420696E20746865206F6E2DD0
:104A900073637265656E206D656E752E004E6F775F
:104AA00020492077696C6C2063616C696272617463
:104AB000652064697374616E6365206265747765EF
:104AC000656E20746970206F6620746865206E6F53
:104AD0007A7A6C6520616E642068656174626564D1
:104AE00020737572666163652E00596F752063616E
:104AF0006E20616C7761797320726573756D6520C6
:104B00007468652057697A6172642066726F6D20DF
:104B100043616C6962726174696F6E202D3E20572B
:104B2000697A6172642E00506C65617365206368F8
:104B300065636B206F75722068616E64626F6F6B66
:104B400020616E6420666978207468652070726FD9
:104B5000626C656D2E205468656E20726573756D8C
:104B600065207468652057697A61726420627920D3
:104B70007265626F6F74696E672074686520707209
:104B8000696E7465722E00416C6C20697320646FCD
:104B90006E652E204861707079207072696E74693C
:104BA0006E672100496620796F75206861766520FF
:104BB0006164646974696F6E616C20737465656C9F
:104BC000207368656574732C2063616C696272611F
:104BD000746520746865697220707265736574739A
:104BE00020696E2053657474696E6773202D2048A8
:104BF00057205365747570202D20537465656C20A3
:104C00007368656574732E00506C6561736520630D
:104C10006C65616E206865617462656420616E64B4
:104C2000207468656E2070726573732074686520E7
:104C30006B6E6F622E00446F20796F752077616E06
:104C40007420746F20726570656174206C61737478
:104C5000207374657020746F20726561646A757367
:104C6000742064697374616E63652062657477652E
:104C7000656E206E6F7A7A6C6520616E642068655F
:104C800061746265643F0053656C656374206E6F88
:104C90007A7A6C6520707265686561742074656DE0
:104CA0007065726174757265207768696368206DDC
:104CB00061746368657320796F7572206D617465C6
:104CC0007269616C2E0049732066696C616D656E56
:104CD00074206C6F616465643F004E6F77204920DB
:104CE00077696C6C2070726568656174206E6F7A8C
:104CF0007A6C6520666F7220504C412E00492077F7
:104D0000696C6C2072756E207A2063616C696272C6
:104D10006174696F6E206E6F772E004E6F77207210
:104D2000656D6F7665207468652074657374207096
:104D300072696E742066726F6D20737465656C2085
:104D400073686565742E00506C65617365207265CB
:104D50006D6F7665207368697070696E672068652D
:104D60006C706572732066697273742E00492077C7
:104D7000696C6C2072756E2078797A2063616C6939
:104D800062726174696F6E206E6F772E2049742095
:104D900077696C6C2074616B6520617070726F78DC
:104DA0002E203132206D696E732E00466972737445
:104DB0002C20492077696C6C2072756E20746865B0
:104DC0002073656C667465737420746F2063686506
:104DD000636B206D6F737420636F6D6D6F6E2061F8
:104DE0007373656D626C792070726F626C656D7340
:104DF0002E0048692C204920616D20796F75722042
:104E00004F726967696E616C2050727573612069B9
:104E100033207072696E7465722E20576F756C64E2
:104E200020796F75206C696B65206D6520746F202B
:104E3000677569646520796F75207468726F75672E
:104E400068207468652073657475702070726F6374
:104E50006573733F0048692C204920616D20796F8C
:104E60007572204F726967696E616C20507275733C
:104E700061206933207072696E7465722E2049203A
:104E800077696C6C20677569646520796F7520742B
:104E900068726F75676820612073686F7274207321
:104EA000657475702070726F636573732C20696E02
:104EB00020776869636820746865205A2D61786975
:104EC000732077696C6C2062652063616C69627223
:104ED000617465642E205468656E2C20796F75208E
:104EE00077696C6C20626520726561647920746FEB
:104EF000207072696E742E00452D636F7272656347
:104F0000743A005A2D636F72726563743A00592DBA
:104F1000636F72726563743A00582D636F727265C5
:104F200063743A00437574746572004D6F64656C08
:104F300000537472696374005761726E0043686550
:104F4000636B73004E6F7A7A6C6520642E004E6F2F
:104F50006E6500416C7068616265740054696D65CE
:104F600000536F72740053442063617264005250A6
:104F70006920706F72740054656D702E2063616CCF
:104F80002E004C696E2E20636F7272656374696FB8
:104F90006E00485720536574757000462E20617569
:104FA000746F6C6F61640044697361626C65207337
:104FB00074657070657273004D6F766520617869F5
:104FC000730054656D706572617475726500546527
:104FD0006D702E2063616C6962726174696F6E001E
:104FE00052657365742058595A2063616C69627206
:104FF0002E005049442063616C6962726174696F6C
:105000006E00426564206C6576656C20636F727219
:10501000656374004D65736820426564204C657655
:10502000656C696E670043616C69627261746520CA
:105030005A0043616C6962726174652058595A0064
:1050400053656C66746573740042656C7420746596
:1050500073740057697A6172640057697A61726487
:1050600020656E642073746174653A2025640A00BB
:1050700053706F6F6C4A6F696E004669726D77612D
:10508000726500466C6173684169720057697A61A4
:1050900072642073746174653A2025640A0045784F
:1050A000706572696D656E74616C004673656E73D0
:1050B0006F7220446574656374696F6E0044697330
:1050C00061626C65206661726D206D6F6465004D74
:1050D0003834004D3434004732382057004E6F20AA
:1050E000307846462072656365697665640053656D
:1050F0006E64696E67203078464600202225732250
:10510000002025236C78004449525F4558495400DB
:105110004449525F454E5445523A2025732022257A
:1051200073220A0046696C652073656C656374655B
:1051300064002053697A653A200046696C65206FE7
:1051400070656E65643A20004E6F772066726573F5
:10515000682066696C653A20004E6F7720646F693D
:105160006E672066696C653A20002220706F7300BC
:105170002220706172656E743A2200535542524F7C
:105180005554494E452043414C4C2074617267652B
:10519000743A2200747279696E6720746F206361BB
:1051A0006C6C207375622D67636F64652066696C33
:1051B0006573207769746820746F6F206D616E79F4
:1051C000206C6576656C732E0046696C616D656E4A
:1051D000742073656E736F7220626F6172642063F6
:1051E00068616E67652064657465637465643A2000
:1051F0007265766973696F6E25530A0053442063A4
:10520000617264206F6B006F70656E526F6F7420F7
:105210006661696C656400766F6C756D652E696E8C
:105220006974206661696C656400534420696E6925
:1052300074206661696C006F70656E206661696CD0
:1052400065642C2046696C653A200043616E6E6F80
:105250007420656E746572207375626469723A2099
:1052600000536F7274696E672066696C65730053D2
:105270006F6D652066696C65732077696C6C206E54
:105280006F7420626520736F727465642E204D61A7
:10529000782E204E6F2E206F662066696C65732015
:1052A000696E203120666F6C64657220666F7220B3
:1052B000736F7274696E67206973203130302E000D
:1052C00046696E697368696E67206D6F76656D6596
:1052D0006E7473004272696768746E65737300411F
:1052E00073736973740053696C656E74004F6E63F9
:1052F00065004C6F756400536F756E64004D4D55BD
:10530000204D6F6465004372617368206465742E7C
:1053100000537465616C7468004E6F726D616C004F
:1053200046616E7320636865636B005061757365D9
:1053300000436F6E742E00465320416374696F6E94
:105340000046696C2E2073656E736F72004368614E
:105350006E67652066696C616D656E7400466C6F82
:1053600077005370656564004E2F41004D61676E94
:1053700065747320636F6D702E005A2D70726F62AA
:1053800065206E722E004D6573680054696D656FFF
:10539000757400427269676874004D6F64650041FE
:1053A00075746F0044696D004C6576656C204469C6
:1053B0006D6D6564004C6576656C20427269676846
:1053C000740046616E207370656564004265640018
:1053D0004E6F7A7A6C650053657474696E677300FA
:1053E0005072696E742061626F72746564005374E8
:1053F0006F70207072696E7400436865636B696ECC
:10540000672066696C650046696C6520696E636F2C
:105410006D706C6574652E20436F6E74696E756572
:1054200020616E797761793F000452656672657319
:1054300068004D61696E004D363030004D203834C3
:10544000004D3834004D3234004D32332025730086
:10545000052E2E002F2F20616374696F6E3A6361F1
:105460006E63656C0046696C616D656E74206F7566
:1054700074206F662072616E6765202564200A00C3
:105480000000803F555585410000803F0000C84125
:1054900000000040555505420000C03F0000484252
:1054A0000000204055558542000070C1ABAAA642BD
:1054B000000060C10000A0410000C0C00000204109
:1054C00000002041ABAA3A41000020C15555D5400B
:1054D000000048C2555505424D3730312045340053
:1054E0004D373031204533004D37303120453200C3
:1054F0004D373031204531004D37303120453000B7
:1055000046696C616D656E74206E72206F757420D3
:105510006F662072616E67652100206661696C6547
:10552000642E00207375636365656465642E004DA9
:105530004D552063616E5F6C6F61643A0041646435
:105540006974696F6E616C206C6F61642061747442
:10555000656D7074206E722E2025640A00773235D6
:10556000783230636C5F63666D0A0077323578326B
:1055700030636C5F656E7465720A00737461727477
:105580000A0043757474696E672066696C616D65A5
:105590006E7400506C656173652072656D6F766521
:1055A0002066696C616D656E7420616E642074683C
:1055B000656E20707265737320746865206B6E6F02
:1055C000622E00456A656374696E672066696C6166
:1055D0006D656E74004D4D55206C6F616420666181
:1055E000696C65640020746F6F206C6F6E67206556
:1055F0007874727573696F6E2070726576656E74FB
:1056000065640020636F6C642065787472757369DB
:105610006F6E2070726576656E7465640020413A25
:105620000020503A002042403A0020403A00202F0B
:1056300000205400202F0020423A00202F00543A2E
:1056400000206D6963726F6E7300457863657373D4
:1056500069766520626564206C6576656C696E6745
:1056600020636F7272656374696F6E3A20004265E1
:1056700064206C6576656C696E67206661696C652F
:10568000642E2053656E736F72207472696767654C
:1056900072656420746F6F20686967682E004265C8
:1056A00064206C6576656C696E67206661696C65FF
:1056B000642E2053656E736F7220646973636F6E1E
:1056C0006E6563746564206F72206361626C65202F
:1056D00062726F6B656E2E0020453A00205A3A00C8
:1056E00020593A0020453A00205A3A0020593A0001
:1056F000583A0067636F64655F4D373031206265EB
:1057000067696E0A00536F6D652070726F626C6519
:105710006D20656E636F756E74657265642C205ABA
:105720002D6C6576656C696E6720656E666F726359
:105730006564202E2E2E0020436F756E7420583A1B
:10574000200045303A25642052504D2050524E31B1
:105750003A25642052504D204530403A257520505E
:10576000524E31403A25640A00776F726C642063B0
:105770006F6F7264696E617465733A2028252E33E9
:10578000662C20252E33662C20252E3366290A0010
:1057900043757272656E7420706F73205A5F415842
:1057A00049533A252E33660A43757272656E74202A
:1057B000706F7320455F415849533A252E33660A6E
:1057C0000041667465722077616974696E6720664E
:1057D0006F722074656D703A0A43757272656E74EB
:1057E00020706F7320585F415849533A252E336615
:1057F0000A43757272656E7420706F7320595F4131
:105800005849533A252E33660A007265636F7665F0
:10581000725F6D616368696E655F73746174655F03
:1058200061667465725F706F7765725F70616E69D3
:10583000632C20696E697469616C20005052555365
:10584000412075766C6F004734205330004D32365E
:105850002053256C75004D3130362053004D3232C7
:10586000302053256400473120462564004D3832EE
:10587000004739322045004731204525302E336618
:10588000204632373030004D3230342050256620EB
:1058900052256620542566004731205A256600505F
:1058A00052555341204D424C20563100473120582B
:1058B00025662059256620463330303000506F73FE
:1058C0006974696F6E20726561642066726F6D2005
:1058D000656570726F6D3A004D3233202573002E6E
:1058E00067636F002C20666565646D756C74697004
:1058F0006C793A0046656564726174653A004731B7
:105900002045252D302E3366204632373030004773
:10591000312045352046313230004D3833004D318D
:10592000303920532564004D31393020532564002F
:105930004D313034205325640047323820582059E7
:10594000004731205A252E33662046383030004734
:1059500031205A252D302E33662046252D302E330A
:10596000660047312045252D302E336620463237DC
:105970003030004D38330000002110422063308465
:1059800040A550C660E770088129914AA16BB18C8F
:10599000C1ADD1CEE1EFF13112100273325222B516
:1059A000529442F772D662399318837BB35AA3BDDF
:1059B000D39CC3FFF3DEE36224433420040114E6E6
:1059C00064C774A44485546AA54BB528850995EE2F
:1059D000E5CFF5ACC58DD55336722611163006D7F6
:1059E00076F6669556B4465BB77AA719973887DF7F
:1059F000F7FEE79DD7BCC7C448E5588668A778403E
:105A000008611802282338CCC9EDD98EE9AFF948CE
:105A10008969990AA92BB9F55AD44AB77A966A7155
:105A20001A500A333A122AFDDBDCCBBFFB9EEB791E
:105A30009B588B3BBB1AABA66C877CE44CC55C22A5
:105A40002C033C600C411CAEED8FFDECCDCDDD2A6E
:105A5000AD0BBD688D499D977EB66ED55EF44E1335
:105A60003E322E511E700E9FFFBEEFDDDFFCCF1BBE
:105A7000BF3AAF599F788F8891A981CAB1EBA10C29
:105A8000D12DC14EF16FE18010A100C230E320049E
:105A900050254046706760B9839893FBA3DAB33D05
:105AA000C31CD37FE35EF3B1029012F322D23235EE
:105AB00042145277625672EAB5CBA5A89589856ED5
:105AC000F54FE52CD50DC5E234C324A0148104663E
:105AD00074476424540544DBA7FAB79987B8975FE5
:105AE000E77EF71DC73CD7D326F2369106B016578E
:105AF000667676154634564CD96DC90EF92FE9C82D
:105B000099E9898AB9ABA94458654806782768C0DD
:105B100018E1088238A3287DCB5CDB3FEB1EFBF944
:105B20008BD89BBBAB9ABB754A545A376A167AF12D
:105B30000AD01AB32A923A2EFD0FED6CDD4DCDAA94
:105B4000BD8BADE89DC98D267C076C645C454CA27D
:105B50003C832CE01CC10C1FEF3EFF5DCF7CDF9B24
:105B6000AFBABFD98FF89F176E367E554E745E93CD
:105B70002EB23ED10EF01E5265636F766572696E6D
:105B800067207072696E7400506C65617365207770
:105B9000616974006F6B0A0073746172740A004D5E
:105BA0004D5532206669726D776172652076657237
:105BB00073696F6E20696E76616C69642E20526520
:105BC0007175697265642076657273696F6E3A20CB
:105BD0006275696C64206E756D6265722025642043
:105BE0006F72206869676865722E004D4D55203DC3
:105BF0003E20276F6B270A004D4D55203D3E202744
:105C00006F6B270A002564004D4D55203D3E20272F
:105C10006F6B272C20726573756D65207072696ECD
:105C2000740A004D4D552072657472792061747448
:105C3000656D7074206E722E2025640A004D4D55DE
:105C4000203D3E20276F6B270A00410A004D4D552D
:105C5000203C3D202741270A004D363030004D368C
:105C60003030204155544F002568687500410A00C6
:105C70004D4D55203C3D202741270A0050300A0059
:105C80004D25640A004D4D55203C3D20274D25648F
:105C9000270A0057300A004D4D55203C3D2027571C
:105CA00030270A0053330A004D4D55203C3D202734
:105CB0005333270A0052300A004D4D55203C3D20F9
:105CC000275230270A004B25640A004D4D55203CD1
:105CD0003D20274B2564270A004525640A004D4DC9
:105CE00055203C3D2027452564270A0055300A00F1
:105CF0004D4D55203C3D20275530270A0043300AA2
:105D0000004D4D55203C3D20274330270A004C25AF
:105D1000640A004D4D55203C3D20274C2564270A40
:105D2000005425640A004D4D55203C3D2027542544
:105D300064270A004D4D55202D20454E41424C45CB
:105D40004400256868750050300A004D310A004D46
:105D50004D55203C3D20274D31270050300A004D45
:105D60004D552076657273696F6E2076616C69643B
:105D7000004D4D55203D3E202725646F6B270A00BE
:105D800025750053320A004D4D55203C3D202753C8
:105D90003227004D4D55203D3E202725646F6B274F
:105DA0000A002575004D4D55206E6F742072657385
:105DB000706F6E64696E67202D2044495341424CD8
:105DC00045440053310A004D4D55203C3D2027539A
:105DD0003127004D4D55203D3E202773746172746C
:105DE00027006572726F723A20756E6B6E6F776EF8
:105DF000206D6F7665006E6F206D6F766500542D97
:105E0000636F646500756E6C6F6164006C6F6164D4
:105E1000006D6D755F6765745F726573706F6E732B
:105E200065202D20626567696E206D6F76653A206A
:105E3000006D6D755F6765745F726573706F6E730B
:105E40006528292072657475726E696E673A20251F
:105E5000640A00556E6C6F6164696E672066696ED6
:105E60006973686564203200556E6C6F616420321E
:105E700000556E6C6F6164696E672066696E697348
:105E8000686564203100556E6C6F61642031004D8F
:105E90004D552073746172747320726573706F6EE8
:105EA00064696E67004D4D55206E6F742072657386
:105EB000706F6E64696E6700506C65617365207504
:105EC0007064617465206669726D776172652069BE
:105ED0006E20796F7572204D4D55322E20576169B5
:105EE00074696E6720666F722072657365742E0028
:105EF0004D4D55204F4B2E20526573756D696E6761
:105F00002E2E2E004D4D55204F4B2E205265737571
:105F10006D696E6720706F736974696F6E2E2E2EB7
:105F2000004D4D55204F4B2E20526573756D696E97
:105F3000672074656D70657261747572652E2E2EA2
:105F400000466978207468652069737375652061FF
:105F50006E64207468656E2070726573732062755C
:105F600074746F6E206F6E204D4D5520756E697480
:105F70002E00507265737320746865206B6E6F62BB
:105F800020746F20726573756D65206E6F7A7A6C00
:105F9000652074656D70657261747572652E004D53
:105FA0004D55206E6565647320757365722061744C
:105FB00074656E74696F6E2E0025632533642F251A
:105FC000642563002F2F20616374696F6E3A7061DE
:105FD000757365002573202534642052504D0A25C1
:105FE00073202534642052504D0A00686F77746F17
:105FF0002E707275736133642E636F6D00666F72FD
:10600000756D2E707275736133642E636F6D0070E1
:106010007275736133642E636F6D005072696E74B4
:106020002046414E004E6F7A7A6C652046414E0004
:106030004D4D5520706F776572206661696C7300F5
:106040004D4D55206C6F6164206661696C73004D25
:106050004D55206661696C7300546F74616C2066E5
:1060600061696C757265730043726173680046699B
:106070006C2E2072756E6F75747300506F77657239
:10608000206661696C75726573004C617374207071
:1060900072696E74206661696C7572657300546F05
:1060A00074616C004C617374207072696E7400418D
:1060B0006D6269656E740044756D70206D656D6FFD
:1060C000727900566F6C74616765730054656D700A
:1060D00065726174757265730042656C74207374C7
:1060E000617475730053656E736F7220696E666FAD
:1060F00000457874727564657220696E666F005829
:10610000595A2063616C2E2064657461696C730058
:10611000756E6B6E6F776E004D4D553220636F6EEE
:106120006E656374656400446174653A00746F2041
:10613000756E6C6F61642066696C616D656E74006C
:10614000746F206C6F61642066696C616D656E743C
:1061500000507265737320746865206B6E6F620007
:1061600050726568656174696E6720746F2063752D
:10617000740050726568656174696E6720746F2081
:10618000656A6563740050726568656174696E67FD
:1061900020746F20756E6C6F616400507265686565
:1061A0006174696E6720746F206C6F6164002553A1
:1061B0000A20252D31362E313653252D33640A2001
:1061C000252D31362E313653252D33640025530AC3
:1061D00020252D31362E313653252D33640A2025C6
:1061E0002D31362E313653252D33640A20252D319D
:1061F000362E313653252D33640025530A20252DA4
:1062000031362E313653252D33640A20252D313673
:106210002E313653252D33640A20252D372E375342
:106220005820252D336420205920252D336400204B
:10623000257325336401200A000A204952203A20A0
:1062400020202020202025332E3166560020505754
:10625000523A20202020202025342E3166560A2054
:106260004245443A20202020202025342E316656F5
:106270000025530A20582025640A2059202564004F
:1062800025752E25752E25752E2575002573002064
:10629000005072696E7465722049502041646472C6
:1062A0003A002573002000466C61736841697220D2
:1062B000495020416464723A004D4D5532202020EF
:1062C000202020204E2F410025642E25642E256499
:1062D0002D2564002046573A0046696C2E207365D0
:1062E0006E736F7220762E3A004665622031372039
:1062F0003230323200453344763666756C6C004578
:10630000494E53795F31306100315F37356D6D5FD4
:106310004D4B33002D2D2D2D2D2D2D2D2D2D2D2D96
:106320000020332E31302E312D3436393700466976
:10633000726D776172653A004D373032004D3730FB
:1063400031004D373032004D373031007C3C3E3F1C
:106350002F2A225C004D494E54454D50004D494E68
:1063600054454D502042454400452D6D6F746F7269
:106370002063757272656E74207363616C696E67F9
:1063800020656E61626C656400746D633231333018
:106390005F686F6D655F656E74657228617865739F
:1063A0005F6D61736B3D307825303278290A007457
:1063B0006D63323133305F686F6D655F6578697426
:1063C00020746D63323133305F73675F686F6D695E
:1063D0006E675F617865735F6D61736B3D307825C3
:1063E0003032780A00544D432044524956455220D9
:1063F0004F56455254454D50004D3234004D3233C6
:10640000202573006175746F25692E670022206650
:1064100061696C65643A20427566666572206675CE
:106420006C6C2100456E717565696E6720746F2014
:106430007468652066726F6E743A2022004572722D
:106440006F723A002200456E717565696E6720743F
:106450006F207468652066726F6E743A2022006542
:1064600063686F3A00454550524F4D204572726F38
:1064700072004D494E54454D5020424544206669B6
:10648000786564004D494E54454D5020484F544561
:106490004E4420666978656400200A200A2000477F
:1064A00039390044697361626C65206661726D20E0
:1064B0006D6F64653F004C6F616420616C6C0050CF
:1064C0006C656173652070756C6C206F75742066E7
:1064D000696C616D656E7420696D6D656469617468
:1064E000656C7900556E6C6F6164696E67206669D2
:1064F0006C616D656E740052657365740052656EF3
:10650000616D65004669727374206C6179657220F3
:1065100063616C2E0053656C65637400537465652C
:106520006C2073686565747300537570706F727456
:10653000004661696C207374617473204D4D550081
:106540004661696C2073746174730053746174697B
:1065500073746963730043616C6962726174696F1B
:106560006E004175746F4C6F61642066696C616D7B
:10657000656E74004375742066696C616D656E7438
:1065800000456A6563742066696C616D656E7400B0
:10659000556E6C6F61642066696C616D656E740028
:1065A0004C6F616420746F206E6F7A7A6C65004C5A
:1065B0006F61642066696C616D656E74004E6F205A
:1065C00053442063617264005072696E7420667275
:1065D0006F6D20534400526573756D65207072694C
:1065E0006E74005061757365207072696E7400502E
:1065F0007265686561740054756E65004C697665F6
:106600002061646A757374205A00496E666F207346
:10661000637265656E004572723A205052494E545D
:106620002046414E204552524F52004572723A2048
:10663000455854522E2046414E204552524F52004A
:106640002F2F20616374696F6E3A70617573656492
:10665000002F2F20616374696F6E3A726573756DD8
:106660006564002F2F20616374696F6E3A726573E1
:10667000756D650078797A63616C5F7370697261BA
:106680006C322063783D25642063793D2564207A4F
:10669000303D256420647A3D25642072616469750B
:1066A000733D25642061643D25640A005061747463
:1066B00065726E2063656E746572205B25662025A9
:1066C000665D2C206D6174636820256625250A00AF
:1066D000205B25662C2025665D5B25665D2066694E
:1066E0006E616C20636972636C650A00746D63325D
:1066F0003133305F676F746F5F737465702025642A
:10670000202564202564202564200A0057726974BE
:10671000696E6720746F2066696C653A200046696F
:106720006C6520616C7265616479206F70656E655F
:1067300064004E6F00596573004E6F74207370696A
:106740006E6E696E67005370696E6E696E670046A3
:10675000616E20746573740053656C667465737440
:10676000206661696C6564002573206C6576656CD4
:106770002065787065637465640046616C7365209C
:1067800074726967676572696E670046696C616DEE
:10679000656E742073656E736F72005377617070ED
:1067A00065640046726F6E742F6C65667420666156
:1067B0006E7300417869730041786973206C656E6F
:1067C000677468004C6F6F73652070756C6C6579C9
:1067D000004C65667420686F74656E642066616E37
:1067E0003F0046726F6E74207072696E742066612D
:1067F0006E3F00456E6473746F70206E6F74206816
:10680000697400456E6473746F70004D6F746F72BD
:1068100000456E6473746F707300576972696E67B8
:10682000206572726F72004265642F4865617465FD
:1068300072004E6F7420636F6E6E656374656400E2
:106840004865617465722F546865726D6973746F01
:106850007200506C6561736520636865636B3A0014
:1068600053656C6674657374206572726F72210073
:10687000526573656E640025533A20256C640A25C1
:10688000530A00536865657400252D392E39535B12
:10689000002563252D31382E3138732563000B0216
:1068A000F90111241FBECFEFD1E2DEBFCDBF00E062
:1068B0000CBF14E0A0E0B2E0EAE8F7E703E00BBFAA
:1068C00002C007900D92AC33B107D9F728E1ACE3D1
:1068D000B4E001C01D92A632B207E1F714E3C0E5AF
:1068E000D4E300E006C021970109802FFE010F9438
:1068F000A5BACF34D10780E00807A9F70F94D98251
:106900000D94B4BB0C9400642F923F924F925F920F
:106910006F927F928F929F92AF92BF92CF92DF92AF
:10692000EF92FF920F931F93CF93DF93CDB7DEB714
:10693000C454D1090FB6F894DEBF0FBECDBF80910D
:106940005D05823061F483E080935D058091B60C33
:10695000882319F00F94945002C00F949A5080919C
:10696000B6079091B707892B11F40C94126282E05C
:106970008093600286E691E10E943A648823C1F028
:1069800080918F05909190056AE270E005960F94D2
:1069900000BB009711F0DC011C9280918F05909153
:1069A000900505960E9458EA87E08093140716C068
:1069B00083E691E10E943A64811117C08FE591E16D
:1069C0000E943A64811111C0A1C00F94653B80916F
:1069D000D60C882309F490C01092140781E08093AC
:1069E00060020F94C87D0C94126200918F05109183
:1069F000900580E50E944E64882309F482C00E94BD
:106A00002F646B017C01BB24B394672B682B692B2B
:106A100009F4B12C83E50E944E64882381F00E9422
:106A20002F649B01AC01A8EEB3E00F949EB56B01FF
:106A30007C01AA24A394672B682B692B09F4A12C51
:106A40000E5F1F4F6AE270E0C8010F9400BB009711
:106A500011F0FC0110829801C9012F5F3F4FDC014A
:106A60004C914032C9F326E020931407B11008C0BE
:106A7000A11006C02C91222319F00E9458EA0BC0E5
:106A80008091F706811105C080E595E10E9452EAE8
:106A900002C01092140781E080939F0610929E0618
:106AA0000E94DAA389EB9CE00E94748DC114D1048A
:106AB000E104F10409F489CF0E94556FC60ED71E78
:106AC000E81EF91E84E0809360020E94556F6C15E9
:106AD0007D058E059F0510F00C9414600E94B59AF8
:106AE00081110C9414600E9457D381E00E9445BA32
:106AF00080E00E94EF99E9CF87E697E10E9452EA91
:106B00006DCFB12CC12CD12C760184CFC090A509BA
:106B1000D090A60986010554184F46E050E068E57C
:106B200071E1C8010F9417AE892B09F0F4C089E414
:106B300091E10E943A64882309F4B9C088E50E9473
:106B40004E64182F89E50E944E64811112600E94E4
:106B5000DAA319821A821B821C82FE01359681E11A
:106B6000DF011D928A95E9F748EC5FEA60E070E08A
:106B70008EEB9CE00E94EE8C811110923E040091FD
:106B80003E040F5F00933E048EEB9CE00E94748DE8
:106B900080913D04812B80933D0481E00E94B3A24B
:106BA0000E9482A282E00E94EF9910FF15C086E643
:106BB0009FE00F941DB561E0680F86E69FE00F949B
:106BC0003EB585E09FE00F942AB5BC016F5F7F4F13
:106BD00085E09FE00F9458B511FF15C088E69FE04F
:106BE0000F941DB561E0680F88E69FE00F943EB5F5
:106BF00083E09FE00F942AB5BC016F5F7F4F83E075
:106C00009FE00F9458B581E00E94B3A282E00E94F9
:106C1000EF99612FCE0101960E940E64CE0101967C
:106C20000E9458EA40E061E081E00F948A380E94B7
:106C3000DAA3033020F461E085E09EE035C0E09106
:106C4000DB17F0E0EE0FFF1FEF5FF84F11821082AD
:106C500080E00E94B3A20E9482A260913D04CE0116
:106C600001960E940E6410923D04CE0101960E948E
:106C7000759B61E080E00E94109C86ED95E60E9485
:106C8000FB9B8FE30E94FF9B60E080E00E94E3C6D5
:106C9000182F81E00E94B3A261E0112319F087EF61
:106CA0009DE002C08AEE9DE00E948E8A97CE8BE323
:106CB00091E10E943A64882379F060E070E080E816
:106CC0009FE30F94983B0E94E4F6882309F486CE54
:106CD00081E08093110282CE8EE291E10E943A64BB
:106CE000882309F47BCE1092110781E08093110272
:106CF00080915E05811103C00F9439176FCE8130EA
:106D000009F06CCE84E594E50E94C36A0E94E46BAE
:106D10000E94718C63CE44E050E069E271E1C801E9
:106D20000F9417AE892B09F007C186010154184F43
:106D300049E050E06FE171E1C8010F9417AE892B73
:106D4000C9F4F601E853F84F1081153429F01855AD
:106D5000143008F043CE01C013E04AE050E060E098
:106D600070E0C6018753984F0F94D1AB812F0F94D9
:106D7000296334CE49E050E065E171E1C8010F9428
:106D800017AE892B51F5F601E853F84F10811534F1
:106D900029F01855143008F021CE01C013E04AE064
:106DA00050E060E070E0C6018753984F0F94D1AB7C
:106DB000E12FF0E0E05BFA4F40E051E0008002C0DC
:106DC000569547950A94E2F7842F880F880F8150D3
:106DD0006823812F0F94226F01CE49E050E06BE0D1
:106DE00071E1C8010F9417AE892B09F0F7CDF601B8
:106DF000E853F84F8081853441F008EAB02EB80E90
:106E0000B3E0BB1508F4EACD02C013E0B12EEB2CC1
:106E1000F12C4701880C991CF401EB56FD4F1081B1
:106E2000012F0F70712E7294BFE07B22272D2770E7
:106E3000722E111F1127111F61816770660F162BAB
:106E4000F401EA56FD4F9081A92EA694A694A6942B
:106E50003A2D3370A32E1A821982C6018753984F98
:106E6000DC012C912223E1F14AE050E0BE016F5F8A
:106E70007F4F0F94D1AB062F0F7089819A810097B5
:106E800079F1FC012081222359F14AE050E0BE0152
:106E90006F5F7F4F0F94D1AB6770762E89819A8197
:106EA0000097F1F0DC012C912223D1F04AE050E070
:106EB000BE016F5F7F4F0F94D1AB162F1F7089817A
:106EC0009A81009769F0FC012081222349F04AE071
:106ED00050E0BE016F5F7F4F0F94D1AB6370A62E61
:106EE000F401EB56FD4F272D27702295207F612F4F
:106EF000679566276795202B262B2083212F2695C3
:106F00001181107E9A2D9370990F990F990F122B62
:106F1000192B1183C701865E9D4FD701A25EBD4F1D
:106F2000B701605B7A4FFC0120814C91DB016C91D1
:106F30008B2D0F94785B52CD85E091E10E943A64ED
:106F4000882309F4C6C180E091E10E943A64882355
:106F500081F08091F706882309F440CD0E94556F97
:106F60006093D00C7093D10C8093D20C9093D30C7F
:106F700035CD8CEF90E10E943A64882341F08091F6
:106F8000D9061F928F938EE398E00C941E4182EFF6
:106F900090E10E943A64882309F43FC01092B7063A
:106FA00014E6C12CD12C76016F9A779864E170E0D9
:106FB00080E090E00E941D6F0E94F76E4B015C0123
:106FC000F8946F98679BFECF78940E94F76EDC016F
:106FD000CB0188199909AA09BB09C816D906EA067E
:106FE000FB0610F46C017D011150F1F68FED9DE070
:106FF0000E94C36AB5EFCB16B1E0DB06E104F104F1
:1070000018F08BED9DE002C088ED9DE00E94C36A00
:107010000E94E46B6F98779AE1CC8EEE90E10E942B
:107020003A648823D9F040911805509119052CE352
:10703000249FC001259F900D11249F938F93409111
:10704000160550911705249FC001259F900D11240E
:107050009F938F9387E298E00C94F05F8AEE90E123
:107060000E943A64882319F010925A05B7CC85EE35
:1070700090E10E943A64882349F060E085EA9FE04D
:107080000F943EB561E081EE90E10ECE8AED90E185
:107090000E943A64882319F00F94B7469FCC84ED80
:1070A00090E10E943A64882381F08AEA95E5DC0148
:1070B0008093FC1F9093FD1FA093FE1FB093FF1FB2
:1070C00088E08093FB1F0E94E26383E293E00E94CA
:1070D0003A64882381F180918F059091900561E059
:1070E00003960F949E0D85E69FE00F9433548C0118
:1070F00080916D0F90916E0FA0916F0FB091700FF6
:107100008093E90F9093EA0FA093EB0FB093EC0FED
:10711000802F0E94AB6A0A30110529F785E69FE0AF
:107120000F94125585E69FE00F948E561092D40C62
:107130001092D50C53CC81ED90E10E943A648823E3
:10714000A1F044E150E065E17DE0CE0101960F94AD
:107150000DB58C89882321F086EC90E10C94645E57
:10716000CE0101960F9484BB39CC82EC90E10E9451
:107170003A64882319F086E293E008C08EEB90E130
:107180000E943A64882329F082E393E00E94F16B25
:1071900025CC89EB90E10E943A6481111FCC86EBEB
:1071A00090E10E943A64882371F081EA9DE00F9497
:1071B0001DB5EBE08E9FC001112460E070E0805BA4
:1071C000924F0C941D6083EB90E10E943A648823F7
:1071D00051F00E9482A240E060E070E084E690E01E
:1071E0000F946923FBCB8FEA90E10E943A648823D5
:1071F000E1F086E50E944E64882309F4EFCB0E94FB
:10720000226411E0892B09F410E00E94DAA3212FF7
:1072100030E08091D20B90E02817390709F4DECBDB
:107220001093D20B0F94CA6FD9CB88EA90E10E94D9
:107230003A64882309F4D2CB84E40E944E64882304
:10724000A1F00F94B69020E030E04AE754E40F94A8
:1072500096A920E030E040E05FE30F94B8B50F94CA
:107260001DB7CB010F94D196B9CB84EA90E10E946F
:107270003A64882311F40C9421608091F7068823E6
:1072800011F40C94216080918F05909190050296E5
:107290009093900580938F050F94B6906B017C01BD
:1072A0006FEF87EA9DE00F943EB520E030E04AE7BB
:1072B00054E4C701B6010F9496A920E030E040E005
:1072C0005FE30F94B8B50F941DB785EA9DE00C9469
:1072D0001D6087E40E944E64182F882309F490C72C
:1072E0000E9422649093400480933F048B34910564
:1072F00009F414C208F077C08430910509F48AC1FA
:1073000048F42091F8068230910509F475C108F41B
:10731000AEC078C18531910509F46CC748F48A3054
:10732000910509F4BDC10B9709F04DC780E0B9C1C3
:107330008C31910509F4B8C14E9709F044C70E94F9
:10734000DAA381E08093C6060E9469638C0180E025
:1073500090E0A8E4B4E480939E0290939F02A093EF
:10736000A002B093A10243E060E070E080E291EC03
:107370000F9423708091D5178F938091D4178F939A
:107380008091D3178F938091D2178F938091D117CB
:107390008F938091D0178F938091CF178F93809187
:1073A000CE178F938091CD178F938091CC178F93A9
:1073B0008091CB178F938091CA178F932CEC33E574
:1073C0003F932F9322E038E03F932F930F9437AFF2
:1073D000C8010E944F631092C6060FB6F894DEBF34
:1073E0000FBECDBF07C78835910509F403C7C0F4A8
:1073F0008135910509F4EAC548F48C34910509F406
:10740000B0C18035910509F4DEC5DDC6863591052C
:1074100009F431C68735910509F0D5C681E02CC63F
:107420008C35910509F431C660F48A35910509F46B
:1074300026C68B35910509F0C6C680911307876073
:1074400021C68236910509F4A1C68336910509F05B
:10745000BAC61092F70681E080935B0260E084EC8C
:107460009FE00F943EB582E00E94EF99A9C62111DA
:10747000C1C60F9496A820E030E040E85FEB609131
:1074800065027091660280916702909168020F9484
:107490002DB08823F9F0E091A509F091A609E854F0
:1074A000F84F80818B7F8230A9F480E1E5E6F2E03D
:1074B000A2E4B7E001900D928A95E1F780E090E0B8
:1074C000A0E8BFEB8093650290936602A0936702E9
:1074D000B0936802609116077091170780911807A2
:1074E000909119070F9431B06B017C014090D61731
:1074F0005090D7176090D8177090D91780904E078A
:1075000090904F07A0905007B0905107A5019401AB
:10751000C301B2010F94B7B520E030E048EC52E46B
:107520000F9496A99B01AC01C701B6010F9403B853
:107530001816E4F4A3019201C501B4010F94B7B584
:1075400020E030E048EC52E40F9496A99B01AC0196
:10755000C701B6010F94B8B50F941DB76093160715
:1075600070931707809318079093190780918817D5
:10757000882309F43EC088E50E944E64811139C019
:1075800089E50E944E64811134C08AE50E944E64F0
:1075900081112FC085E40E944E64882351F120910F
:1075A000D6173091D7174091D8175091D9176091BD
:1075B0004E0770914F0780915007909151070F949B
:1075C000B7B56B017C012DEC3CEC4CEC5DEB0F9402
:1075D0002DB087FF02C00C9434602DEC3CEC4CECD9
:1075E0005DE3C701B6010F9403B8181614F40C94A8
:1075F0003D600F94A2A6FEC52111FCC50F9461A9A0
:1076000081E005C02111F6C50F9461A980E00F94B7
:1076100043A3F0C580E50E944E64882339F00F949F
:10762000B6900F941DB76B017C0103C0C12CD12C07
:10763000760183E50E944E64882361F00F94B69032
:1076400020E030E04AE754E40F9496A90F941DB768
:107650006B017C01C114D104E104F10421F08EE13D
:1076600098E00E9452EA0E94DAA30E94556FC60E6B
:10767000D71EE81EF91E89EB9CE00E94748D0E94C3
:10768000556F6C157D058E059F0508F0B3C50E94EA
:1076900057D380E00E9445BA80E00E94EF99EFCF77
:1076A00081E00F9450A1A6C588E50E944E648DA785
:1076B0000E942F641B012C0189E50E944E64682EF4
:1076C0000E942F6469AB7AAB8BAB9CAB8AE50E94BE
:1076D0004E64D82E0E942F644B015C0187E50E9406
:1076E0004E64782E83E40E944E647F928F93CD2C5B
:1076F000E9A8FAA80BA91CA9262DB201A1018DA504
:107700000F949F360F900F903DA5311173C56110F6
:1077100071C571106FC5D1106DC555C408E210E078
:10772000F9EFEF2EF7E0FF2E602F70E080E090E0A1
:107730000F9431B00E9496B49F938F937F936F9371
:107740001F930F93FF92EF920F9437AF0F5F1F4F6E
:107750000FB6F894DEBF0FBECDBF0F36110521F76F
:1077600049C520E030E040E251E46091F3067091B9
:10777000F4068091F5069091F6060F9403B887FF02
:1077800003C080E990E172C40E94036A8A3F28F036
:107790008EE295E10E94AFC82DC5809188058823AF
:1077A00041F080918905882321F080918A0581111B
:1077B00008C081E08093B50789E890E10F94DB640D
:1077C00019C587EE94E10E94AFC840E060E08AEE00
:1077D00090E20E949EC8882309F45FC080E090E098
:1077E000A0EAB0E48093D2179093D317A093D41754
:1077F000B093D51760E070E088E492E40F948519A7
:1078000080E090E0A8E4B2E48093D2179093D3177D
:10781000A093D417B093D51780E090E0A4E3B3E42D
:107820008093CE179093CF17A093D017B093D11712
:1078300060E070E088E492E40F9485190E94DAA376
:1078400082EC90E20E94AFC8E2EBF3E28591959161
:10785000A591B4918093CE179093CF17A093D01792
:10786000B093D117EEEAF3E285919591A591B49189
:107870008093CA179093CB17A093CC17B093CD17D2
:1078800060E070E088E492E40F9485190E94DAA326
:1078900041E060E080E00F948A3820E030E04CE086
:1078A00052E46091F3067091F4068091F506909190
:1078B000F6060F9403B818160CF07CC08091F706FA
:1078C000811178C080E090E0A8ECB2E48093D217F8
:1078D0009093D317A093D417B093D51760E070E0BE
:1078E00088E492E40F94851980E090E0ACE0B2E483
:1078F0008CA39DA3AEA3BFA319821A821B821C82F4
:10790000CE0101960F94E606109200071092FF0632
:1079100019821A821B821C821D82CE0101960E944E
:10792000748D2CA13DA14EA15FA16091F3067091D1
:10793000F4068091F5069091F6060F9403B8181698
:107940007CF58CE994E10E9486C864E080E00E94A6
:10795000109C82E00E94328783EF96E00E94378A73
:107960000E94759B8FE20E943287CE0184960E940E
:10797000378A0E94759B81E00E94328788EE93E0EF
:107980000E949BBE0E94DFB340E053E567E070E0D9
:10799000CE0101960E94EE8C882319F210E001C0FE
:1079A00011E081E00E94B3A2111104C080E00F94A5
:1079B000139820C40E94DAA311E01093C60681E058
:1079C0000E94B3A2109360028BE690E10E94C36A0A
:1079D0000E94E46BC090F306D090F406E090F506A8
:1079E000F090F60620E030E040EA50E4C701B6012E
:1079F0000F94A6B60F9417B725E0269FA001279FE6
:107A0000500D1124BA01550F880B990B0F9433B008
:107A10001B012C0120E030E04CE052E40F942DB02B
:107A200087FF06C0212C312C7CE0472EE2E45E2E3D
:107A3000A7019601622D732D842D952D0F942DB0E5
:107A400087FF0CC020E030E040EA50E4622D732D47
:107A5000842D952D0F94B8B51B012C015F924F9288
:107A60003F922F9280EE97E09F938F930F9437AFC2
:107A700020E030E040EF51E4622D732D842D952DF0
:107A80000F94B7B520E030E04CE852E40F94B8B55D
:107A90000F9417B7709300076093FF0684E08093FC
:107AA000140781E08093AD0687E79FE40E9452EAC5
:107AB00080E090E0A0EAB0E48093D2179093D317CF
:107AC000A093D417B093D51760E070E088E492E4F7
:107AD0000F94851980E090E0A0EAB1E48093CA1782
:107AE0009093CB17A093CC17B093CD1780E090E084
:107AF000A0E7B2E48093CE179093CF17A093D0174E
:107B0000B093D11760E070E088E492E40F94851997
:107B10008AE999E9A9E1BEE38093D2179093D3173C
:107B2000A093D417B093D51760E070E088E492E496
:107B30000F9485190E94DAA30F900F900F900F9069
:107B40000F900F90222D332D442D552D6091F3066B
:107B50007091F4068091F5069091F6060F942DB081
:107B600087FF07C088EE93E00E949BBE0E94DFB3B0
:107B7000E9CF60E086EA9FE00F943EB580E090E0B8
:107B8000A0EAB0E48093D2179093D317A093D417B0
:107B9000B093D51760E070E088E492E40F94851903
:107BA000EEEAF3E285919591A591B4918093CA177D
:107BB0009093CB17A093CC17B093CD17E2EBF3E2E1
:107BC00085919591A591B4918093CE179093CF17FD
:107BD000A093D017B093D11760E070E088E492E4EE
:107BE0000F9485190E94DAA343E060E070E080E81A
:107BF0009FEB0F942370882309F4E0C1B091D21752
:107C0000BDA7E091D317E9ABF091D417FDAB20915C
:107C1000D51729AF2F93FF93EF93BF9383ED97E091
:107C20009F938F930F9437AF0F900F900F900F90FB
:107C30000F900F904EEAC42E4FE0D42EAA24AA949F
:107C4000BA2C63E2E62EF12C812C912C8501B70130
:107C50000F2C000C880B990B0F9433B09B01AC01D7
:107C60003401AFEF6A1A7A0AFF92EF927F926F9215
:107C7000A7E9B7E0BF93AF9322966FAF2297239601
:107C80003FAF239724964FAF249725965FAF259754
:107C90000F9437AF0F900F900F900F900F900F90A1
:107CA00022962FAD229723963FAD239724964FAD72
:107CB000249725965FAD2597FFEFAF16BF0611F409
:107CC0000C94F96160E070E0C6010F9458B52296FB
:107CD0002FAD229723963FAD239724964FAD24973F
:107CE00025965FAD2597622D732D842D952D0F94CC
:107CF0002DB018168CF425E08216910459F035E069
:107D0000E30EF11C8FEFA81AB80A92E0C90ED11C3D
:107D100043019CCF05E010E078013FEFE31AF30A3E
:107D20006801CC0CDD1C25E0209FC001219F900D37
:107D30001124212C312CDC019D962196BFAFAEAFD2
:107D40002197412C512C30EA632E31E4732E35E01B
:107D5000E316F1040CF031C121966EAD7FAD219791
:107D6000620D731D072E000C880B990B0F9433B016
:107D70004B015C01C70102969F938F93AAE8B7E07D
:107D8000BF93AF930F9437AF82E08E0D8093AD0613
:107D900020E030E040EF51E4C501B4010F94B7B5E5
:107DA00020E030E040E251E40F9496A920E030E07A
:107DB00040EA50E40F94A6B620E030E048E452E4F4
:107DC0000F94B8B50F9417B7709300076093FF0630
:107DD00080E090E0A0EAB0E48093D2179093D317AC
:107DE000A093D417B093D51760E070E088E492E4D4
:107DF0000F9485194092CA175092CB176092CC17F6
:107E00007092CD1780E090E0A0E7B2E48093CE17A7
:107E10009093CF17A093D017B093D11760E070E084
:107E200088E492E40F9485198AE999E9A9E1BEE30F
:107E30008093D2179093D317A093D417B093D517EC
:107E400060E070E088E492E40F9485190E94DAA360
:107E50000F900F900F900F90A50194016091F30681
:107E60007091F4068091F5069091F6060F942DB06E
:107E700087FF07C088EE93E00E949BBE0E94DFB39D
:107E8000EBCF80E090E0A0EAB0E48093D21790932B
:107E9000D317A093D417B093D51760E070E088E4AF
:107EA00092E40F948519EEEAF3E285919591A591FC
:107EB000B4918093CA179093CB17A093CC17B0932B
:107EC000CD17E2EBF3E285919591A591B491809362
:107ED000CE179093CF17A093D017B093D11760E02F
:107EE00070E088E492E40F9485190E94DAA343E0DD
:107EF00060E070E080E89FEB0F942370460192E011
:107F0000890E911CA5E02A0E311C811103C00F942B
:107F1000139853C07DA569A99DA989AD272F362F38
:107F2000492F582F6091D2177091D3178091D41791
:107F30009091D5170F94B7B5162F072FB82EA92EED
:107F40002091121730911317409114175091151763
:107F5000D801F5016B2F7A2F8F2F9E2F0F9496A9A2
:107F60000F9417B76BAF7CAF8DAF9EAFAF92BF9240
:107F70000F931F938091F6068F938091F5068F9350
:107F80008091F4068F938091F3068F93AEE5B7E06E
:107F9000BF93AF930F9437AF6BAD7CADC6018E54DA
:107FA000904F0F9458B5FFEFEF1AFF0A0FB6F894F1
:107FB000DEBF0FBECDBF6401CACE81E00F9413981F
:107FC0001092C60617C10F94B89814C18091D20BB5
:107FD000882309F449C081E690E10E94C36A67E002
:107FE00070E080E090E00E94556B8CE20E94AB6AEA
:107FF00067E070E080E090E00E94556B8EE490E1D5
:108000000E94C36A42E060E070E080EA90E40E946F
:108010006F6B8CE390E10E94C36A0E94E46B97E06F
:10802000F92EFA948FEFF81609F4E4C09CE1F99E5A
:108030006001112400E010E089E390E10E94C36A2E
:10804000F801EC0DFD1DEE52F44F618172818381C8
:10805000948145E00E946F6B0C5F1F4F0C3111053E
:1080600059F70E94E46BDDCF8BE190E10E94C36A77
:108070000E94E46BBFC086EE0E94FE69BBC0809187
:108080001307887F80931307B5C06E01A4E2CA0E60
:10809000D11CFE0131967F0146010FE113E05F0123
:1080A00084E0782E700ED8018D918D010E944E646F
:1080B000F40181934F01882341F00F94B690D701CA
:1080C0006D937D938D939C931397B4E0EB0EF11C0D
:1080D0007012E9CFFFA0FF2001F120E030E0A901FC
:1080E0006D857E858F8598890F942DB0811115C07F
:1080F0008CA1811112C08DA181110FC08EA181119F
:108100000CC01092D6171092D7171092D817109251
:10811000D91781E0809320056DC00E94DAA300E0AA
:1081200010E0F60181916F018823D1F09801265368
:10813000384E4901F801E25AF84E208131814281DE
:108140005381F501E00FF11F60817181828193817C
:108150000F94B8B5D4016D937D938D939C93139731
:108160000C5F1F4F0C301105E1F6FF2061F08D858B
:108170009E85AF85B8898093D6179093D717A09323
:10818000D817B093D9170F94163434C081E0809378
:10819000F7060E94556F6093D00C7093D10C8093BA
:1081A000D20C9093D30C6091F70684EC9FE00F946F
:1081B0003EB510920F0760E08FEF9FE00F943EB541
:1081C0000E943EF617C08091A5099091A60985549A
:1081D000984F9F938F931F9287E48F9389E497E042
:1081E0009F938F930F9437AF0F900F900F900F9036
:1081F0000F900F901092400410923F040C94EE34B4
:108200008DE40E944E64882311F40C94185EE09172
:108210008F05F0919005319691919032E9F3993064
:10822000D9F390539A30A0F08091A5099091A609B6
:108230008554984F9F938F9387E090E19F938F93FE
:108240000F9437AF0F900F900F900F900C94EE3467
:108250000E9422649093800780937F07883C910559
:1082600011F40C94CE4B08F04EC18934910509F4F9
:10827000F3C508F0C9C08B31910509F420C3B8F5E6
:108280008631910509F4B4C210F58231910511F4DB
:108290000C94584978F4419711F00C94FB5D8EEDE5
:1082A00094E10E9452EA179816980F942D3B149867
:1082B0000C94125E8431910509F45FC2459711F068
:1082C0000C94FB5D81E00F941F0F0C94125E8831BB
:1082D000910509F4B4C208F49BC28931910511F4E7
:1082E0000C94FE574A9709F4DCC20C94FB5D803273
:1082F000910509F45EC408F053C08D31910511F465
:108300000C94125E08F485C38E31910509F4ABC359
:108310004F9711F00C94FB5D0E94556F60932207FC
:1083200070932307809324079093250700911E07DD
:1083300010911F072091200730912107601B710BBE
:10834000820B930B28EE33E040E050E00F947CB5B5
:10835000CA01B9012CE330E040E050E00F947CB555
:108360007F936F933F932F9388EF9FE09F938F931B
:108370008E010F5F1F4F1F930F930F9490AF8FE5E8
:1083800094E60E94C36AC8010E94F16BC8010E9472
:1083900058EA0FB6F894DEBF0FBECDBF0C94125E44
:1083A0008D32910509F4EAC4F8F48A32910509F492
:1083B000A9C48C9711F00C94FB5D8FEF0E94FE69AD
:1083C00081EA9DE00F941DB53BE0839FC00111241D
:1083D00060E070E0805B924F0F9458B50E949A96CF
:1083E0000E947C960C94125E8E32910509F4CDC4E5
:1083F0008F9711F00C94FB5D84E0809360020E94E3
:1084000082A20E94DF69F2C48D36910509F436C656
:10841000F0F58635910509F49EC7D8F483359105AA
:1084200009F43FC760F48235910511F00C94FB5DAF
:1084300080911307877F809313070C94125E843515
:10844000910509F435C78535910509F469C70C9480
:10845000FB5D8936910509F4D7C550F48C3591053B
:1084600009F498C78836910509F499C50C94FB5D09
:108470008A36910509F4FFC68B36910511F00C94EC
:10848000FB5D1092DE171092DD170C94125E83379D
:10849000910511F40C94844AC8F48037910509F4CD
:1084A0009DC530F48E36910509F4FAC70C94FB5D36
:1084B0008137910511F40C94634A8237910511F0CC
:1084C0000C94FB5D0F9421360C94125E8C38910550
:1084D00009F489C570F48737910511F40C94684B41
:1084E0008B37910511F00C94FB5D0F94EC350C94D7
:1084F000125E8B39910509F49FC58E3B910509F4F5
:1085000033C60C94FB5D8339B1E09B0711F40C94E6
:108510008A5008F086C08D3D910511F40C94894E67
:10852000E0F58E3C910511F40C949C4D10F58B3CBC
:10853000910511F40C94704C80F4893C910511F074
:108540000C94FB5D6FE1C62E63E0D62E7AE2E72E37
:1085500077E1F72E10E00C94294C8C3C910511F436
:108560000C94C84C8D3C910511F40C94234D0C9443
:10857000FB5D803D910511F40C94F04D10F40C94CA
:10858000B94D813D910511F40C94184E8C3D910527
:1085900011F40C94494E0C94FB5D8E32F1E09F0770
:1085A00011F40C944050D0F4803F910511F40C94D8
:1085B000125E38F4823E910511F40C94BF4E0C9477
:1085C000FB5D8C3231E0930711F40C941E4F8D3219
:1085D000914011F40C94484F0C94FB5D8E35B1E042
:1085E0009B0711F40C94115D68F48F32F1E09F0742
:1085F00011F40C9455508033914011F40C94C44FF5
:108600000C94FB5D8F3531E0930711F40C94125EEE
:108610008039914011F00C94FB5D0E94DAA30C9418
:10862000125E8D3BB2E09B0711F40C94DF5D08F005
:1086300047C08D3FF1E09F0711F40C94AD53E8F46F
:10864000853F31E0930711F40C94CD5048F4843FFA
:10865000914011F00C94FB5D0E94706D0C94125EC1
:10866000863FE1E09E0711F40C94D150873F914082
:1086700011F40C94D5500C94FB5D893522E09207DF
:1086800011F40C94FE5768F48832A2E09A0711F4B2
:108690000C9429548835924011F40C945C540C9439
:1086A000FB5D8A35E2E09E0711F40C940B588B3584
:1086B000924011F00C94FB5D0F9439170C94125EEC
:1086C0008E3523E0920711F40C941F5AD8F48335A9
:1086D000A3E09A0711F40C94B75338F48E3B924000
:1086E00011F40C94EA5D0C94FB5D8C35F3E09F076C
:1086F00011F40C9412588D35934011F40C94BB581E
:108700000C94FB5D8C3833E0930711F40C94125EEB
:1087100090F48438B3E09B0711F40C940E5C8B3812
:10872000934011F00C94FB5DAFE1AA2EA3E0BA2EAA
:1087300010E00C94FA5C803AF3E09F0709F4B5C2AC
:10874000873E934011F00C94FB5D1092F806109256
:10875000C4068091080690910906A0910A06B0917E
:108760000B068093910590939205A0939305B09387
:1087700094050F94E47D0C94125E81E08093600276
:1087800089E397E00E94C36A0E94E46B84E50E943B
:108790004E64182F8CE40E944E6400E080FB00F9C8
:1087A00010FB01F940E050E0BA018CE59DE00F9428
:1087B000555583E2ECE5FDE0DE01119601900D9246
:1087C0008A95E1F720E040E050E0BE016F5F7F4F07
:1087D00080EC93E00F94F206CE0101960E94636450
:1087E0008BE297E00E94C36A0E94E46B0C94125ED5
:1087F0001092D60C1092D70C8FE594E60E94C36AB3
:1088000083E592E40E94C36A0E94E46B0C94125EBA
:1088100080918F05909190056AE270E004960F9424
:1088200000BB009711F0DC011C9280918F059091A4
:10883000900561E004960F949E0D0C94125E809159
:108840005F05882321F00F94DC6A0C94125E8091FE
:10885000680F882361F08091E90F9091EA0FA09151
:10886000EB0FB091EC0F892B8A2B8B2B29F40F94F3
:10887000609080E00E94AC878091D70C882329F01B
:1088800081E08093D60C1092F8060E94556F609399
:108890001E0770931F0780932007909321070C9465
:1088A000125E8091D70C882311F40C94125E83E53C
:1088B0000E944E6481110C9468600C94125E80E5F5
:1088C0000E944E6490915F059923C1F08091110739
:1088D000882361F080915E05811108C088EC9DE0DD
:1088E0000E94C36A0E94E46B0C94125E8CEB9DE0C4
:1088F0000E94C36A0E94E46B0C94125E9091D60CA5
:10890000992309F47EC0882329F00F945C060E9405
:10891000E46B0BC08091ED0C811103C088ED9CE0ED
:1089200002C08DEE9CE00E94F16B8AE096E00E940E
:10893000C36A6091E90F7091EA0F8091EB0F9091FB
:10894000EC0F4AE00E94D06A8FE20E94AB6A60910D
:10895000E20F7091E30F8091E40F9091E50F4AE0F0
:108960000E94D06A0E94E46B0E94556F00911E071E
:1089700010911F072091200730912107601B710B78
:10898000820B930B20E63AEE40E050E00F947CB56A
:10899000C9016CE370E00F9462BA7C01CB019927A6
:1089A0000AE010E0B8010F9476BA282FCB01B80185
:1089B0000F9476BA90E3980F9093EB06205D209386
:1089C000EC061092ED068BEE96E00E94E66B8AE3D1
:1089D0000E94AB6AC701B8010F9476BA282FCB0169
:1089E000B8010F9476BA805D8093EB06205D2093EA
:1089F000EC061092ED068BEE96E00E94F16B0C9463
:108A0000125E8CEA9DE00E94C36A0E94E46B0C94A3
:108A1000125E80918F05909190056AE270E0049655
:108A20000F9400BB8C01892BA9F08091A50990912E
:108A3000A6096EE470E08554984F0F9400BB60E285
:108A400070E00F9400BB01969093900580938F0582
:108A5000F801108280918F059091900504960F94F3
:108A6000D4A20C94125E8091D70C882311F40C943C
:108A7000125E85E69FE00F94125585E69FE00F9405
:108A80008E561092D40C1092D50C80918F05909137
:108A900090056AE270E004960F9400BB7C01892B7C
:108AA000A9F08091A5099091A6096EE470E0855423
:108AB000984F0F9400BB60E270E00F9400BB0196EA
:108AC0009093900580938F05D7011C92E0908F05BD
:108AD000F0909005B4E0EB0EF11C8091D70C882348
:108AE00011F40C94125E85E69FE00F948E5610925E
:108AF000D60CFDA2ECA2CE0184960F94080D88231B
:108B000011F40C94125E4CA15DA160917F0D7091E7
:108B1000800D19821C8222E0CE0101960F949E598D
:108B20008823F1F0CE0101960F9457668823C1F097
:108B30006D857E858F85988941E00E94F991882313
:108B400079F0E98920E2E29FF0011124E955F64F1E
:108B5000309731F085EE80831C820E94B991182FE6
:108B6000CE0101960E9463641123A1F08EE99DE07D
:108B70000E94C36A8CA19DA10E94F16B1092E90F23
:108B80001092EA0F1092EB0F1092EC0F0F942A0A3A
:108B90000C94125E86E89DE00E94C36A8CA19DA1A0
:108BA0000E94E66B8EE20E94AB6A0E94E46B0C941A
:108BB000125E8091D60C81110E94DAA300918F057C
:108BC000109190050C5F1F4F6AE270E0C8010F948E
:108BD00000BB7C0161E270E0C8010F9400BB00970C
:108BE00019F08C010F5F1F4FE114F10411F0D70150
:108BF0001C9280E50E944E64F82E80918F05909122
:108C000090050817190708F4F12C8091D70C8823D8
:108C100011F40C94125E61E06F25C8010F949E0D53
:108C200083E50E944E64882399F080918F0590918E
:108C300090058017910760F40E942F646093E90FFC
:108C40007093EA0F8093EB0F9093EC0F0F94C06436
:108C50008091D70C882329F081E08093D60C109264
:108C6000F806F1100C94125E8091680F882361F071
:108C70008091E90F9091EA0FA091EB0FB091EC0F6A
:108C8000892B8A2B8B2B29F40F94609080E00E9413
:108C9000AC870E94556F60931E0770931F078093E7
:108CA0002007909321070C94125E80918F0590917C
:108CB00090056AE270E005960F9400BB8C01892B49
:108CC000A9F08091A5099091A6096EE470E0855401
:108CD000984F0F9400BB60E270E00F9400BB0196C8
:108CE0009093900580938F05F801108280918F05F5
:108CF0009091900521E02093D50C05960F94D4A275
:108D00000C94125E83E50E944E64882311F40C9447
:108D1000125E0F94A990082F80E50E944E6488236C
:108D200021F00F94A990182F01C01DE0ECEDFFE099
:108D30008CE18E0F9491911711F40C94125E319680
:108D40008E13F8CF163039F4802F90E09093DE1711
:108D50008093DD1704C017FF02C00C94125E61E01F
:108D6000812F0E94D6F1602F812F0E94A7F1602FE2
:108D700070E0812F0E9412F20C94125E8AE50E942C
:108D80004E640E943B700C94125E8091460F8823C3
:108D900029F1CE0101960F94617B8823C9F0898166
:108DA0000E94AB6A8EE20E94AB6A8A810E94AB6A23
:108DB0008EE20E94AB6A8B810E94AB6A8EE20E94B7
:108DC000AB6A8C810E94AB6A0E94E46B0C94125EC9
:108DD0008CEB9FE00E94C36A0C94125E88EB9FE0CC
:108DE0000E94C36A0E94E46B0C94125E0E9457D3E7
:108DF00081E00E9445BA47E75DE060E080E00E94C4
:108E0000E19F1E9903C041E75DE002C044E75DE0D9
:108E100061E080E00E94E19F1D9903C04BE65DE0A8
:108E200002C04EE65DE062E080E00E94E19F1C9996
:108E300003C045E65DE002C048E65DE063E080E037
:108E40000E94E19F0E94B59A882381F20E9482A22B
:108E50000E9440D90C94125E80E50E944E648823E3
:108E600021F00F94A99080933B0282E50E944E640A
:108E7000882341F00F94B6900F941DB77093400271
:108E800060933F0281E50E944E64882321F00F9495
:108E9000A99080933A0283E50E944E64882341F0B2
:108EA0000F94B6900F941DB77093440260934302E1
:108EB00083E40E944E648823B1F00F947E906B018E
:108EC0007C0120E030E0A9010F942DB018162CF49D
:108ED000C701B6010F941DB702C06FEF7FEF70930B
:108EE0003E0260933D0284E40E944E648823B1F008
:108EF0000F947E906B017C0120E030E0A9010F947B
:108F00002DB018162CF4C701B6010F941DB702C07E
:108F10006FEF7FEF709342026093410280913E02B7
:108F20008F9380913D028F93809140028F93809127
:108F30003F028F9380913B02282F082E000C330BA9
:108F40003F938F9381ED96E09F938F9308ED16E00A
:108F50001F930F930F9437AF809142028F938091AC
:108F600041028F93809144028F93809143028F93AB
:108F700080913A02282F082E000C330B3F938F93D9
:108F80008AEC96E09F938F931F930F930F9437AFC4
:108F90000FB6F894DEBF0FBECDBF0C94125EBE01BB
:108FA0006F5F7F4F88E690E00F943F9681110C949D
:108FB000125E83E50E944E64882311F40C94125EC5
:108FC00019810F94B69011110C94125E0F9417B77B
:108FD00070930207609301070C94125E63E08CE7C4
:108FE00095E20E9402BA83E50E944E64882311F440
:108FF0000C94125E0F94B6900F9417B770930007FD
:109000006093FF060C94125EBE016F5F7F4F89E68E
:1090100090E00F943F9681110C94125E84EB9FE0D8
:109020000E94C36A89810F94AE380E941F8C81E030
:109030008093B5070C94125E83E50E944E648823EA
:1090400069F00F94A9908093B00C882329F081EBEC
:109050009CE00E94748D02C01092B10C83E40E94C7
:109060004E64882331F00F94A9908093AF0C0C9438
:10907000125E81E08093AF0C0C94125EBE016F5FB4
:109080007F4F8DE690E00F943F9681110C94125E15
:1090900086E29EE30E9452EA81E080939C068091E2
:1090A000F706882321F060E081E00E94FEFB83E563
:1090B0000E944E64811105C082E50E944E6488239F
:1090C00059F019810F94B690111106C00F9417B77B
:1090D00070930207609301070E94556F4B015C017A
:1090E000F9800F2D10E0F801EE0FFF1FEF5FF84F32
:1090F00080819181BC01990F880B990B0F9433B03B
:10910000F801EE0FFF1FEE0FFF1FE054F94F11E0C3
:1091100020813181428153810F9403B818160CF0DD
:1091200010E010930C0681E0809360021092120709
:109130004F2DC501B4010E9462BD88E19EE30E94EB
:1091400052EA82E08093600280939C068091F70649
:10915000882321F060E082E00E94FEFB89EB9CE026
:109160000E94748D0C94125E8CE09EE30E9452EA81
:1091700083E080939C068091F706882321F060E0CD
:1091800081E00E94FEFB83E50E944E64882351F03B
:109190000F94B6900F9417B7709300076093FF0673
:1091A00011E00EC082E50E944E64882341F00F94C6
:1091B000B6900F9417B7709300076093FF0610E006
:1091C0000E94556F6B017C01109212076091FF069F
:1091D00070910007072E000C880B990B0F9433B089
:1091E00001E02091490530914A0540914B0550918D
:1091F0004C050F9403B818160CF000E000930C0611
:1092000081E0809360028091120781110C947E604E
:1092100020910C068091FF0690910007BC01990FE8
:10922000880B990B222391F00F9433B020914905BC
:1092300030914A0540914B0550914C050F9403B86D
:10924000181614F40C948D600C947E600F9433B057
:109250002091490530914A0540914B0550914C05AC
:109260000F942DB087FD02C00C947E6011110C94F8
:109270007E600C948D6083E50E944E64882349F0E3
:109280000F94A99090E09093DE178093DD170C94D3
:10929000125E8FEF90E09093DE178093DD170C94B1
:1092A000125E809113078860809313070C94125EFE
:1092B00083E50E944E648823A1F00F94B69020E0CD
:1092C00030E04AE754E40F9496A90F941DB76093D9
:1092D0002E0270932F0280933002909331020C94EF
:1092E000125E88E50E944E6481110C94DD6089E570
:1092F0000E944E6481110C94DD608AE50E944E64E8
:1093000081110C94DD6085E40E944E6481110C94FF
:10931000DD600E94DAA3149A0E94A9B90C94125E2F
:1093200083E50E944E64882311F40C94125E0F941E
:10933000B69020E030E04AE754E40F9496A90F94E9
:109340001DB76093040670930506809306069093FC
:1093500007060C94125E83E50E944E64882311F484
:109360000C94125E0F94B69020E030E04AE754E48B
:109370000F9496A90F941DB760932A0270932B0245
:1093800080932C0290932D0283EC9CE00E94748DBC
:109390000C94125EAFE1B3E0BEA7ADA706E017E103
:1093A000A7E5CA2EA7E0DA2EF12CEDA5FEA5819146
:1093B000FEA7EDA70E944E64882309F466C0F3E07F
:1093C000FF125AC00F94B6902B013C0120E030E010
:1093D00040EA51E40F942DB087FF48C0A3019201E9
:1093E000D80114966D917D918D919C9117970F9452
:1093F000A6B64B015C019B01AC0160915A177091BC
:109400005B1780915C1790915D170F9496A96093FC
:109410005A1770935B1780935C1790935D17209099
:109420007B0230907C02A5019401F1016485758571
:10943000868597850F9496A9D1011C966D937D938F
:109440008D939C931F97F601608171818281938136
:109450000F9431B0A50194010F9496A90F941DB7F4
:10946000D6016D937D938D939C931397F80144825D
:1094700055826682778209C00F94B690D8011496FF
:109480006D937D938D939C931797F3940C5F1F4F6F
:10949000B4E0CB0ED11CE4E0FE1287CF0C94125E38
:1094A0008EE40E944E64882311F40C94125E0E9494
:1094B0002F64609391057093920580939305909328
:1094C00094050C94125E83E50E944E64882331F06B
:1094D0000F94A990809304020C94125E8FE594E699
:1094E0000E94C36AC0900402D12CE12CF12C82EAC4
:1094F0009FE00E94C36A4AE0C701B6010E94D06A99
:109500000E94E46B0C94125E86E50E944E648823F0
:1095100041F088E797E40E94C36A0E94E46B0C94D0
:10952000125E85E50E944E64882309F46AC00091AA
:109530008F05109190050F5F1F4F109390050093BA
:109540008F05BE016F5F7F4FC8010F941597882369
:1095500011F40C94125E85E493E4DE011196BE01D1
:10956000675F7F4FFC01259134914D915D912417E8
:10957000350758F04217530710F40C94125E029608
:10958000A617B70779F70C94125E8CE794E10E9456
:1095900086C844E65DE062E080E00E94E19FD80179
:1095A000FD908D018F2D0F940797811104C08F2D91
:1095B0000E94FF9BF4CF4CE654E163E080E00E9400
:1095C000E19F40E068EE73E082E390E00F9469234E
:1095D00084EF91E00E949BBE40E068EE73E082E37E
:1095E00090E00F9469238EE190E00E947FC781E0B4
:1095F0000E94B3A20E9482A280E00E94EF990C9484
:10960000125E84E89FE00E94C36A88E797E40E94A4
:10961000C36A8AE29FE00E94C36A86E29FE00E94DA
:10962000C36A87E19FE00E94C36A89E09FE00E94CD
:10963000C36A88EF9EE00E94C36A86EF9EE00E94A4
:10964000C36A8FEE9EE00E94C36A8AEC9EE00E948D
:10965000C36A0E94E46B1F92F1E3FF2EFF9284E540
:109660009DE09F938F930DE01DE01F930F930F9448
:1096700037AF1F92FF9284E49DE09F938F931F93D7
:109680000F930F9437AF1F92FF9280E39DE09F935B
:109690008F931F930F930F9437AF1F92FF9283E224
:1096A0009DE09F938F931F930F930F9437AF1F925B
:1096B000FF9288E19DE09F938F931F930F930F94E8
:1096C00037AF0FB6F894DEBF0FBECDBF0C94125E5D
:1096D00081EB96E00E94C36A0E94E46B89EA96E0FF
:1096E0000E94C36A1E9B03C08FE996E002C08AE90C
:1096F00096E00E94C36A0E94E46B82E996E00E94B1
:10970000C36A8091060182FF03C08FE996E002C020
:109710008AE996E00E94C36A0E94E46B8AE896E0B8
:109720000E94C36A1D9B03C08FE996E002C08AE9CC
:1097300096E00E94C36A0E94E46B82E896E00E9471
:10974000C36A8091060187FF03C08FE996E002C0DB
:109750008AE996E00E94C36A0E94E46B8AE796E079
:109760000E94C36A1C9B03C08FE996E002C08AE98D
:1097700096E00E94C36A0E94E46B82E796E00E9432
:10978000C36A019903C08FE996E002C08AE996E0B6
:109790000E94C36A0E94E46B0C94125E1091DB1766
:1097A00084E50E944E64882379F00F94A990182FC5
:1097B000882351F08FE594E60E94C36A8BE596E01A
:1097C0000E94E66B0C94125E84E40E944E6488232F
:1097D00011F40C94125E0F94B69020E030E0A901D1
:1097E0000F942DB0811103C010929D172EC00F94BD
:1097F000B69024E0129FF0011124E256F84E6083E7
:10980000718382839383C0909E17D0909F17E090BE
:10981000A017F090A11720E030E0A901C701B60120
:109820000F942DB0811106C0C12CD12CE0EEEE2E8C
:10983000EFE3FE2EC0929E17D0929F17E092A017E2
:10984000F092A11781E080939D170E94BAB80C9402
:10985000125ED6018D916D010E944E648823A9F19C
:109860000F94B6900F941DB71230ACF4653CB9E07C
:109870007B0781059105A0F4562F472F382F292FFC
:10988000613CE3E07E078105910590F050EC43E0F8
:1098900030E020E00DC0562F472F382F292F08C069
:1098A00050EC43E030E020E064EC79E080E090E0D0
:1098B000D7016D937D938D939C931397F701E85790
:1098C000FF4F50834183328323831F5FB4E0EB0E4D
:1098D000F11C143009F0BDCF0F9406240C94125ED5
:1098E0004FE1A42E43E0B42E56E0C52E57E1D52E0D
:1098F000912CF50181915F010E944E64882309F447
:109900003EC00F94B6907B018C01F1E0F91510F187
:1099100020E030E048E453E40F9403B818163CF418
:10992000512C612C28E4722E33E4832E04C05E2C6B
:109930006F2C702E812E20E030E048EC52E4B7010D
:10994000C8010F9403B818164CF4E12CF12C08EC64
:1099500012E404C0562E6F2C782E812E852D962D64
:10996000A72DB82DF601848B958BA68BB78BC701DD
:10997000D801E456FF4F80839183A283B3839394ED
:10998000F4E0CF0ED11C24E09212B3CF0C94125EFF
:1099900083E50E944E64882329F10F94B69060936A
:1099A000C6177093C7178093C8179093C917609311
:1099B0003A1770933B1780933C1790933D1784E5BB
:1099C0000E944E64882311F40C94125E0F94B6909A
:1099D00060933E1770933F17809340179093411701
:1099E0000C94125E80E50E944E64882351F00F941F
:1099F000B69060933A1770933B1780933C179093FF
:109A00003D1782E50E944E64882351F00F94B69072
:109A100060933E1770933F178093401790934117C0
:109A200084E50E944E64882311F40C94125E0F9416
:109A3000B6906093C6177093C7178093C81790931A
:109A4000C9170C94125E83E50E944E64882351F07E
:109A50000F94B69060934217709343178093441706
:109A60009093451784E50E944E64882351F00F942B
:109A7000B69060934617709347178093481790935A
:109A8000491782E40E944E64882361F00F94B690D7
:109A90000F941DB760934A1770934B1780934C1720
:109AA00090934D1788E50E944E64882391F00F949F
:109AB000B6906093521770935317809354179093F6
:109AC000551760934E1770934F17809350179093CC
:109AD000511789E50E944E64882351F00F94B69087
:109AE00060935217709353178093541790935517A0
:109AF0008AE50E944E64882351F00F94B6906093DB
:109B0000561770935717809358179093591785E4F9
:109B10000E944E64882311F40C94125E0F94B69048
:109B20000E94458760935A1770935B1780935C1768
:109B300090935D170C94125E9FE1E92E93E0F92E4D
:109B400000E010E0D7018D917D010E944E648823D2
:109B500049F00F94B690F801E25AF84E6083718391
:109B6000828393830C5F1F4F0C30110559F70C94BF
:109B7000125E83E50E944E64882351F00F94B690E4
:109B80006093891770938A1780938B1790938C1723
:109B900086E40E944E64882381F00F94B69020E002
:109BA00030E040E752E40F94A6B660938D177093AF
:109BB0008E1780938F17909390178AE50E944E64BA
:109BC000882311F40C94125E0F94B6906093911751
:109BD0007093921780939317909394170C94125E3E
:109BE00083E50E944E64882351F00F94B6906093F1
:109BF000951770939617809397179093981786E40C
:109C00000E944E64882311F40C94125E0F94B69057
:109C100020E030E040E752E40F94A6B66093991735
:109C200070939A1780939B1790939C170C94125ED5
:109C300083E50E944E64882311F40C94125E0F9405
:109C4000A990882341F0813061F4809388171092A5
:109C5000DA170C94125E109288171092DA170C948F
:109C6000125E8FE594E60E94C36A88E496E00E9443
:109C7000C36A8091A5099091A6098554984F0E94C6
:109C8000E66B85EC9EE00E94C36A0E94E46B0C9434
:109C9000125E82E40E944E64882351F08091630238
:109CA00090916402909303028093020211E001C03C
:109CB00010E083E50E944E64882339F00E942264FC
:109CC000909364028093630211E082E50E944E64E7
:109CD000882351F0809102029091030290936402D4
:109CE000809363020C94125E11110C94125E8091A9
:109CF00064028F93809163028F938FEB9EE09F931A
:109D00008F930F9437AF0F900F900F900F900C948C
:109D1000125E83E50E944E64882301F10E94226452
:109D20008C0184E50E944E64882399F0BE016F5F28
:109D30007F4F8DED90E00F943F9681110C94125E51
:109D4000E981F0E0EE0FFF1FE050FE4F118300832A
:109D50007CCD1093A3020093A20277CD8091A30241
:109D60008F938091A2028F9389EB9EE09F938F93B4
:109D70000F9437AF0F900F900F900F9066CD80E546
:109D80000E944E64882311F40C94125E0E94226497
:109D90008C0183E50E944E64882321F00E94226496
:109DA0007C0103C0EE24EA94FE2CC70101960397C0
:109DB00010F00C94125EECEDFFE02CE12E0F84917C
:109DC000082E000C990B8017910711F40C94125E69
:109DD00031962E13F4CF17FF02C00C94125E0E942E
:109DE000DAA3D02E60E0802F0E94D6F1BFEFEB16F1
:109DF000FB0631F0EA94EF2871F401E010E00DC0A9
:109E0000802F0F94A89631E020E0892B09F030E0F4
:109E1000032F122F02C000E010E08D2D0F94A896A2
:109E20008017910711F40C94125E0E9457D380E0C2
:109E30000E9445BA80E00E94EF99EFCF83E50E942F
:109E40004E64882331F00F94B6900F941DB78B01A8
:109E500002C00EE610E080E50E944E64882331F0D7
:109E60000F94B6900F941DB7CB0102C088EE93E01B
:109E70000115110531F040E0B8010F9469230C94ED
:109E8000125EBC0180E090E00E941D6F0C94125E97
:109E900080E50E944E64882351F00F94B690609341
:109EA0006E1770936F17809370179093711789E4F2
:109EB0000E944E64882381F00F94B6902CEA35EC12
:109EC00047E25EE30F9496A960937217709373173D
:109ED000809374179093751784E40E944E648823CE
:109EE00081F00F94B6902CEA35EC47E25EE30F94D4
:109EF000A6B6609376177093771780937817909330
:109F000079170E94D3D881E898E10E94C36A81E55D
:109F100093E00E94E66B60916E1770916F178091CD
:109F200070179091711742E00E946F6B85E593E086
:109F30000E94E66B2CEA35EC47E25EE36091721713
:109F40007091731780917417909175170F94A6B63E
:109F500042E00E946F6B89E593E00E94E66B2CEA79
:109F600035EC47E25EE36091761770917717809148
:109F70007817909179170F9496A942E00E946F6B21
:109F80000E94E46B0C94125E80E50E944E6488236C
:109F900051F00F94B69060937A1770937B1780936B
:109FA0007C1790937D1789E40E944E64882381F08A
:109FB0000F94B6902CEA35EC47E25EE30F9496A935
:109FC00060937E1770937F1780938017909381170B
:109FD00084E40E944E64882381F00F94B6902CEAAA
:109FE00035EC47E25EE30F94A6B660938217709358
:109FF000831780938417909385170E94D3D881E8A4
:10A0000098E10E94C36A81E593E00E94E66B60914B
:10A010007A1770917B1780917C1790917D1742E0A1
:10A020000E946F6B85E593E00E94E66B2CEA35ECAD
:10A0300047E25EE360917E1770917F1780918017F1
:10A04000909181170F94A6B642E00E946F6B89E54C
:10A0500093E00E94E66B2CEA35EC47E25EE3609108
:10A0600082177091831780918417909185170F94B0
:10A0700096A942E00E946F6B0E94E46B0C94125E02
:10A0800083E50E944E64882319F00F94B69003C0B4
:10A0900060E070E0CB01609375027093760280936C
:10A0A0007702909378020C94125E85E40E944E64CD
:10A0B000882331F00E9422648C0197FF03C009C0FD
:10A0C00000E010E0C12CD12CA6E1EA2EA3E4FA2E88
:10A0D00006C0C12CD12CFCE8EF2EF2E4FF2E83E564
:10A0E0000E944E64882321F00F94B6906B017C018E
:10A0F00083E40E944E64882319F00E94226402C007
:10A1000085E090E09C01A801C701B6010F9466921A
:10A110000C94125E80914805882311F40C94125E11
:10A1200085E40E944E64882321F00F94A990182F93
:10A1300001C01FEF86E40E944E64882321F00F9433
:10A14000A990082F01C00FEF1F920F931F921F932A
:10A150008CEF9CE09F938F930F9437AF1F920F93D8
:10A160001F921F9384EF9CE09F938F930F94DB4685
:10A170000FB6F894DEBF0FBECDBF1AE00F94CC46E9
:10A18000181614F40C94125E115011F40C94125E13
:10A1900084E690E00E949BBEF1CF0E94086C0C9474
:10A1A000125E0E94F36B0C94125E809169178F937C
:10A1B000809168178F93809167178F9380916617AE
:10A1C0008F93809165178F93809164178F938091FF
:10A1D00063178F93809162178F93809161178F938C
:10A1E000809160178F9380915F178F9380915E1796
:10A1F0008F930FE514E61F930F931F930F93809196
:10A200005D178F9380915C178F9380915B178F936D
:10A2100080915A178F93809159178F938091581777
:10A220008F93809157178F93809156178F938091BA
:10A2300055178F93809154178F93809153178F9355
:10A24000809152178F93809151178F93809150175F
:10A250008F9380914F178F9380914E178F9380919A
:10A260004D178F9380914C178F9380914B178F933D
:10A2700080914A178F93809149178F938091481747
:10A280008F93809147178F93809146178F9380917A
:10A2900045178F93809144178F93809143178F9325
:10A2A000809142178F931F930F931F930F93809169
:10A2B000C9178F938091C8178F938091C7178F9379
:10A2C0008091C6178F93809141178F93809140178B
:10A2D0008F9380913F178F9380913E178F9380913A
:10A2E0003D178F9380913C178F9380913B178F93ED
:10A2F00080913A178F931F930F931F930F93809121
:10A30000C1178F938091C0178F938091BF178F9340
:10A310008091BE178F938091BD178F938091BC174A
:10A320008F938091BB178F938091BA178F938091F1
:10A33000B9178F938091B8178F938091B7178F9328
:10A340008091B6178F938091B5178F938091B41732
:10A350008F938091B3178F938091B2178F931F9330
:10A360000F931F930F93809139178F938091381714
:10A370008F93809137178F93809136178F938091A9
:10A3800035178F93809134178F93809133178F9364
:10A39000809132178F93809131178F93809130176E
:10A3A0008F9380912F178F9380912E178F93809189
:10A3B0002D178F9380912C178F9380912B178F934C
:10A3C00080912A178F931F930F931F930F93809160
:10A3D000B1178F938091B0178F938091AF178F93A0
:10A3E0008091AE178F938091AD178F938091AC17AA
:10A3F0008F938091AB178F938091AA178F93809141
:10A40000A9178F938091A8178F938091A7178F9387
:10A410008091A6178F938091A5178F938091A41791
:10A420008F938091A3178F938091A2178F931F937F
:10A430000F931F930F93809129178F938091281763
:10A440008F93809127178F93809126178F938091F8
:10A4500025178F93809124178F93809123178F93C3
:10A46000809122178F93809121178F9380912017CD
:10A470008F9380911F178F9380911E178F938091D8
:10A480001D178F9380911C178F9380911B178F93AB
:10A4900080911A178F931F930F931F930F9380919F
:10A4A000C5171F928F938091C4171F928F9380912D
:10A4B000C3171F928F938091C2171F928F931F9380
:10A4C0000F931F930F93809119178F9380911817F3
:10A4D0008F93809117178F93809116178F93809188
:10A4E00015178F93809114178F93809113178F9363
:10A4F000809112178F93809111178F93809110176D
:10A500008F9380910F178F9380910E178F93809167
:10A510000D178F9380910C178F9380910B178F934A
:10A5200080910A178F931F930F931F930F938BE1C3
:10A530009AE09F938F930F9437AF0FB6F894DEBFD6
:10A540000FBECDBF2CEA35EC47E25EE36091761793
:10A550007091771780917817909179170F9496A939
:10A560009F938F937F936F932CEA35EC47E25EE3E2
:10A57000609172177091731780917417909175178D
:10A580000F94A6B69F938F937F936F9380917117CB
:10A590008F93809170178F9380916F178F93809115
:10A5A0006E178F931F930F931F930F938EEE99E067
:10A5B0009F938F930F9437AF2CEA35EC47E25EE31D
:10A5C00060918217709183178091841790918517FD
:10A5D0000F9496A99F938F937F936F932CEA35ECFA
:10A5E00047E25EE360917E1770917F17809180173C
:10A5F000909181170F94A6B69F938F937F936F933B
:10A6000080917D178F9380917C178F9380917B171A
:10A610008F9380917A178F931F930F931F930F93AC
:10A6200089EB99E09F938F930F9437AF0FB6F8940F
:10A63000DEBF0FBECDBF809188171F928F931F93EF
:10A640000F931F930F9320E030E040E752E46091B6
:10A65000991770919A1780919B1790919C170F945E
:10A6600096A99F938F937F936F93809198178F9361
:10A67000809197178F93809196178F93809195175C
:10A680008F931F930F931F930F93809194178F9322
:10A69000809193178F93809192178F938091911748
:10A6A0008F9320E030E040E752E460918D17709185
:10A6B0008E1780918F17909190170F9496A99F9362
:10A6C0008F937F936F9380918C178F9380918B17CB
:10A6D0008F9380918A178F93809189178F931F93FF
:10A6E0000F931F930F9388EB98E09F938F930F9492
:10A6F00037AF0FB6F894DEBF0FBECDBF80919D1768
:10A700008823E9F08091A1178F938091A0178F93F0
:10A7100080919F178F9380919E178F931F930F9314
:10A720001F930F9382E998E09F938F930F9437AF15
:10A730000FB6F894DEBF0FBECDBF0C94125E1F9310
:10A740000F9383E798E09F938F930F9437AF0F9009
:10A750000F900F900F900C94125E8FE594E60E947C
:10A76000C36A89EA9EE00E94C36A0C94125E8AE57D
:10A770000E944E64882309F450C00F94B6906B0178
:10A780007C0120E030E040E751EC0F9403B887FDF6
:10A7900024C020E030E040EA50ECC701B6010F943D
:10A7A0002DB01816D4F0F7FAF094F7F8F094C092A0
:10A7B0006A17D0926B17E0926C17F0926D178FE5C5
:10A7C00094E60E94C36A8FE396E00E94C36A0E94E7
:10A7D000E46B0E94E46B0C94125E8FE594E60E9499
:10A7E000C36A8FE396E00E94C36A8AE796E00E94FC
:10A7F000C36A61EF7FEF8FEF9FEF0E94556B82E797
:10A8000096E00E94C36A6BEF7FEF8FEF9FEF0E948D
:10A81000556B0E94E46B0C94125E8FE594E60E94E7
:10A82000C36A8FE396E00E94C36A0E94E46B809142
:10A830006A1790916B17A0916C17B0916D17BC01BE
:10A84000CD01905842E00E946F6B0E94E46B0C9423
:10A85000125E80E50E944E64882311F40C94125E0F
:10A8600010929107109292071092930710929407FA
:10A87000E1E9EE2EE7E0FE2E10E00AE2E0918F051E
:10A88000F091900500830E942264D7018D937D0191
:10A890001F5F143011F40C94125E8EE20E944E641D
:10A8A0008111ECCF109291071092920710929307AA
:10A8B000109294070C94125E0E94DAA385E40E9421
:10A8C0004E64882339F00F94B6906DA77EA78FA7AA
:10A8D00098AB08C080E090E0A0E0B0EC8DA79EA708
:10A8E000AFA7B8AB8CE40E944E6481110F94B69070
:10A8F0008AE50E944E64882319F00F94B69016C022
:10A900006091D2177091D3178091D4179091D51779
:10A910000F941DB7862F693118F46BE1681B01C0D5
:10A9200062E070E080E090E00F9431B02B013C01D8
:10A9300088E50E944E64882329F00F94B6906B013D
:10A940007C0106C0C12CD12C73E5E72E73E4F72EF1
:10A9500089E50E944E64882329F00F94B6904B013C
:10A960005C0103C0812C912C5401809148058823FF
:10A9700011F40C94F96084EA9EE00E943A64882302
:10A9800011F40C94F96011E00E94DAA38091F706AB
:10A99000882321F060E086E10E94FEFB20906302A4
:10A9A00030906402E091DB17F0E0EE0FFF1FEF5FE5
:10A9B000F84FA081B181BAABA9ABBD01BB0F880B29
:10A9C000990B0F9433B06DAB7EAB8FAB98AFE0912A
:10A9D000DD17F091DE17FAAFE9AF8091CA179091B9
:10A9E000CB17A091CC17B091CD1789839A83AB83F5
:10A9F000BC838091CE179091CF17A091D017B091C2
:10AA0000D1178D839E83AF83B8878091D2179091A1
:10AA1000D317A091D417B091D51789879A87AB87A0
:10AA2000BC876091D6177091D7178091D8179091F5
:10AA3000D9176D877E878F87988B2DA53EA54FA54B
:10AA400058A90F94B8B56093D6177093D717809311
:10AA5000D8179093D91760E070E088EE92E40F94D5
:10AA600085190E94DAA3A30192016091D217709117
:10AA7000D3178091D4179091D5170F94B8B56093E0
:10AA8000D2177093D3178093D4179093D51760E0A3
:10AA900070E080E791E40F9485190E94DAA3C092D8
:10AAA000CA17D092CB17E092CC17F092CD178092B4
:10AAB000CE179092CF17A092D017B092D11760E026
:10AAC00070E088E492E40F9485190E94DAA38091E3
:10AAD0004805811121C084E0809360020E94556F77
:10AAE0004B015C0183E393E10E9486C8DD24D3948B
:10AAF00000E0E12CF12C01110C943E610E94B59A0A
:10AB0000882311F40C943E619FB7F8948091020160
:10AB10008B7F809302019FBF10923C048091480577
:10AB2000882319F00F94312103C081E00F94F96B51
:10AB30000E94DAA380914805811137C084E0809398
:10AB4000600241E060E08CE494E10E949EC8809342
:10AB50003C0481112AC00E9482A248E85BE562E0C1
:10AB600080E00E94E19F20E030E048EC52E46091F8
:10AB7000CA177091CB178091CC179091CD170F9475
:10AB8000B7B56093CA177093CB178093CC17909387
:10AB9000CD1760E070E088E492E40F9485190E947C
:10ABA000DAA38CE194E10E94AFC880914805882324
:10ABB00009F479C011116FC080911107882329F021
:10ABC00060E080913C020F94932084E080936002C7
:10ABD0008CE593E10E9486C801E0E12CF12C0E94F3
:10ABE000B59A81113CC00E9457D381E00E9445BABA
:10ABF000A4EFEA16A1E0FA0611F4E12CF12C809101
:10AC00000101846080930101E114F104A1F48091B9
:10AC10003705833031F0882321F08130C1F40023DF
:10AC2000B1F09FB7F8948091020184608093020193
:10AC30009FBF00E00CC0B4E1EB16F10441F49FB7F4
:10AC4000F894809102018B7F809302019FBFEFEF08
:10AC5000EE1AFE0A84E090E00E949BBEC0CF9FB730
:10AC6000F894809102018B7F809302019FBF8091B5
:10AC70001107882381F00E9482A248E85BE562E028
:10AC800080E00E94E19F87E10F94A24640E060E0EF
:10AC900080E00F9473434DA95EA96FA978AD812F11
:10ACA0000F94599837C00E9482A245EB53E161E0AE
:10ACB00080E00E94E19F80911302811105C042EA69
:10ACC00053E162E00E94E19F84E0809360020E9471
:10ACD000B59A811110C00E9457D381E00E9445BAF5
:10ACE0000E94C888882399F340E068EE73E082E30D
:10ACF00090E00F94692382E0809360020F94269F76
:10AD000040E068EE73E082E390E00F94692380E016
:10AD10000E94B3A2112341F181E00E94B3A229ADA8
:10AD20003AAD3093DE172093DD171111F7C020E004
:10AD300030E040EA50E46091D6177091D7178091C7
:10AD4000D8179091D9170F94B8B56093D617709310
:10AD5000D7178093D8179093D91760E070E080E000
:10AD600090E40F948519DAC010923C0404E08091BD
:10AD70003C04813089F210923C04009360020E94EE
:10AD800082A24BEE53E160E080E00E94E19F45E348
:10AD900057E661E081E00E94E19F47ED53E162E008
:10ADA00081E00E94E19F45EC53E163E081E00E9475
:10ADB000E19F4EE361E080E00E94FDA1C090DF17BB
:10ADC0000C2C000CDD080E94DF69EE24E394F12CCA
:10ADD00080913C04811164C00E9457D381E00E949D
:10ADE00045BA8091DF17082E000C990B9601281B9D
:10ADF000390B37FF03C031952195310925303105D5
:10AE0000F4F18C159D051CF431E0E31AF108C81625
:10AE1000D90644F48FEFE81AF80A94E0E916F10431
:10AE2000ACF004C0A4E0EA16F1043CF087E00F9413
:10AE3000032383E0E82EF12C09C0E114F10431F47E
:10AE400087E00F940323EE24E394F12C44E658E0CA
:10AE500061E080E00E94E19F4EE36E2D80E00E9461
:10AE6000FDA1C090DF170C2C000CDD0886E00F94CC
:10AE7000032364E670E080E090E00E941D6F0E9472
:10AE8000B59A882309F4A4CF80E00F940323E092BD
:10AE90003C0464EF71E080E090E00E941D6F98CF69
:10AEA0000E9482A20E9440D982E080936002809139
:10AEB0003C048230D9F0833041F50E94DAA30F942C
:10AEC0007E3B0E9482A24EEF53E160E080E00E9450
:10AED000E19F48E85BE562E080E00E94E19F87E94E
:10AEE0009DE10F948B960E94DAA341CF8091480593
:10AEF000882341F04DA95EA96FA978AD80E00F9439
:10AF0000599835CF0F94269F32CF0E9482A24CE0F1
:10AF100054E162E080E00E94E19F29CFE090D217E7
:10AF2000F090D3170091D4171091D5172D813E8141
:10AF30004F81588569817A818B819C811F921F92F4
:10AF4000E091DB17EF93812C912CE8E4AE2EE2E444
:10AF5000BE2EF6EDCF2EF7E1DF2E0F94A3240E9434
:10AF6000DAA3E984FA840B851C852D813E814F810B
:10AF7000588569817A818B819C811F921F92E09113
:10AF8000DB17EF93812C912CA0E7AA2EA1E4BA2E17
:10AF90000F94A3240E94DAA3CE010D960F9470247F
:10AFA00080E1FE013196AAECB7E101900D928A95FD
:10AFB000E1F70E94696420926302309264023F923A
:10AFC0002F928AE698E09F938F938E010C5D1F4F1E
:10AFD0001F930F930F9490AF60E0C8010E948E8A78
:10AFE0000E94C88887E697E10E9452EA10921407EF
:10AFF0000FB6F894DEBF0FBECDBF14C680915F05BB
:10B00000811110C60E94DAA30F94C87D0E941F8C84
:10B010000F949A5007C680915F05882309F402C6F1
:10B020000C94234483E50E944E64882309F4FAC5F6
:10B030000E9422646C0188E89BE50E9452EA81E844
:10B040009EE00E94C36A0D2C000CEE08FF08C701A9
:10B05000B6010E94556B0E94E46B0E94556F4B0134
:10B060005C01109212076091FF0670910007072E95
:10B07000000C880B990B0F9433B020E030E0A9014D
:10B080000F942DB0811113C06091010770910207D8
:10B09000072E000C880B990B0F9433B011E020E0C1
:10B0A00030E0A9010F942DB0882309F449C010E0C5
:10B0B00047C080911207811159C0C701B6010F9492
:10B0C00033B09B01AC016091F3067091F40680915E
:10B0D000F5069091F6060F942DB087FF47C00E94A9
:10B0E000556FDC01CB0188199909AA09BB09893E72
:10B0F0009340A105B105E0F08EE79EE00E94C36A8F
:10B100006091F3067091F4068091F5069091F60631
:10B1100041E00E946F6B8FE20E94AB6AC701B601EB
:10B120000E94556B0E94E46B0E94556F4B015C01BD
:10B130000E9457D380E00E9445BA80E00E94EF99B8
:10B14000112309F4B6CFC701B6010F9433B09B01A8
:10B15000AC016091F3067091F4068091F506909130
:10B16000F6060F9403B818160CF4B9CF81E898E1ED
:10B170000E9452EA57C58FE30E944E64882309F467
:10B180007CC00E94F469882319F08DE593E002C029
:10B1900081E793E00E94F16B85E893E00E94F16BF8
:10B1A00044244A94542C320163E2862E912CA12C23
:10B1B000B12C00EB1FE0212C312C6101032C000C81
:10B1C000EE08FF08C701B6010F9433B020911217A3
:10B1D0003091131740911417509115170F94A6B67C
:10B1E00069AB7AAB8BAB9CAB4DA6942D9F3F29F4FA
:10B1F0008AE79EE00E94C36A04C0C301B2010E94B4
:10B20000556B87E79EE00E94C36AC501B4010E94A6
:10B21000556B84E79EE00E94C36AC701B6010E9495
:10B22000556B81E79EE00E94C36A20E030E04AE768
:10B2300054E469A97AA98BA99CA90F9496A942E024
:10B240000E946F6B0E94E46B0A3BAFE01A0709F49F
:10B25000E9C42DA52E3F21F0C8010F942AB51C0189
:10B260000E5F1F4F35E0830E911CA11CB11C8FEFA8
:10B27000481A580A680A780AA0CF81E20E944E64F0
:10B28000882341F161E086EA9FE00F945CB568E0B5
:10B2900070E080EB9FE00F9458B568E170E082EBBE
:10B2A0009FE00F9458B560E370E084EB9FE00F944B
:10B2B00058B560E570E086EB9FE00F9458B568E7FD
:10B2C00070E088EB9FE00F9458B58CE993E00E9402
:10B2D000F16BA8C48AE50E944E648823B9F061E04E
:10B2E00086EA9FE00F945CB500EB1FE060E070E041
:10B2F000C8010F9458B50E5F1F4F0A3BBFE01B07F4
:10B30000A9F78DEA93E00E94F16B8CC483E50E945B
:10B310004E64882309F48EC00E9422648C0189E463
:10B320000E944E64882309F47DC40F94A99085304F
:10B3300008F078C4282F30E0C901880F991FB801A0
:10B340008055904F0F9458B587EB93E00E94F16BB6
:10B3500085E893E00E94F16B88248A94982C54012C
:10B3600043E2442E512C612C712C00EB1FE080E055
:10B3700090E06C01990FEE08FF08C701B6010F9429
:10B3800033B0209112173091131740911417509138
:10B3900015170F94A6B66DA77EA78FA798AB382C6C
:10B3A0003FEF831205C08DE69EE00E94C36A04C091
:10B3B000C501B4010E94556B8AE69EE00E94C36AF3
:10B3C000C301B2010E94556B87E69EE00E94C36AEA
:10B3D000C701B6010E94556B84E69EE00E94C36AD5
:10B3E00020E030E04AE754E46DA57EA58FA598A93A
:10B3F0000F9496A942E00E946F6B0E94E46B0A3B97
:10B400008FE0180709F40EC4EEEF3E1621F0C801D4
:10B410000F942AB502C080E090E00E5F1F4FF5E068
:10B420004F0E511C611C711C2FEF821A920AA20A46
:10B43000B20A9FCF83E59EE00E94C36AF3C30F94D4
:10B440007E90AE014C5D5F4F0F94E3B820E030E09A
:10B4500040E251E40F9496A920E030E040E05FE341
:10B460000F94B8B50F941DB7633009F47CC028F46D
:10B47000613051F06230C9F1D5C3643009F4F5C0D0
:10B48000653009F48FC1CEC380E50E944E648823E5
:10B49000A1F00F94B69020E030E04AE754E40F9416
:10B4A00096A920E030E040E05FE30F94B8B50F9438
:10B4B0001DB7CB010F94D196B5C381E50E944E64B0
:10B4C000882309F4AFC385EA9DE00F942AB5BC0137
:10B4D00080E090E00F9431B020E030E04AE754E49F
:10B4E0000F94A6B60F9424639DC380E50E944E641A
:10B4F000882339F10E942F648091D306882309F4B0
:10B5000091C320914605309147056217730709F4EE
:10B5100089C3813051F0823009F084C386EA92E118
:10B520000E94AFC80F9439177DC380E792E10E9453
:10B5300086C88EE190E00E947FC781E00E94B3A29E
:10B5400071C381E50E944E64882309F46BC3609146
:10B5500046057091470580E090E04AE00E94D06A7D
:10B560000E94E46B5FC380E50E944E64882309F467
:10B570006DC000918F051091900519821A821B826F
:10B580001C82FE01359689E0DF011D928A95E9F75C
:10B5900080914405909145050F94F6AD6C0162E2EF
:10B5A00070E0C8010F9400BB009779F48091D30636
:10B5B000813009F43FC0823009F034C386EA92E159
:10B5C0000E94AFC80F9439172DC38C010F5F1F4F16
:10B5D00062E270E0C8010F9400BB009739F37C0170
:10B5E000E01AF10A0115110509F3CE14DF0410F475
:10B5F000A60101C0A7014F5F5F4FB801CE010196C0
:10B600000F9459AECE14DF0430F46AEB73E0CE0130
:10B6100001960F94F5BAEC14FD0441F660914405CF
:10B6200070914505A701C8010F94FFAD892B09F45E
:10B63000F9C2BCCF80E792E10E9486C88EE190E01B
:10B640000E947FC781E00E94B3A2ECC281E50E9404
:10B650004E64882309F4E6C2809144059091450523
:10B660000E94C36A0E94E46BDDC280E50E944E64C2
:10B67000882309F48FC080918F05909190050196E1
:10B680009093900580938F052091D206222309F490
:10B69000C9C2BE016F5F7F4F0F9415978AE090E09B
:10B6A0000F942AB59C0149815A818417950730F07F
:10B6B00091E04217530718F490E001C092E0F92E90
:10B6C000F294FF0CFF0CB0ECFB228CE090E00F94A6
:10B6D0002AB52B813C818217930730F001E02817AF
:10B6E000390718F400E001C002E0B0E10B9F8001CF
:10B6F00011240F0D111D8EE090E00F942AB59C01CE
:10B700004D815E818417950730F091E04217530711
:10B7100018F490E001C092E0E4E09E9F000D111D3E
:10B72000112480E190E00F942AB59C014F81588547
:10B730008417950730F091E04217530718F490E012
:10B7400001C092E09801290F311DC901253531054D
:10B7500009F468C22091D206853591051CF4213088
:10B7600009F460C2213051F0223009F05BC281EF50
:10B7700091E10E94AFC80F94391754C282E492E15C
:10B780000E9486C88EE190E00E947FC781E00E94FF
:10B79000B3A248C281E50E944E64882309F442C2E4
:10B7A0000C94894A80E50E944E64882341F10E94EE
:10B7B0002F648091D106882309F434C26130710569
:10B7C00009F430C2672B19F4813009F42BC281309F
:10B7D00051F0823009F026C28AE991E10E94AFC897
:10B7E0000F9439171FC28BE691E10E9486C88EE143
:10B7F00090E00E947FC781E00E94B3A213C281E55E
:10B800000E944E64882309F40DC261E070E080E07C
:10B8100090E00E94556B0E94E46B04C28BE40E948E
:10B820004E648823B1F00F947E907B018C0120E060
:10B8300030E0A9010F942DB081110FC01092520772
:10B840001092530710925407109255070E94AC872C
:10B850007EC0E12CF12C00E010EC80919505811167
:10B8600019C020E030E0A901B701C8010F942DB044
:10B8700087FD58C020E030E040E251E4B701C80144
:10B880000F942DB0881F8827881F92E0981B892F5E
:10B890000E94AC878091950520E030E0A901B701B6
:10B8A000813081F4C8010F9403B887FD3BC020E0CC
:10B8B00030E040E251E4B701C8010F942DB087FD9C
:10B8C00028C030C0C8010F9403B887FD2BC02FE6F5
:10B8D00032E143E05BE3B701C8010F9496A92AE087
:10B8E00037ED43E25CE30F94B7B57B018C0120E0B8
:10B8F00030E0A9010F942DB087FD1BC020E030E09F
:10B9000040E251E4B701C8010F9403B818160CF4D3
:10B910007CC520E030E0A901B701C8010F942DB02B
:10B9200087FF0BC08CE498E00E94C36A0E94E46B1E
:10B930000EC0E12CF12C00E010E0C701D80180938B
:10B94000520790935307A0935407B09355078FE580
:10B9500094E60E94C36A81E498E00E94C36A609101
:10B9600052077091530780915407909155070F9497
:10B97000246358C1133009F444C071D70F9433B015
:10B980006B017C0120E030E0A9010F942DB087FD10
:10B990000EC520E030EA40E854E4C701B6010F9438
:10B9A00003B818160CF4FBC420E030E047E054E480
:10B9B000C701B6010F9403B887FDFCC420E030E056
:10B9C0004CE752E4C701B6010F9496A920E030EA93
:10B9D00040E854E40F94A6B60F941DB7062F812FAC
:10B9E0000F94679F602F812F0F94569F1F5F143015
:10B9F00009F418C1D5018D915D0150D78823B1F3A9
:10BA0000B9CF0E94DDF6882309F4B7CF89E693E623
:10BA10000E94C36A82E49EE00E94C36A0E94E46BB3
:10BA2000E5CFEFE1F3E0FEA7EDA766E0C62E67E104
:10BA3000D62E76EEA72E76E1B72E00E010E0812C10
:10BA40009924939409ABADA5BEA58D91BEA7ADA7D2
:10BA500025D7782E882309F4A5C00F94B6900F94AB
:10BA60001DB71B012C017B016830710581F060312D
:10BA7000710569F021E06032710509F020E00330C2
:10BA8000110579F0C1010197029730F40CC0033021
:10BA9000110509F4BFC421E091E034E0E316F1049C
:10BAA00019F090E001C0972D922B0330110551F44D
:10BAB00080E4E816F10439F077247394A0E8EA16DC
:10BAC000F10409F0712C911103C0772009F46AC0C8
:10BAD0000E94DAA3F801E05BFA4F3401008002C053
:10BAE000769467940A94E2F7B10189A90F946D5C8A
:10BAF000F801EE53F84E20826E147F0448F5C7011A
:10BB0000B3010F9462BA2B01612C712CC301B201F5
:10BB10000F9431B09B01AC01F6016481758186817F
:10BB200097810F9496A9D60114966D937D938D936A
:10BB30009C931797F5012081318142815381C30184
:10BB4000B2010F946DB560837183828393832AC0A1
:10BB5000C301B7010F9462BA2B01612C712CC30190
:10BB6000B2010F9431B09B01AC01F6016481758183
:10BB7000868197810F94A6B6D60114966D937D9316
:10BB80008D939C931797F5016081718182819381D8
:10BB9000A30192010F9489BAD5012D933D934D9342
:10BBA0005C9313970F5F1F4FB4E0CB0ED11CE4E002
:10BBB000AE0EB11C0430110509F044CF33C08091A2
:10BBC0004805882321F085E469D6811100C40F94CB
:10BBD000633528C083E462D690914805882329F014
:10BBE000992301F10F9431211DC09111FBCF80E009
:10BBF0000F94F96B17C08091A5099091A6098554FF
:10BC0000984F9F938F931F928DE48F9389E497E0D1
:10BC10009F938F930F9437AF0F900F900F900F90CB
:10BC20000F900F901092800710927F070C94EE34C3
:10BC300084E534D6882309F411C120918F05309111
:10BC40009005F90131968F01021B130B7F01819141
:10BC50008032C9F38930B9F3082E000C990B0F9488
:10BC6000BDBAD7018C9380918F0590919005FC010E
:10BC7000E00FF11F808190ED980F953008F466C0B9
:10BC80008F3309F44CC0883729F0833679F182E389
:10BC90009EE0C4C180914805882311F40C94EE34D1
:10BCA00040E050E067ED76E48DEC94E10F949A6CFF
:10BCB00080935F0290913C0289130AC0809128070B
:10BCC000882331F088E19EE00F945FAF0C94EE344E
:10BCD0000E94DAA380915F028F5F0F94A24643E037
:10BCE00061E081E00F9473430C94EE348091480539
:10BCF000882311F40C94EE340E94DAA38091B60CE0
:10BD0000811106C081E09091C806963009F080E06C
:10BD10000F94CC1F80915F0280933C0257C08091AA
:10BD2000480540E050E0882351F067ED76E48DEC63
:10BD300094E10F949A6C80935F0211E01BC061E460
:10BD400075E48CEB94E10F949A6C69C30F94B690F0
:10BD50000F941DB7862F60935F0290914805992339
:10BD600041F090917604992321F090916102911114
:10BD700054C310E00E94DAA39091480580915F02BD
:10BD8000992341F190913C02891304C090912807B6
:10BD9000911198CF8F5F0F94A24643E061E081E05C
:10BDA0000F9473438091B60C811106C081E090918D
:10BDB000C806963009F080E00F94CC1F80915F0296
:10BDC00080933C02112311F40C94EE340F9454210F
:10BDD0000C94EE34882399F08FE594E60E94C36AB0
:10BDE00084E50E94AB6A60915F0270E080E090E0C1
:10BDF0000E94556B0E94E46B8EE296E00FC186E4D0
:10BE00004DD58823D9F00F94B6906B017C016093D7
:10BE1000E2177093E3178093E4179093E51720E0FF
:10BE200030E0A9010F9403B8181644F4C0929E02A2
:10BE3000D0929F02E092A002F092A1028FE594E6D8
:10BE40000E94C36A8CE196E00E94C36A6091DB178E
:10BE500070E080E090E00E94556BE2C084E41ED563
:10BE6000882309F4C9C0EED486309105E1F194F439
:10BE700082309105E1F08330910549F1019609F096
:10BE8000A2C086EF95E09F938F930F9437AF0F90EA
:10BE90000F900CC08531910509F456C0863191058B
:10BEA00009F470C0449709F08EC02FC0FFCF41EF56
:10BEB000C42E45E0D42E52E0E52E00E020E032E230
:10BEC00040E050E060E072E080E090E01AC02AEECE
:10BED000C22E25E0D22E33E0E32E01E020E030E157
:10BEE00040E050E00BC083EEC82E85E0D82E96E0EF
:10BEF000E92E03E020E030E044E050E060E070E054
:10BF0000CB010F94E7900C94EE3485E40F94D2901B
:10BF1000882329F080E00E94ACF50C94EE340E9456
:10BF2000556F6B017C010E94D9F50E94556FDC01B1
:10BF3000CB018C199D09AE09BF09BF93AF939F93A5
:10BF40008F938AEC95E04CC080E090E00E9405F66B
:10BF5000811103C087EB95E02EC081E080936002E1
:10BF600080EA95E09F938F930F9437AF03E020E032
:10BF700033E240E050E060E070ED83E090E00F9449
:10BF8000B7A01DC080E090E00E9405F6811103C0BB
:10BF90008DE895E010C08CE58CBD1DBC0E941C6E28
:10BFA00040E050ED63E070E080E20E94DB6D0E94B3
:10BFB000BA6D8FE795E09F938F930F9437AF0F90F3
:10BFC0000F900C94EE348091A5099091A6098554A8
:10BFD000984F9F938F931F9284E48F9389E497E007
:10BFE0009F938F930F9437AF0F900F900F900F90F8
:10BFF0000F900F900C94EE348FE594E60E94C36A84
:10C0000088E496E00E94C36A8091A5099091A609F0
:10C010008554984F0E94E66B83E19EE00E94C36ABC
:10C020000E94E46B0C94EE3482E0809360021092E4
:10C030009F0610929E060C94E7340F9458B50C940A
:10C04000EE3485EA9DE00F942AB5BC0180E090E0D3
:10C050000F9431B020E030E04AE754E40F94A6B6E4
:10C060000F9424630C94EE34E091DB17F0E0E65279
:10C07000F84E80818111B0C10AC0E091DB17F0E079
:10C08000E652F84E8081882311F40C94F93A0E940C
:10C09000DAA380914E0790914F07A0915007B0917D
:10C0A00051078093D6179093D717A093D817B093C2
:10C0B000D91786ED97E10F947024E091DB17F0E03B
:10C0C000E652F84E908181E089270F9450A1AAC1D1
:10C0D000C6D36B017C016093E90F7093EA0F8093E4
:10C0E000EB0F9093EC0F0F94C064C0928B05D0922D
:10C0F0008C05E0928D05F0928E0594CD83E09EE351
:10C100000E9452EA82E08093600284E080939C0661
:10C1100089EB9CE00E94748D85CD0E94556FDC01F7
:10C12000CB018C199D09AE09BF09893E9340A10539
:10C13000B105C8F18091F706811131C0E091DB179C
:10C1400094E0E99FF0011124E054F94FC080D180C0
:10C15000E280F38081EB9FE00E94C36A42E0C70166
:10C16000B6010E946F6B8DEA9FE00E94C36A6091E6
:10C17000DB1770E080E090E00E94556B89EA9FE059
:10C180000E94C36A6091490570914A0580914B05F0
:10C1900090914C0541E00E946F6B0E94E46B0E94FD
:10C1A000556F6B017C010E9457D380E00E9445BA15
:10C1B00080E00E94EF990C9403490E94DAA388E57D
:10C1C0006DD3882319F0179A1092880589E566D3F4
:10C1D000882319F0169A109289058AE55FD3811198
:10C1E0000F944B3B85E45AD3882309F41BCD149A52
:10C1F00019CD10E00C94C454E12CF12C8091010174
:10C20000846080930101E114F10409F04FC0809132
:10C210003705833009F440C08823F1F18130D1F132
:10C220002FEFE21AF20A013009F452C008F04CC0B4
:10C2300084E090E00E949BBE0E94556F240135016E
:10C2400030EC430E37E2531E39E0631E711C461674
:10C2500057066806790610F00C947B5584E093E14C
:10C260000E9486C81CA21DA21EA21FA2CE018496F7
:10C270000F9487060E94DAA3149A01E00E9457D314
:10C2800081E00E9445BAF4EFEF16F1E0FF0609F0F5
:10C29000B5CFB2CFDD2021F29FB7F8948091020193
:10C2A0008460809302019FBFD12CBACFF4E1EF16D6
:10C2B000F10409F0B5CF9FB7F894809102018B7F0C
:10C2C000809302019FBFACCF0230C9F00C947B5524
:10C2D00084E090E00E949BBE0E94B59A882371F290
:10C2E000E091DB17F0E0EE0FFF1FEF5FF84F89A939
:10C2F0009AA9918380830E9426C902E0BFCFE09172
:10C30000DB176E2E712CF301EE0FFF1FEF5FF84F5E
:10C3100060817181072E000C880B990B0F9433B04C
:10C32000F301EE0FFF1FEE0FFF1FE054F94F2081C6
:10C330003181428153810F94B7B59F7720E030E07F
:10C3400040E85FE30F942DB087FF0BC083E393E1D8
:10C350000E9486C80E94556F4B015C0100E00C945E
:10C360007E5564E081E00E94109CE091DB1794E030
:10C37000E99FF0011124E054F94F80819181A2815D
:10C38000B3818CA39DA3AEA3BFA3CE0184960E94CC
:10C39000378A0E94759B24E1E22EF12C6FCFC12CCD
:10C3A000F0EADF2EF0E8EF2EF4E4FF2E07CBC12CED
:10C3B000D12C760120E030E04CE752E4C701B60111
:10C3C0000F9496A920E034EB40E954E403CB0F949A
:10C3D000A99080935F02FBCB2DEC3CEC4CEC5DE331
:10C3E000C701B6010F9403B818160CF450CE0C9484
:10C3F000F93A622D732D842D952D0F942DB01816BA
:10C4000014F40C947F3E0C948C3EE12CF12C00E251
:10C4100011E493CA90E021E047CB0F9420928093DF
:10C420005F02A7CCCC5BDF4F0FB6F894DEBF0FBE28
:10C43000CDBFDF91CF911F910F91FF90EF90DF90D3
:10C44000CF90BF90AF909F908F907F906F905F90B4
:10C450004F903F902F900895FC01659175918591C3
:10C4600094910895EF92FF920F931F93CF93DF93D0
:10C47000C82FD0E08E01000F111F000F111FC8013F
:10C480008F56934EE9DF98012653384E7901E80123
:10C49000C25AD84E288139814A815B810F94B8B540
:10C4A000F7016083718382839383C8018B57934E16
:10C4B000D3DF980120553D4F7901288139814A8188
:10C4C0005B810F94B8B5F701608371838283938396
:10C4D000C8018758934EC0DF0C551D4F2881398104
:10C4E0004A815B810F94B8B5F801608371838283C0
:10C4F0009383DF91CF911F910F91FF90EF9008955B
:10C500008091510490915004981781F0E82FF0E049
:10C51000ED5AFB4F208130E08F5F90914F048917D7
:10C5200008F080E080935104C90108958FEF9FEFD8
:10C5300008959091D00095FFFCCF8093D60080E0C5
:10C5400090E008958091060186FF34C080E00F944A
:10C5500059391092D2171092D3171092D417109203
:10C56000D5170F94163420E030E040EA50E4609193
:10C57000D2177091D3178091D4179091D5170F943B
:10C58000B8B56093D2177093D3178093D417909354
:10C59000D517E0917B02F0917C02608571858285E0
:10C5A00093850F9485190E94DAA360E086EB97E2E9
:10C5B0000C9402BA089589EB9CE00C94748DCF9290
:10C5C000DF92EF92FF92CF936B017C01C42F9B010E
:10C5D000AC016091D2177091D3178091D4179091CC
:10C5E000D5170F9403B887FF54C0C092D217D092CA
:10C5F000D317E092D417F092D51783B190918A05A2
:10C60000911102C084FF12C0CC2309F442C0E09112
:10C610007B02F0917C026085718582859385CF9144
:10C62000FF90EF90DF90CF900D9485190F942D3BE4
:10C630000E94DAA381E00E9413AFF82E84E00F94E9
:10C64000465D65E575E585E591E40F9485190E94E1
:10C65000DAA30F94B522882391F08091AC029091D7
:10C66000AD02A091AE02B091AF028093D217909329
:10C67000D317A093D417B093D5170F9416340F94F3
:10C68000D15C8F2DCF91FF90EF90DF90CF900C94E5
:10C6900013AFCF91FF90EF90DF90CF90089510925D
:10C6A0009D0240917C0550917D0560917E057091C1
:10C6B0007F0540939E0250939F026093A002709367
:10C6C000A102909364028093630289EB9CE00C9436
:10C6D000748D1F93CF93DF93182F80919E029091BA
:10C6E0009F02A091A002B091A10280937C0590933B
:10C6F0007D05A0937E05B0937F05C0916302D09124
:10C70000640284E690E0909364028093630289EB74
:10C710009CE00E94748D10939D02CE01DF91CF9119
:10C720001F91089540E050E0BA018DEE9FE00F9414
:10C7300050B540E050E0BA0181EF9FE00F9450B552
:10C7400060E086E69FE00F943EB560E088E69FE0FB
:10C750000F943EB560E085E69FE00F943EB560E043
:10C7600084E69FE00F943EB560E070E085E09FE0D6
:10C770000F9458B560E070E083E09FE00F9458B5E7
:10C7800060E070E081E09FE00F9458B560E070E0F9
:10C790008FEF9EE00F9458B560E070E083ED9EE06F
:10C7A0000F9458B560E070E080ED9EE00F9458B5AE
:10C7B00060E082ED9EE00F943EB560E08FEC9EE07D
:10C7C0000D943EB5F89498E088E10FB6F894A895DA
:10C7D000809360000FBE90936000FFCFC82F8FB78B
:10C7E000F894E2E0F1E09081946090838FBF6C2F29
:10C7F00083E09DE00F943EB58C2F0E94ACF5E2DF04
:10C800001F920F920FB60F92112483E0E7DF1F9261
:10C810000F920FB60F92112482E0E0DF60FF04C098
:10C8200028E5FC012083019661FF04C029E5FC0195
:10C830002083019620E2FC012193CF0161E17DE19B
:10C840000D94EFAD80918F05909190054AE050E0F6
:10C8500060E070E001960F94D1ABCB010895809118
:10C860008F05909190054AE050E060E070E00196FD
:10C870000D94D1AB2091A5093091A609BC01C90145
:10C880008554984F0F943FAE9C01909390058093F0
:10C890008F0581E0232B09F480E00895682F880F2D
:10C8A000770B8091A5099091A6098554984F0F9414
:10C8B00000BB9C019093900580938F0581E0232B12
:10C8C00009F480E00895FC01238121110D948E5616
:10C8D000089580E1EAECF7E1A2E4B7E001900D925F
:10C8E0008A95E1F708952F923F924F925F926F924F
:10C8F0007F928F929F92AF92BF92CF92DF92EF92F0
:10C90000FF920F931F93CF93DF93CDB7DEB72D9791
:10C910000FB6F894DEBF0FBECDBF8D876D835887ED
:10C920004F8320919D022B877724739470929D02F0
:10C93000823008F0E0C1282E312CF101E353F34E90
:10C9400044914C87842F082E000C990B9A87898775
:10C950004101880C991C880C991C9401255F3C4F5F
:10C96000D9018D919D910D90BC91A02D89839A83C1
:10C97000AB83BC8380939E0290939F02A093A002FE
:10C98000B093A10281E00D8401C0880F0A94EAF7F8
:10C990000F94465DF401E653F84E5F011082118258
:10C9A000128213820F94163494DFBC856B2FBB0F59
:10C9B000770B880B990B0F9433B06B017C018401CA
:10C9C0000E5B184F20E030E040E450EC0F9496A945
:10C9D000F801608371838283938320E030E040E735
:10C9E00052E460919E0270919F028091A00290910A
:10C9F000A1020F94A6B60F9452190E94DAA30F94C5
:10CA0000C32210929D02D5011D921D921D921C926F
:10CA100013970F941634F801C082D182E282F38218
:10CA200020E030E040E752E460919E0270919F0266
:10CA30008091A0029091A1020F94A6B60F94521972
:10CA40000E94DAA370929D02C4018F53934E04DDBD
:10CA50002B013C012DEC3CEC4CE85FE3C701B60137
:10CA60000F9496A9A30192010F9496A9D8016D93F2
:10CA70007D938D939C93139720E030E040E752E440
:10CA800060919E0270919F028091A0029091A102FC
:10CA90000F94A6B60F9452190E94DAA3BD814B2EB3
:10CAA000512C612C712CBE82AD82580109EA1CE127
:10CAB0006414750409F47AC00F94C32210929D0285
:10CAC000ED81FE8110821182128213820F9416343E
:10CAD00020E030E040E251ECC701B6010F9496A986
:10CAE000D5016D937D938D939C93139720E030E057
:10CAF00040E752E460919E0270919F028091A002F3
:10CB00009091A1020F94A6B60F9452190E94DAA335
:10CB10000F94C322B1E0B0939D0220E030E040E3E7
:10CB200051E4C701B6010F9496A9F50160837183A2
:10CB30008283938389819A81AB81BC8180939E0299
:10CB400090939F02A093A002B093A10220E030E056
:10CB500040E752E4BC01CD010F94A6B60F945219E0
:10CB60000E94DAA38D850F945F5B9C0144E03695AB
:10CB700027954A95E1F7AF81B885109721F0FD011F
:10CB8000E60DF71D20839F938F933F932F937F9202
:10CB90006F921F930F930F9437AFBFEF6B1A7B0AFF
:10CBA0000FB6F894DEBF0FBECDBF82CF0F94C32265
:10CBB00010929D02F101E25BFA4F6081F101E95EA2
:10CBC000FD4F108180914D058823B9F06034A8F4A1
:10CBD00040E051E0F101E05BFA4F008002C0569561
:10CBE00047950A94E2F78D850F94226F112361F027
:10CBF0004C854195612F70E004C04C85419568E0FB
:10CC000070E08D850F94D06E0F94D15C8D852ADCF9
:10CC1000F101E857FA4F81E0808369857A85719543
:10CC200061957109072E000C880B990B0F9433B096
:10CC30002AE037ED43E25CE30F9496A96B017C0197
:10CC4000F101EB5EFD4F8081682F70E080E090E0A5
:10CC50000F9433B09B01AC01C701B6010F9496A9A4
:10CC60006B017C0184010653184E9B01AC01D80175
:10CC70006D917D918D919C910F94B7B5F801608372
:10CC80007183828393830F941634D8012D913D9143
:10CC90004D915C91C701B6010F94B8B5F80160835E
:10CCA000718382839383F401EE5BF84F6083718319
:10CCB0008283938320E030E040E05FE360919E0256
:10CCC00070919F028091A0029091A1020F9496A969
:10CCD00020E030E040E752E40F94A6B60F945219DA
:10CCE0000E94DAA310929E0210929F021092A0025C
:10CCF0001092A102C0C0FD85F23009F0BCC081E0F5
:10CD00000F945939EFECFCE114911092D217109264
:10CD1000D3171092D4171092D5170F94163489ECAC
:10CD20009CE19ADB1B012C01612F110F770B880B03
:10CD3000990B0F9433B06B017C0120E030E040ECA4
:10CD40005FE3C201B1010F9496A9A70196010F9468
:10CD500096A960934A0770934B0780934C07909372
:10CD60004D0780E090E0A8E4B4E480939E029093A5
:10CD70009F02A093A002B093A10265E575E585E549
:10CD800091E40F9452190E94DAA3DCDB1092D217BF
:10CD90001092D3171092D4171092D5170F941634FF
:10CDA00085EA9CE159DB9058A70196010F9496A95A
:10CDB00060934A0770934B0780934C0790934D07FD
:10CDC00020E030E040E752E460919E0270919F02C3
:10CDD0008091A0029091A1020F94A6B60F945219CF
:10CDE0000E94DAA385EA9CE137DB9B01AC010F943A
:10CDF000B8B5A70196010F9496A960934A0770935E
:10CE00004B0780934C0790934D0780E090E0A8EC8F
:10CE1000B3E480939E0290939F02A093A002B093EC
:10CE2000A10265E575E585ED90E40F9452190E9425
:10CE3000DAA388DB82E016DB8091D2179091D317BA
:10CE4000A091D417B091D51780934A0790934B07C0
:10CE5000A0934C07B0934D0710929E0210929F0230
:10CE60001092A0021092A1020F94C32270928A0520
:10CE700080E00F9459392B8520939D022D960FB693
:10CE8000F894DEBF0FBECDBFDF91CF911F910F9100
:10CE9000FF90EF90DF90CF90BF90AF909F908F90DA
:10CEA0007F906F905F904F903F902F9008958F925A
:10CEB0009F92AF92BF92DF92EF92FF920F931F93D8
:10CEC000CF93DF930E9482A245EF5DE361E080E0B3
:10CED0000E94E19FD0909D0281E080939D02EFEC43
:10CEE000FCE1C491DD27C1950CF4D09584E00F944A
:10CEF000465D8AECE82E87E1F82EF7011086118650
:10CF0000128613860F941634E4DC89EC9CE1A4DAD3
:10CF100002E417E02DEC3CEC4CE85FE30F9496A99B
:10CF20004B015C01BE010D2E000C880B990B0F9478
:10CF300033B09B01AC01C501B4010F9496A99B01CC
:10CF4000AC01F80160857185828593850F94B8B531
:10CF5000F801608771878287938780E090E0A8E47A
:10CF6000B4E480939E0290939F02A093A002B0939A
:10CF7000A10265E575E585E591E40F9452190E94DB
:10CF8000DAA30F94D15C10929D02F70110861186EE
:10CF9000128613860F9416349CDC8AE08C9FB001B5
:10CFA0008D9F700D1124072E000C880B990B0F9488
:10CFB00033B09B01AC01F801608571858285938552
:10CFC0000F94B8B5F801608771878287938780E0F6
:10CFD00090E0A8ECB3E480939E0290939F02A0930C
:10CFE000A002B093A10265E575E585ED90E40F948C
:10CFF00052190E94DAA3D0929D0280E090E0ABE546
:10D00000B3E4F70180879187A287B3870F94163422
:10D0100081E0DF91CF911F910F91FF90EF90DF9012
:10D02000BF90AF909F908F9008953F924F925F92E4
:10D030006F927F928F929F92AF92BF92CF92DF9228
:10D04000EF92FF920F931F93CF93DF93309041079E
:10D05000332009F480C08B01EC0131FE54C088807C
:10D060009980AA80BB80FB01C080D180E280F380E0
:10D070002091AE053091AF054091B0055091B105BA
:10D08000C501B4010F9496A92B013C012091B20572
:10D090003091B3054091B4055091B505C701B60173
:10D0A0000F9496A99B01AC01C301B2010F94B8B5CE
:10D0B0002B013C012091A6053091A7054091A805C0
:10D0C0005091A905C501B4010F9496A94B015C01CB
:10D0D0002091AA053091AB054091AC055091AD056A
:10D0E000C701B6010F9496A99B01AC01C501B4011B
:10D0F0000F94B8B5688379838A839B83F801408253
:10D1000051826282738230FE26C0209139073091AD
:10D110003A0740913B0750913C07688179818A81A9
:10D120009B810F94B8B5688379838A839B83209110
:10D130003D0730913E0740913F0750914007F8016D
:10D1400060817181828193810F94B8B5F801608309
:10D15000718382839383DF91CF911F910F91FF9011
:10D16000EF90DF90CF90BF90AF909F908F907F9087
:10D170006F905F904F903F9008952F923F924F9203
:10D180005F926F927F928F929F92AF92BF92CF9257
:10D19000DF92EF92FF920F931F93CF93DF93CDB760
:10D1A000DEB728970FB6F894DEBF0FBECDBF8C0157
:10D1B0001B01FC0180819181A281B3818D839E83BB
:10D1C000AF83B887FB0180819181A281B38189837C
:10D1D0009A83AB83BC83BE016F5F7F4FCE01059600
:10D1E00024DFCD80DE80EF80F88420E030E0A901EC
:10D1F000C701B6010F942DB087FF05C01D821E82A6
:10D200001F82188612C020E030E04FE753E4C701C8
:10D21000B6010F9403B818165CF480E090E0AFE715
:10D22000B3E48D839E83AF83B887FF24F39401C05A
:10D23000F12C89809A80AB80BC8020E030E040E80F
:10D2400050ECC501B4010F942DB087FF05C080E0FC
:10D2500090E0A0E8B0EC0EC020E030E844E553E4F4
:10D26000C501B4010F9403B818164CF480E090E89F
:10D27000A4E5B3E489839A83AB83BC8303C0FF2016
:10D2800009F483C0C980DA80EB80FC808D809E80A9
:10D29000AF80B8847090410771100BC0F801808294
:10D2A0009182A282B382F101C082D182E282F382B2
:10D2B0006AC070FE1CC02091390730913A07409136
:10D2C0003B0750913C07C501B4010F94B7B54B0122
:10D2D0005C0120913D0730913E0740913F075091FE
:10D2E0004007C701B6010F94B7B56B017C0171FE11
:10D2F0004AC02091290730912A0740912B0750916D
:10D300002C07C501B4010F9496A92B013C01209173
:10D310002D0730912E0740912F0750913007C701FC
:10D32000B6010F9496A99B01AC01C301B2010F9401
:10D33000B8B5F801608371838283938320913107AC
:10D34000309132074091330750913407C501B40141
:10D350000F9496A94B015C01209135073091360757
:10D360004091370750913807C701B6010F9496A92D
:10D370009B01AC01C501B4010F94B8B5F101608304
:10D38000718382839383FF24F3948F2D28960FB6A5
:10D39000F894DEBF0FBECDBFDF91CF911F910F91EB
:10D3A000FF90EF90DF90CF90BF90AF909F908F90C5
:10D3B0007F906F905F904F903F902F9008951092C4
:10D3C000E0178091CA068B7F8093CA0608958091EA
:10D3D000F7049091F8042091F9043091FA04821B2B
:10D3E000930B8F779927089586EA9FE00F941DB5D8
:10D3F00091E0811101C090E0892F0895682F87EF97
:10D400009FE00D943EB587EF9FE00D941DB52091F0
:10D41000F9043091FA048091F7049091F80482178E
:10D42000930771F0F901E958FB4F80812F5F3F4F5F
:10D430002F7733273093FA042093F90490E008956E
:10D440008FEF9FEF08951F920F920FB60F92112446
:10D450000BB60F922F933F934F936F937F938F93BE
:10D460009F93EF93FF938091C80084FF03C0809146
:10D47000CE001DC04091CE008091DC178130B9F400
:10D480002091F7043091F804C90101968F7799270C
:10D490006091F9047091FA048617970741F0F90139
:10D4A000E958FB4F40839093F8048093F704FF9171
:10D4B000EF919F918F917F916F914F913F912F911C
:10D4C0000F900BBE0F900FBE0F901F9018951F92DC
:10D4D0000F920FB60F9211240BB60F922F933F931A
:10D4E0004F936F937F938F939F93EF93FF938091CD
:10D4F000C00084FF03C08091C6001DC04091C600DB
:10D500008091DC17811117C02091F7043091F80445
:10D51000C90101968F7799276091F9047091FA04F7
:10D520008617970741F0F901E958FB4F4083909324
:10D53000F8048093F704FF91EF919F918F917F9171
:10D540006F914F913F912F910F900BBE0F900FBE97
:10D550000F901F9018959091DC17911107C0909132
:10D56000C00095FFFCCF8093C6000895913031F440
:10D570009091C80095FFFCCF8093CE000895EBDF1B
:10D5800080E090E00895CF93DF93EC01FE01849159
:10D59000882319F0E0DF2196F9CFDF91CF9108952C
:10D5A0004F925F926F927F928F929F92AF92BF92B3
:10D5B000CF92DF92EF92FF920F931F93CF93DF935F
:10D5C000CDB7DEB7A0970FB6F894DEBF0FBECDBFC4
:10D5D0006115710581059105C1F480E3A0960FB630
:10D5E000F894DEBF0FBECDBFDF91CF911F910F9199
:10D5F000FF90EF90DF90CF90BF90AF909F908F9073
:10D600007F906F905F904F90A6CF9E012F5F3F4F0E
:10D610007901812C912C54018901442E512C612CCB
:10D62000712C3FEF831A930AA30AB30AA301920154
:10D630000F947CB5F70161937F01B901CA016115AF
:10D6400071058105910569F77401C12CD12CF1E0B8
:10D650008F1A9108A108B108F401EC19FD09E00F37
:10D66000F11F80818A3010F4805D01C0895C73DF16
:10D670002FEFC21AD20ACE14DF0471F7A0960FB6AC
:10D68000F894DEBF0FBECDBFDF91CF911F910F91F8
:10D69000FF90EF90DF90CF90BF90AF909F908F90D2
:10D6A0007F906F905F904F900895CF92DF92EF92AE
:10D6B000FF926B017C0197FF0AC08DE24CDFF09472
:10D6C000E094D094C094C11CD11CE11CF11C4AE030
:10D6D000C701B601FF90EF90DF90CF9061CF8F929E
:10D6E0009F92AF92BF92CF92DF92EF92FF92CF9331
:10D6F000DF936B017C01C42F20E030E0A9010F947F
:10D700002DB087FF06C08DE226DFF7FAF094F7F818
:10D71000F094D0E060E070E080E09FE3DC1741F03F
:10D7200020E030E040E251E40F94A6B6DF5FF6CF90
:10D730009B01AC01C701B6010F94B8B56B017C0128
:10D740000F941DB74B015C010F9431B09B01AC01EC
:10D75000C701B6010F94B7B56B017C014AE0C50162
:10D76000B4011EDFCC2311F08EE2F5DECC2309F1EB
:10D7700020E030E040E251E4C701B6010F9496A9E1
:10D780004B015C010F9417B76B01770FEE08FF0890
:10D79000C701B6018ADFC701B6010F9433B09B0100
:10D7A000AC01C501B4010F94B7B56B017C01C15048
:10D7B000DDCFDF91CF91FF90EF90DF90CF90BF90C2
:10D7C000AF909F908F9008958AE0C5CECF93DF935E
:10D7D000EC018991882311F0BEDEFBCFDF91CF9160
:10D7E0000895F4DFF1CF44EC50E067E77BE186E099
:10D7F00097E10F94DBAD0F9406240E94D3D80E94CA
:10D80000BAB88FE594E6BFDE85E59BE1BCDEDCCFF0
:10D810004F925F926F927F928F929F92AF92BF9240
:10D82000EF92FF920F931F93CF93DF9300D01F923D
:10D83000CDB7DEB786E592E3A0E0B0E089839A83B6
:10D84000AB83BC8346E0E42E47E1F42E04E110E014
:10D85000C8010F941DB5F70181937F010F5F1F4F22
:10D8600008311105A9F743E050E066E077E1CE0109
:10D8700001960F941BBB892B09F009C136E0E32EFA
:10D8800037E1F32E04E110E0C8010F941DB5F70154
:10D8900081937F010F5F1F4F083D1105A9F70E947B
:10D8A000BAB800E010E0B80164567F4F9B012A5FD0
:10D8B000384E94E0915038F0F901E90FF11D808164
:10D8C0008F3FC1F307C06958744E44E050E0C9016E
:10D8D0000F94DBADB80164557F4FCB018A5F984E42
:10D8E000FC0180809180A280B3808B208A208920D7
:10D8F000809431F46958744E44E050E00F94DBADED
:10D900000C5F1F4F0031110571F60AE117E182EA41
:10D91000E82E87E1F82E94EC892E99E0992EA12C1F
:10D92000B12C20EC422E23E0522E612C712C20E0F1
:10D9300030E048E453E4F801608171818281938191
:10D940000F9403B818164CF480E090E0A8E4B3E418
:10D95000F80180839183A283B38320E030E048EC18
:10D9600052E4F70160817181828193810F9403B841
:10D9700018164CF480E090E0A8ECB2E4F701808344
:10D980009183A283B383F80180899189A289B389A5
:10D99000853C9940A105B10528F0F801808A918A5B
:10D9A000A28AB38AF70180899189A289B389813CCF
:10D9B0009340A105B10528F0F701408A518A628A97
:10D9C000738A0C5F1F4FF4E0EF0EF11C27E1023267
:10D9D000120709F0ACCF8091C2178F3F19F480E194
:10D9E0008093C2178091C3178F3F19F480E1809311
:10D9F000C3178091C4178F3F19F480E18093C41737
:10DA00008091C5178F3F19F480E28093C51760910C
:10DA1000C21770E080E00F946D5C6091C31770E0F6
:10DA200081E00F946D5C6091C41770E082E00F9408
:10DA30006D5C6091C51770E083E00F946D5C84E0CD
:10DA4000815040F0E82FF0E0EA53F84E90819F3F7C
:10DA5000B9F310C080913A1790913B17A0913C17F1
:10DA6000B0913D178093C6179093C717A093C8171E
:10DA7000B093C9170F9406240E94D3D88FE594E67B
:10DA800082DD8BE39BE17FDD9FDE91E015C0ABDEA5
:10DA900084E190E00F941DB58F3F69F485E190E03B
:10DAA0000F941DB58F3F39F486E190E00F941DB5BA
:10DAB00091E08F3F09F090E0892F0F900F900F9029
:10DAC0000F90DF91CF911F910F91FF90EF90BF903A
:10DAD000AF909F908F907F906F905F904F90089540
:10DAE00061EC73E086E097E10F9414BB64EC86E090
:10DAF00097E10F94016165EC73E086E097E10F9484
:10DB000014BB64E086E097E10F9401618FE594E631
:10DB10003ADD8BE29BE137DD57CE853010F00F9474
:10DB2000B9BA21E030E0A90102C0440F551F8A951F
:10DB3000E2F7CA01809590917E07892380937E0742
:10DB40000895CF93813069F0C82F8FEF8C0FF9DFE4
:10DB5000C15021E030E001C0220FCA95EAF7822BC4
:10DB600001C081E0CF9108958EBD0DB407FEFDCFB9
:10DB70008EB50895459885E0F7DF8FEFF5DF459A7C
:10DB800080FDF8CF0895CF93DF9300D01F92CDB7DB
:10DB9000DEB749835A836B837C83E6DF8B81E4DFC6
:10DBA0008A81E2DF8981E0DF0F900F900F900F9064
:10DBB000DF91CF9108954598E6DF459A0895EF9259
:10DBC000FF920F931F93CF93DF937A0189014598BA
:10DBD000AB01BC0182E0D7DFE7010E0D1F1DC017AE
:10DBE000D10719F08991C0DFFACF459ADF91CF9123
:10DBF0001F910F91FF90EF900895EF92FF920F9376
:10DC00001F93CF93DF937A0189014598AB01BC0143
:10DC100083E0B9DFE7010E0D1F1DC017D10721F00A
:10DC20008FEFA2DF8993F9CF459ADF91CF911F91B2
:10DC30000F91FF90EF900895459886E095DF459A03
:10DC40000895CF93459A3D9A8CE58CBD1DBC4598AF
:10DC500080E98ADF80E088DF80E086DF80E084DFA3
:10DC60008FEF82DFC82F8FEF7FDF982F459ACF3E4F
:10DC700011F0C83C19F481E0913109F080E0CF91B6
:10DC800008951F920F920FB60F9211240BB60F92A8
:10DC90002F933F934F935F936F937F938F939F93B4
:10DCA000AF93BF93EF93FF932091D60080915004E0
:10DCB00090915104E82FF0E0ED5AFB4F20838F5FE5
:10DCC00020914F04821708F080E0891719F08093A3
:10DCD000500404C089E19BE10F945FAFFF91EF9185
:10DCE000BF91AF919F918F917F916F915F914F9174
:10DCF0003F912F910F900BBE0F900FBE0F901F9072
:10DD00001895FF920F931F93CF93DF938C01F090A0
:10DD10005104C0915004D0914F04D1500F94F6ADEE
:10DD2000F801E80FF11D0195802F8E0FC9F0CF1576
:10DD3000C9F0C15008F4CD2F31979491AC2FB0E0C9
:10DD4000A15BBB4F14968C91981771F39D3019F419
:10DD50008A3051F4E9CF9A3039F48D3029F304C078
:10DD600081E003C080E001C08FEFDF91CF911F9170
:10DD70000F91FF9008951F920F920FB60F921124EA
:10DD80000BB60F928F939F93EF93FF939FB7F894E7
:10DD9000E2E0F1E080818B7F80839FBFFF91EF9174
:10DDA0009F918F910F900BBE0F900FBE0F901F9001
:10DDB00018951F920F920FB60F9211240BB60F9267
:10DDC0008F939F93EF93FF939FB7F894E2E0F1E076
:10DDD0008081846080839FBFFF91EF919F918F919D
:10DDE0000F900BBE0F900FBE0F901F9018953FB76E
:10DDF000F8948091780590917905A0917A05B09179
:10DE00007B052091B200B89B05C02F3F19F0019609
:10DE1000A11DB11D3FBFBA2FA92F982F8827820FB0
:10DE2000911DA11DB11DBC01CD0142E0660F771F00
:10DE3000881F991F4A95D1F708958F929F92AF92AC
:10DE4000BF92CF92DF92EF92FF926B017C01CFDF06
:10DE50004B015C01C114D104E104F104E9F0C7DF16
:10DE6000DC01CB0188199909AA09BB09883E9340B6
:10DE7000A105B10578F321E0C21AD108E108F10843
:10DE800088EE880E83E0981EA11CB11CC114D10439
:10DE9000E104F10421F7DECFFF90EF90DF90CF9007
:10DEA000BF90AF909F908F9008952FB7F894609196
:10DEB0000D0670910E0680910F06909110062FBFEF
:10DEC00008958F929F92AF92BF92CF92DF92EF927E
:10DED000FF928091F706811145C0E7DF6B017C015D
:10DEE000209104022223B1F140916002413091F16E
:10DEF0008091220290912302A0912402B0912502E8
:10DF000046015701881A990AAA0ABB0A30E0A8EE0E
:10DF1000B3E00F94A8B586169706A806B90614F1C3
:10DF2000443089F044F44230ACF08FE594E62BDBCA
:10DF300088E69CE10DC0453069F48FE594E623DB6B
:10DF40008BE39CE105C08FE594E61DDB82E59CE157
:10DF50001ADB3ADCC0922202D0922302E092240221
:10DF6000F0922502FF90EF90DF90CF90BF90AF909E
:10DF70009F908F9008951F920F920FB60F921124C9
:10DF80002F933F938F939F93AF93BF9380910D06F1
:10DF900090910E06A0910F06B09110063091770572
:10DFA00023E0230F2D3720F40196A11DB11D05C0DC
:10DFB00026E8230F0296A11DB11D209377058093BB
:10DFC0000D0690930E06A0930F06B0931006809155
:10DFD000780590917905A0917A05B0917B0501961D
:10DFE000A11DB11D8093780590937905A0937A05C2
:10DFF000B0937B05BF91AF919F918F913F912F91EE
:10E000000F900FBE0F901F901895982F9F7083FF51
:10E0100004C080917B00886003C080917B00877F73
:10E0200080937B0080917C009770887F892B809300
:10E030007C0008951092300610921F064091FB0458
:10E040005091FC04E0E2F6E080E090E061E070E0F6
:10E050009B01082E02C0220F331F0A94E2F72423EB
:10E060003523232B11F411821082019632968830C9
:10E07000910571F708952F923F924F925F926F92A0
:10E080007F928F929F92AF92BF92CF92DF92EF9248
:10E09000FF920F931F93CF93DF93CDB7DEB7CD5C85
:10E0A000D1090FB6F894DEBF0FBECDBF182F81E0A7
:10E0B0000F94593981E00E94568D111125C010929C
:10E0C00000071092FF0619821A821B821C82CE0161
:10E0D00001960F94870661E080EC9FE00F943EB5B7
:10E0E00060E08FEB9FE00F943EB560E08EEB9FE029
:10E0F0000F943EB560E08DEB9FE00F943EB560E07D
:10E100008CEB9FE00F943EB580E00E94B3A20F9489
:10E1100019700E947C9610928705109286051092C5
:10E1200088051092890510928A0581E00E94696332
:10E13000CC54DF4F99838883C45BD0408FE891E251
:10E140000E9486C841E060E070E080EA90E40E94AE
:10E15000DF620E94DAA30E94696440E050E061E05F
:10E1600080E00E94736440E050E061E081E00E9442
:10E1700073640F9416340F94C32210929D0220E012
:10E1800030E040EA50E46091CA177091CB1780915B
:10E19000CC179091CD170F94B8B56093CA177093B0
:10E1A000CB178093CC179093CD1720E030E040EA56
:10E1B00050E46091CE177091CF178091D017909155
:10E1C000D1170F94B8B56093CE177093CF17809383
:10E1D000D0179093D11760E070E080EA91E40F943B
:10E1E00085190E94DAA30E945767882311F40C94C2
:10E1F0008C8185E591E20E94AFC8112339F085E258
:10E2000091E20E9486C846E152E206C085E091E2B2
:10E210000E9486C842E152E263E080E00E94E19FF2
:10E220000E94DB62111120C084E08093600240E014
:10E2300060E08AEE90E20E949EC8882321F082EC82
:10E2400090E20E94AFC88CE290E20E94AFC882E0E8
:10E250008093600285E091E20E9486C84EE052E21F
:10E2600063E080E00E94E19F00919D0210929D0278
:10E2700020E030E040E85FE36091D2177091D3175F
:10E280008091D4179091D5170F94B7B56093D2179A
:10E290007093D3178093D4179093D51760E070E0F4
:10E2A00080EA91E40F9485190E94DAA3C12CD12C45
:10E2B00040EAE42E40E4F42EC092D217D092D31755
:10E2C000E092D417F092D51781E080939D0284E00C
:10E2D0000F94465D60E070E080EA91E40F94851948
:10E2E0000E94DAA30F94D15C00939D0282E00E9409
:10E2F000C7A32DEC3CEC44EA50E40F942DB0181663
:10E3000014F40C94888182E00E94C7A323E333E3D2
:10E310004BE950E40F9403B887FF02C00C94888146
:10E320001123D9F0CC54DF4F88819981C45BD04050
:10E330000E944F630E9483980E947E940E94EC9FEB
:10E34000882311F40C943A815ED8803F11F00C942C
:10E35000848181E053D80C9484818AEF4FD881EA7C
:10E360009DE00F941DB52BE0829FC001112460E059
:10E3700070E0805B924F0F9458B50E94DB6284EC92
:10E38000E3EDFBE0DF011D928A95E9F783ED93E26F
:10E39000FAD861E070E080E090E087D915DA85E096
:10E3A00091E20E9486C8C092D217D092D317E09211
:10E3B000D417F092D517B2E0C256DF4FB883CE59CA
:10E3C000D040EEEAF3E2CE55DF4FF983E883C25A3C
:10E3D000D04022ED3BE0C456DF4F39832883CC592F
:10E3E000D040A2963FAF2EAFA2976E96FFAFEEAF92
:10E3F0006E97ED961FAEED97A6961FAE1EAEA69732
:10E400000E94DB6263E080E00E94109CA696EEAD65
:10E41000FFADA6973196A696FFAFEEAFA697FF93F6
:10E42000EF938EEC93E29F938F930E94819B65E51F
:10E4300075E585E591E40E943E946E96EEADFFADE4
:10E440006E9785919591A591B4918093CA179093F9
:10E45000CB17A093CC17B093CD176E96EEADFFAD52
:10E460006E97349685919591A591B4918093CE172E
:10E470009093CF17A093D017B093D11760E070E0BE
:10E4800088E492E40E943E940E94DAA38AE192E238
:10E490009F938F930F9437AF0E943ECD8091700071
:10E4A0008B7F80937000EF9880916F008D7F8093B9
:10E4B0006F000FB6F894A8958091600088618093F2
:10E4C0006000109260000FBE1092850510928405C6
:10E4D0008CEA9EEE909383058093820587EA9EEEF8
:10E4E00090938105809380050091DE161091DF16D0
:10E4F0002091E0163091E1164091DA165091DB162A
:10E500006091DC167091DD168091D6169091D71629
:10E51000A091D816B091D9163F932F931F930F93C4
:10E520007F936F935F934F93BF93AF939F938F931B
:10E530008AEB92E29F938F930F9437AF4090D61659
:10E540005090D7166090D8167090D916D42CC52C40
:10E550008091DA169091DB16A091DC16B091DD1651
:10E56000E0968CAF9DAFAEAFBFAFE097AD96BFACBE
:10E57000AD97AE96AFACAE978091DE169091DF1658
:10E58000A091E016B091E1164C010FB6F894DEBFF1
:10E590000FBECDBF31E3232E32E2332E25E08216AB
:10E5A00027EF92060CF471C01A8219821F921F92F3
:10E5B000B3E0BF93E4E8EF931F92F4E6FF939F92DA
:10E5C0008F92AF92BF92CF92DF923F922F920F9491
:10E5D00037AF0FB6F894DEBF0FBECDBF89819A81E9
:10E5E000803D924030F089819A81803A954050F583
:10E5F00012C0CE0101967C0100E010E024E833E077
:10E60000A4016B2D7A2D8D2D9C2D0F94D97781111E
:10E610000C948E81E8CFDE0111967D0100E010E0C0
:10E620002CE73CEFA401445651096B2D7A2D8D2D1A
:10E630009C2D0F94D977882329F089819A81805362
:10E640009D4F1FC089819A818037984010F00C94AB
:10E65000CC84FE0131967F0104EB10E024E833E026
:10E66000A401485C51096B2D7A2D8D2D9C2D0F94A2
:10E67000D977882311F40C94CC8489819A818056AF
:10E680009A4F9A8389830C948E810091DE161091A3
:10E69000DF162091E0163091E1164091DA16509184
:10E6A000DB166091DC167091DD168091D616909184
:10E6B000D716A091D816B091D9163F932F931F93D8
:10E6C0000F937F936F935F934F93BF93AF939F93FA
:10E6D0008F9389E692E29F938F930F9437AF0FB693
:10E6E000F894DEBF0FBECDBF0FEF1FEFD2C120E207
:10E6F000420E511CAA968EAD9FADAA970297AA967C
:10E700009FAF8EAFAA97411494E0590611F00C9474
:10E71000548281EF92E29F938F930F9437AF0F90C3
:10E720000F90A5EF2A2EAFE03A2E8101B0E29B2E8A
:10E7300083EFC82E82E2D82E91EFE92E92E2F92ED5
:10E74000A12CB12CF801EA0DFB1D80811F928F9343
:10E75000DF92CF920F9437AFBFEFAB1ABB0A0F9087
:10E760000F900F900F90E0E2AE16B10459F7F1EF61
:10E77000AF2EF2E2BF2EFF92EF920F9437AF9A9432
:10E78000005E1F4F0F900F909110DACFBF92AF92A3
:10E790000F9437AF0F900F90E5EFFFE020E030E0EF
:10E7A00040E050E0819181110C94D4854F5F5F4F20
:10E7B00063E1E53FF607B1F7CA01820F931F853881
:10E7C000934014F00C94DC8568961FAE68976296AF
:10E7D0001FAE629722961FAE2297198285EF93E1B2
:10E7E000892B11F40C94FA85AE014F5A5F4FBE018C
:10E7F000695A7F4F85EF93E10F949A76082F8DE049
:10E8000094E1892B11F40C94FD85AE014F5F5F4FAD
:10E81000BE016F5B7F4F8DE094E10F949A76801775
:10E8200010F00C94FE8568966FAD689762961FADE8
:10E830006297083510F40C943E8670E080E090E01A
:10E840000F9433B020E030E040EB50E40F94B8B5C3
:10E850002B013C0165966CAF7DAF8EAF9FAF659786
:10E86000612F70E080E090E00F9433B020E030E062
:10E8700040EB50E40F94B8B54B015C0125966CAFAA
:10E880007DAF8EAF9FAF259780E090E0A0E9B0E428
:10E8900089839A83AB83BC83AE014F5F5F4FBE0118
:10E8A0006F5B7F4FCE018F5A9F4F0F944B73A30125
:10E8B000920165966CAD7DAD8EAD9FAD65970F9461
:10E8C000B7B56B017C019F7720E030E040E450E475
:10E8D0000F9403B8181614F40C940586A50194013E
:10E8E00025966CAD7DAD8EAD9FAD25970F94B7B5D8
:10E8F0009F7720E030E040E450E40F9403B818160E
:10E9000014F40C94058620E030E040EA50E469817C
:10E910007A818B819C810F94B7B59F7720E030E09E
:10E9200040E450E40F9403B8181614F40C940586D0
:10E93000C058DF4F28813981C058D040B901330F0A
:10E94000880B990B0F9433B06B017C0120E030E011
:10E9500048E751E465966CAD7DAD8EAD9FAD659792
:10E960000F94B7B520E030E040E852E40F9496A948
:10E970009B01AC01C701B6010F94B8B56B017C01D6
:10E9800065966CAF7DAF8EAF9FAF6597C457DF4F75
:10E99000A881B981CC58D040BD01BB0F880B990B21
:10E9A0000F9433B04B015C0120E030E048E751E4C4
:10E9B00025966CAD7DAD8EAD9FAD25970F94B7B507
:10E9C00020E030E040E852E40F9496A99B01AC01AE
:10E9D000C501B4010F94B8B525966CAF7DAF8EAF6D
:10E9E0009FAF25972AE037ED43E25CE30F9496A9A9
:10E9F0009F938F937F936F932AE037ED43E25CE31D
:10EA0000C701B6010F9496A99F938F937F936F933D
:10EA100088EF92E29F938F930F9437AF20E030E01E
:10EA200040E05FE325966CAD7DAD8EAD9FAD259743
:10EA30000F94B8B50F9417B76B017C0120E030E05C
:10EA400040E05FE365966CAD7DAD8EAD9FAD6597A3
:10EA50000F94B8B50F9417B7DC01CB0100E028EC98
:10EA600030E0C057DF4F48815981C059D040B601CE
:10EA70000E9484F40FB6F894DEBF0FBECDBF00E055
:10EA800010E0D1011D921D01B5ED2B16B6E13B063C
:10EA9000C1F780E693E29F938F930F9437AF0F9463
:10EAA000331A80917000846080937000EF9A809197
:10EAB0006F00826080936F0098E288E10FB6F8944F
:10EAC000A895809360000FBE9093600080916000D5
:10EAD00080648093600010928505109284051092E6
:10EAE00083051092820510928105109280050F9087
:10EAF0000F900D3FEFEF1E0731F00F3F1F4F11F446
:10EB00000C94E48004C021E0ED962FAFED9720E057
:10EB100030E0A901A296AEADBFADA29711966D915E
:10EB20007D918D919C9114970F9496A92091CA176D
:10EB30003091CB174091CC175091CD170F94B8B5A9
:10EB4000A296EEADFFADA297618372838383948317
:10EB5000C090CE17D090CF17E090D017F090D1177B
:10EB600020E030E0A90165817681878190850F944E
:10EB700096A9A70196010F94B8B5A296AEADBFAD08
:10EB8000A29715966D937D938D939C93189720E093
:10EB900030E040E850ECC701B6010F942DB087FF7C
:10EBA0000CC080E090E0A0E8B0EC8093CE1790938A
:10EBB000CF17A093D017B093D11720E030E040E4F6
:10EBC00050E46091D2177091D3178091D41790912F
:10EBD000D5170F94B8B56093D2177093D31780935D
:10EBE000D4179093D5176E96EEADFFAD6E9738960D
:10EBF0006E96FFAFEEAF6E97A2962EAD3FADA29789
:10EC0000285F3F4FA2963FAF2EAFA297A6968EAD3C
:10EC10009FADA697049709F0F3CBED969FADED97C6
:10EC2000992349F0C256DF4FA881CE59D040A13078
:10EC300011F0B1E0C1CB8DEE91E29F938F930F94D1
:10EC400037AF80E090E00E949BBE0F900F9020E0D5
:10EC500030E040E950EC6091D70B7091D80B809177
:10EC6000D90B9091DA0B0F942DB087FF24C08DEA59
:10EC700093E20E94C36A0E94E46B8BE793E20E94D6
:10EC8000C36A6091D70B7091D80B8091D90B90918A
:10EC9000DA0B42E00E946F6B87E793E20E94C36A3F
:10ECA00060E070E080E990EC0F942463B2E0AD96F0
:10ECB000BFAFAD9703C0AD961FAEAD971092030CDA
:10ECC0001092040C1092050C1092060C1092070C76
:10ECD0001092080C1092090C10920A0CE4E6CC5722
:10ECE000DF4FE883C458D040A4961CAE1DAE1EAEC4
:10ECF0001FAEA497A8961CAE1DAE1EAE1FAEA89761
:10ED00009E012F5F3F4F6A963FAF2EAF6A97CE01AD
:10ED10008F5B9F4F6C969FAF8EAF6C97A8966CAD34
:10ED20007DAD8EAD9FADA8970F94A3B6AC966CAF9A
:10ED30007DAF8EAF9FAFAC97A8966CAD7DAD8EAD1D
:10ED40009FADA8970F9464B9C457DF4F6883798348
:10ED50008A839B83CC58D040A4966CAD7DAD8EAD9C
:10ED60009FADA4970F94A3B6C057DF4F68837983F4
:10ED70008A839B83C059D040A4966CAD7DAD8EAD87
:10ED80009FADA4970F9464B9CC56DF4F6883798305
:10ED90008A839B83C459D04080E46A96AEADBFADF0
:10EDA0006A971D928A95E9F780E16C96EEADFFAD0A
:10EDB0006C9711928A95E9F780E090E00E949BBEE3
:10EDC0008091030C9091040CA091050CB091060C5D
:10EDD000C256DF4F88839983AA83BB83CE59D04024
:10EDE0008091070C9091080CA091090CB0910A0C2D
:10EDF000CC55DF4F88839983AA83BB83C45AD04004
:10EE0000DE01AF5BBF4FC856DF4FB983A883C85937
:10EE1000D040FE013196E696FFAFEEAFE69700E0F8
:10EE2000CC56DF4F88819981AA81BB81C459D040DB
:10EE3000B058EC968CAF9DAFAEAFBFAFEC97C0575C
:10EE4000DF4F88819981AA81BB81C059D040B058D9
:10EE5000C458DF4F88839983AA83BB83CC57D040A3
:10EE6000C457DF4F88819981AA81BB81CC58D0409B
:10EE7000B058C058DF4F88839983AA83BB83C0589A
:10EE8000D040212C312C10E052ED452E5BE0552E68
:10EE900064E0762EC12CD12C7601013011F40C9453
:10EEA0006286113011F40C946E86002321F1023039
:10EEB00081F4D20111962D913D914D915C91149761
:10EEC000C058DF4F688179818A819B81C058D040CA
:10EED0000DC0F2012581368147815085C458DF4F2E
:10EEE000688179818A819B81CC57D0400F9496A903
:10EEF0004B015C0106C0812C912CE0E8AE2EEFE3C3
:10EF0000BE2E112311F1123081F4D20111962D91F0
:10EF10003D914D915C911497C058DF4F6881798184
:10EF20008A819B81C058D0400DC0F2012581368175
:10EF300047815085C458DF4F688179818A819B81E0
:10EF4000CC57D0400F9496A904C060E070E080E8F0
:10EF50009FE39B01AC01C501B4010F9496A99B01ED
:10EF6000AC01C701B6010F94B8B56B017C01002359
:10EF7000E1F11123D1F1023011F00C944286D2015B
:10EF800011962D913D914D915C911497AC966CAD7D
:10EF90007DAD8EAD9FADAC970F9496A94B015C01F2
:10EFA000113011F40C945C86123011F00C944F86E1
:10EFB000D20111962D913D914D915C911497AC9693
:10EFC0006CAD7DAD8EAD9FADAC970F9496A99B01B6
:10EFD000AC01C501B4010F9496A99B01AC01C70116
:10EFE000B6010F94B8B56B017C017A94F8E04F0E2E
:10EFF000511C711052CFE696EEADFFADE697E20DD3
:10F00000F31DC082D182E282F3821F5F24E0220ED0
:10F01000311C30E12316310409F036CF42ED242EA5
:10F020004BE0342E8EEA93E26E969FAF8EAF6E97D2
:10F03000C857DF4F1882C858D040C855DF4F1882D4
:10F04000C85AD040C455DF4F1882CC5AD04010E087
:10F05000002331F1013059F1023081F4D1011196D0
:10F060002D913D914D915C911497C058DF4F68816F
:10F0700079818A819B81C058D0400DC0F1012581E2
:10F08000368147815085C458DF4F688179818A81F4
:10F090009B81CC57D0400F9496A94B015C010AC0CC
:10F0A000812C912C30E8A32E3FE3B32E03C0812C9A
:10F0B000912C5401D10111964D905D906D907C90F2
:10F0C0001497A3019201AC966CAD7DAD8EAD9FAD52
:10F0D000AC970F9496A96B017C01D10115968D9187
:10F0E0009D910D90BC91A02DE4968CAF9DAFAEAFDD
:10F0F000BFAFE4976E96EEADFFAD6E97859195919B
:10F10000A591B491C055DF4F88839983AA83BB83AF
:10F11000C05BD040E4962CAD3DAD4EAD5FADE49705
:10F12000CC56DF4F688179818A819B81C459D04058
:10F130000F9496A99B01AC01C701B6010F94B7B516
:10F14000C256DF4F288139814A815B81CE59D04038
:10F150000F94B8B5C055DF4F288139814A815B8152
:10F16000C05BD0400F94B7B59B01AC01C501B401A1
:10F170000F9496A99B01AC01C857DF4F6881C8580E
:10F18000D040C855DF4F7881C85AD040C455DF4FB2
:10F190008881CC5AD040912F0F94B8B5C857DF4F13
:10F1A000688379838A839B83C858D0400023A9F061
:10F1B0000130B9F00230D9F0E4962CAD3DAD4EAD42
:10F1C0005FADE497EC966CAD7DAD8EAD9FADEC97E9
:10F1D0000F9496A96B017C010AC0C12CD12C760139
:10F1E00006C0C12CD12C20E8E22E2FE3F22E6E9621
:10F1F000EEADFFAD6E97349685909590A590B49046
:10F20000A3019201C457DF4F688179818A819B8174
:10F21000CC58D0400F9496A92B013C01E4962CAD1C
:10F220003DAD4EAD5FADE497C057DF4F688179814A
:10F230008A819B81C059D0400F9496A99B01AC0153
:10F24000C301B2010F94B8B5CC55DF4F2881398185
:10F250004A815B81C45AD0400F94B8B5A50194018E
:10F260000F94B7B59B01AC01C701B6010F9496A9E5
:10F270009B01AC01C857DF4F688179818A819B81EE
:10F28000C858D0400F94B8B5C857DF4F6883C858E6
:10F29000D040C855DF4F7883C85AD040C455DF4F9F
:10F2A0008883CC5AD040192F6E96AEADBFAD6E9705
:10F2B00018966E96BFAFAEAF6E97B8E02B0E311CAE
:10F2C000E2EF2E16EBE03E0609F0C2CEDC01CB01E8
:10F2D000B058C856DF4FE881F981C859D0408193B2
:10F2E0009193A193B193C856DF4FF983E883C8592E
:10F2F000D0400F5FE6962EAD3FADE697205F3F4FC3
:10F30000E6963FAF2EAFE697043009F0BACD2596CA
:10F310008CAD9DADAEADBFAD2597AC968CAF9DAF1E
:10F32000AEAFBFAFAC978D819E81AF81B885E896B7
:10F330008CAF9DAFAEAFBFAFE89789859A85AB859F
:10F34000BC85E4968CAF9DAFAEAFBFAFE4978D8523
:10F350009E85AF85B889EC968CAF9DAFAEAFBFAF41
:10F36000EC9789819A81AB81BC81C458DF4F888337
:10F370009983AA83BB83CC57D04029968CAD9DAD91
:10F38000AEADBFAD2997C058DF4F88839983AA835C
:10F39000BB83C058D04089899A89AB89BC89C4573E
:10F3A000DF4F88839983AA83BB83CC58D040898D53
:10F3B0009A8DAB8DBC8DC057DF4F88839983AA830C
:10F3C000BB83C059D0408D8D9E8DAF8DB8A1CC56DA
:10F3D000DF4F88839983AA83BB83C459D0408D892A
:10F3E0009E89AF89B88DC856DF4F88839983AA83D9
:10F3F000BB83C859D0402D968CAD9DADAEADBFAD91
:10F400002D97C857DF4F88839983AA83BB83C85839
:10F41000D04089A19AA1ABA1BCA1C855DF4F888378
:10F420009983AA83BB83C85AD0408DA19EA1AFA166
:10F43000B8A5C455DF4F88839983AA83BB83CC5A70
:10F44000D0408DA59EA5AFA5B8A9C055DF4F888334
:10F450009983AA83BB83C05BD04089A59AA5ABA53D
:10F46000BCA5CA54DF4F88839983AA83BB83C65B3C
:10F47000D04061968CAD9DADAEADBFAD6197C65429
:10F48000DF4F88839983AA83BB83CA5BD04089A955
:10F490009AA9ABA9BCA9C254DF4F88839983AA83D8
:10F4A000BB83CE5BD0408DA99EA9AFA9B8ADCE538A
:10F4B000DF4F88839983AA83BB83C25CD04089AD28
:10F4C0009AADABADBCADCA53DF4F88839983AA8395
:10F4D000BB83C65CD04021968CAD9DADAEADBFADBB
:10F4E0002197C653DF4F88839983AA83BB83CA5C65
:10F4F000D04014E6C12CD12C7601460157012601DB
:10F500003701A3019201E8966CAD7DAD8EAD9FAD44
:10F51000E8970F9496A99B01AC01AC966CAD7DADBC
:10F520008EAD9FADAC970F94B7B52B013C01A501F3
:10F530009401E4966CAD7DAD8EAD9FADE4970F94D4
:10F5400096A99B01AC01C301B2010F94B7B52B0181
:10F550003C01A7019601EC966CAD7DAD8EAD9FADE3
:10F56000EC970F9496A99B01AC01C301B2010F94D3
:10F57000B7B5C458DF4F288139814A815B81CC57A8
:10F58000D0400F94A6B6A0966CAF7DAF8EAF9FAF64
:10F59000A0979B01AC01C457DF4F688179818A81B4
:10F5A0009B81CC58D0400F9496A99B01AC01C058C8
:10F5B000DF4F688179818A819B81C058D0400F9448
:10F5C000B7B52B013C01A5019401C057DF4F6881FD
:10F5D00079818A819B81C059D0400F9496A99B0163
:10F5E000AC01C301B2010F94B7B54B015C01A70197
:10F5F0009601CC56DF4F688179818A819B81C459FD
:10F60000D0400F9496A99B01AC01C501B4010F94A1
:10F61000B7B5C856DF4F288139814A815B81C85907
:10F62000D0400F94A6B62B013C01A0962CAD3DAD69
:10F630004EAD5FADA097C855DF4F688179818A8153
:10F640009B81C85AD0400F9496A99B01AC01C85722
:10F65000DF4F688179818A819B81C858D0400F949F
:10F66000B7B54B015C01A3019201C455DF4F68811E
:10F6700079818A819B81CC5AD0400F9496A99B01B5
:10F68000AC01C501B4010F94B7B54B015C01A701F2
:10F690009601C055DF4F688179818A819B81C05B6B
:10F6A000D0400F9496A99B01AC01C501B4010F9401
:10F6B000B7B5CA54DF4F288139814A815B81C65B67
:10F6C000D0400F94A6B64B015C01A0962CAD3DAD89
:10F6D0004EAD5FADA097C254DF4F688179818A81BA
:10F6E0009B81CE5BD0400F9496A99B01AC01C65480
:10F6F000DF4F688179818A819B81CA5BD0400F94FA
:10F70000B7B56B017C01A3019201CE53DF4F688135
:10F7100079818A819B81C25CD0400F9496A99B011C
:10F72000AC01C701B6010F94B7B56B017C01A5010F
:10F730009401CA53DF4F688179818A819B81C65CBD
:10F74000D0400F9496A99B01AC01C701B6010F945C
:10F75000B7B5C653DF4F288139814A815B81CA5CC6
:10F76000D0400F94A6B66B017C01115009F0C9CEB0
:10F77000A0962CAD3DAD4EAD5FADA097C256DF4F0C
:10F78000688179818A819B81CE59D0400F94B8B528
:10F790006093030C7093040C8093050C9093060CFB
:10F7A000A3019201CC55DF4F688179818A819B81C9
:10F7B000C45AD0400F94B8B56093070C7093080CEE
:10F7C0008093090C90930A0CA5019401A8966CAD46
:10F7D0007DAD8EAD9FADA8970F94B8B5A8966CAFD0
:10F7E0007DAF8EAF9FAFA897A7019601A4966CAD91
:10F7F0007DAD8EAD9FADA4970F94B8B5A4966CAFB8
:10F800007DAF8EAF9FAFA497CC57DF4F9881C45880
:10F81000D0409150CC57DF4F9883C458D0409111BD
:10F820007DCAA8966CAD7DAD8EAD9FADA8970F94A7
:10F83000A3B66093F30B7093F40B8093F50B909346
:10F84000F60BA8966CAD7DAD8EAD9FADA8970F94CD
:10F8500064B96093F70B7093F80B8093F90B909356
:10F86000FA0BA4966CAD7DAD8EAD9FADA4970F94B1
:10F8700064B9DC01CB01B0588093FB0B9093FC0B77
:10F88000A093FD0BB093FE0BA4966CAD7DAD8EAD39
:10F890009FADA4970F94A3B66093FF0B7093000CD9
:10F8A0008093010C9093020CA8962CAD3DAD4EAD0B
:10F8B0005FADA897A4966CAD7DAD8EAD9FADA497BE
:10F8C0000F94B7B54B015C016B017C01E894F7F82C
:10F8D00021EE3EE245E652E4A4966CAD7DAD8EADE0
:10F8E0009FADA4970F9496A99F938F937F936F9347
:10F8F00021EE3EE245E652E4C501B4010F9496A91B
:10F900009F938F937F936F9389E991E29F938F9356
:10F910000F9437AFB701A60180E69FE00F9450B572
:10F920000FB6F894DEBF0FBECDBF2FE132E449E041
:10F930005BE3C701B6010F9403B818166CF425E316
:10F940003AEF4EE85BE3C701B6010F9403B818160F
:10F9500034F001E010E005C000E010E002C002E079
:10F9600010E025E33AEF4EE85BE3A8966CAD7DAD81
:10F970008EAD9FADA8979F770F9403B818167CF0B3
:10F9800025E33AEF4EE85BE3A4966CAD7DAD8EAD1A
:10F990009FADA4979F770F9403B8181614F402E054
:10F9A00010E08091F30B9091F40BA091F50BB091C6
:10F9B000F60BE8968CAF9DAFAEAFBFAFE8978091E6
:10F9C000FB0B9091FC0BA091FD0BB091FE0BE4960C
:10F9D0008CAF9DAFAEAFBFAFE4978091030C909119
:10F9E000040CA091050CB091060CCC57DF4F888316
:10F9F0009983AA83BB83C458D0408091F70B909120
:10FA0000F80BA091F90BB091FA0BEC968CAF9DAF6F
:10FA1000AEAFBFAFEC978091FF0B9091000CA0911F
:10FA2000010CB091020CC458DF4F88839983AA83DC
:10FA3000BB83CC57D0408091070C9091080CA091CB
:10FA4000090CB0910A0CC058DF4F88839983AA83B0
:10FA5000BB83C058D0409EEA292E93E2392EA2EDF6
:10FA6000BBE06E96BFAFAEAF6E976E96EEADFFADDC
:10FA70006E9781809280A380B48085819681A781D2
:10FA8000B085AC968CAF9DAFAEAFBFAFAC97F10178
:10FA9000C590D590E590F490A5019401E8966CADE1
:10FAA0007DAD8EAD9FADE8970F9496A92B013C01DB
:10FAB000AC962CAD3DAD4EAD5FADAC97E4966CAD64
:10FAC0007DAD8EAD9FADE4970F9496A99B01AC01DF
:10FAD000C301B2010F94B8B5CC57DF4F28813981EB
:10FAE0004A815B81C458D0400F94B8B59B01AC01EA
:10FAF000C701B6010F94B7B56B017C01F1013496D3
:10FB00004590559065907490A5019401EC966CAD6C
:10FB10007DAD8EAD9FADEC970F9496A94B015C0126
:10FB2000AC962CAD3DAD4EAD5FADAC97C458DF4F3C
:10FB3000688179818A819B81CC57D0400F9496A9A6
:10FB40009B01AC01C501B4010F94B8B5C058DF4F9B
:10FB5000288139814A815B81C058D0400F94B8B563
:10FB60009B01AC01C301B2010F94B7B54B015C011D
:10FB7000A7019601C701B6010F9496A96B017C01FC
:10FB8000A5019401C501B4010F9496A99B01AC0194
:10FB9000C701B6010F94B8B50F946FB92DEC3CECCA
:10FBA0004CE45FE30F9403B8181614F40EEF1FEF44
:10FBB0006E96EEADFFAD6E9738966E96FFAFEEAFD8
:10FBC0006E97F8E02F0E311C6E962EAD3FAD6E97FE
:10FBD000225F3B4009F049CF0115110509F07AC1B8
:10FBE000A4962CAD3DAD4EAD5FADA497A8966CAD7F
:10FBF0007DAD8EAD9FADA8970F94B8B520E030E0F5
:10FC000040E05FE30F9496A96B017C010F94A3B6CB
:10FC10002B013C016093F30B7093F40B8093F50B75
:10FC20009093F60BC701B6010F9464B9A4966CAF1C
:10FC30007DAF8EAF9FAFA4976093F70B7093F80BD7
:10FC40008093F90B9093FA0BDC01CB01B058AC9682
:10FC50008CAF9DAFAEAFBFAFAC978093FB0B9093D3
:10FC6000FC0BA093FD0BB093FE0B4092FF0B509248
:10FC7000000C6092010C7092020C1092030C109216
:10FC8000040C1092050C1092060C1092070C1092A6
:10FC9000080C1092090C10920A0CA0961CAE1DAE16
:10FCA0001EAE1FAEA097A8961CAE1DAE1EAE1FAE18
:10FCB000A897C456DF4FA881B981CC59D04011967E
:10FCC0008D909D90AD90BC90149715968D919D91BF
:10FCD0000D90BC91A02DE8968CAF9DAFAEAFBFAF9D
:10FCE000E897CE55DF4FE881F981C25AD040C590E0
:10FCF000D590E590F490A5019401C301B2010F9451
:10FD000096A9E4966CAF7DAF8EAF9FAFE497E8966F
:10FD10002CAD3DAD4EAD5FADE897AC966CAD7DAD15
:10FD20008EAD9FADAC970F9496A99B01AC01E49664
:10FD30006CAD7DAD8EAD9FADE4970F94B8B59B01D2
:10FD4000AC01C701B6010F94B7B52091030C3091F7
:10FD5000040C4091050C5091060C0F94B8B56B0142
:10FD60007C016093030C7093040C8093050C9093BA
:10FD7000060C20E030E040E85FE3A8966CAD7DAD76
:10FD80008EAD9FADA8970F94B8B5A8966CAF7DAF18
:10FD90008EAF9FAFA897CE55DF4FE881F981C25A49
:10FDA000D040349685919591A591B491E4968CAF0D
:10FDB0009DAFAEAFBFAFE497A5019401A4966CAD23
:10FDC0007DAD8EAD9FADA4970F9496A94B015C01BC
:10FDD000E8962CAD3DAD4EAD5FADE897C301B201E5
:10FDE0000F9496A99B01AC01C501B4010F94B8B55D
:10FDF0009B01AC01E4966CAD7DAD8EAD9FADE497FB
:10FE00000F94B7B52091070C3091080C4091090C64
:10FE100050910A0C0F94B8B54B015C016093070C2C
:10FE20007093080C8093090C90930A0C20E030E04A
:10FE300040E85FE3A0966CAD7DAD8EAD9FADA09721
:10FE40000F94B8B5A0966CAF7DAF8EAF9FAFA09763
:10FE5000C456DF4FA881B981CC59D0401896C456FA
:10FE6000DF4FB983A883CC59D040CE55DF4FE8810E
:10FE7000F981C25AD0403896CE55DF4FF983E883D6
:10FE8000C25AD040A25FBB4009F013CFA8962CAD58
:10FE90003DAD4EAD5FADA897C701B6010F94A6B6B4
:10FEA0006093030C7093040C8093050C9093060CE4
:10FEB000A0962CAD3DAD4EAD5FADA097C501B40190
:10FEC0000F94A6B66093070C7093080C8093090CEE
:10FED00090930A0C4090F30B5090F40B6090F50B4C
:10FEE0007090F60BC090FF0BD090000CE090010CCE
:10FEF000F090020C8091F70B9091F80BA091F90B08
:10FF0000B091FA0BA4968CAF9DAFAEAFBFAFA497E4
:10FF10008091FB0B9091FC0BA091FD0BB091FE0B1F
:10FF2000A8968CAF9DAFAEAFBFAFA897A7019601C3
:10FF3000C301B2010F9496A94B015C01A8962CADA8
:10FF40003DAD4EAD5FADA897A4966CAD7DAD8EADC9
:10FF50009FADA4970F9496A99B01AC01C501B40174
:10FF60000F94B7B54B015C019B01AC01C701B60111
:10FF70000F94A6B66B017C01A8966CAD7DAD8EADDD
:10FF80009FADA8979058A50194010F94A6B6A89686
:10FF90006CAF7DAF8EAF9FAFA897A4966CAD7DADD3
:10FFA0008EAD9FADA4979058A50194010F94A6B66D
:10FFB000A0966CAF7DAF8EAF9FAFA097A5019401C7
:10FFC000C301B2010F94A6B64B015C014090030C33
:10FFD0005090040C6090050C7090060C8091070CFA
:10FFE0009091080CA091090CB0910A0CA4968CAFCA
:10FFF0009DAFAEAFBFAFA497C092F30BD092F40BFE
:020000021000EC
:10000000E092F50BF092F60BA0968CAD9DADAEADE7
:10001000BFADA0978093F70B9093F80BA093F90BCB
:10002000B093FA0BA8968CAD9DADAEADBFADA897C1
:100030008093FB0B9093FC0BA093FD0BB093FE0BF6
:100040008092FF0B9092000CA092010CB092020CD7
:10005000C701B6019058A30192010F9496A96B01B4
:100060007C01A4962CAD3DAD4EAD5FADA497A89696
:100070006CAD7DAD8EAD9FADA8970F9496A99B01F9
:10008000AC01C701B6010F94B7B56093030C709330
:10009000040C8093050C9093060CA0966CAD7DAD7E
:1000A0008EAD9FADA0979058A30192010F9496A991
:1000B0006B017C01A4962CAD3DAD4EAD5FADA49718
:1000C000C501B4010F9496A99B01AC01C701B6010B
:1000D0000F94B7B56093070C7093080C8093090CCC
:1000E00090930A0C80E090E00E949BBE17FD5BC0DD
:1000F00087ED91E29F938F930F9437AF43E05CE0DD
:100100006BEF7BE083EF9BE00E94F9944091030C3E
:100110005091040C6091050C7091060C85EE9FE0E7
:100120000F9450B54091070C5091080C6091090C48
:1001300070910A0C89EE9FE00F9450B54091F30B3B
:100140005091F40B6091F50B7091F60B8DED9FE0E3
:100150000F9450B54091F70B5091F80B6091F90B4B
:100160007091FA0B81EE9FE00F9450B54091FB0B1C
:100170005091FC0B6091FD0B7091FE0B85ED9FE0A3
:100180000F9450B54091FF0B5091000C6091010C01
:100190007091020C89ED9FE00F9450B50E947E94FF
:1001A0000F900F9019C00E3F1F4F89F4AD96AFAD61
:1001B000AD97A23079F480EB91E29F938F930F94E7
:1001C00037AF0F900F9006C0AD961FAEAD970FEFF3
:1001D0001FEF02C00EEF1FEFCC54DF4F88819981D3
:1001E000C45BD0400E944F6380E090E0A0EAB0E49E
:1001F0008093D2179093D317A093D417B093D517A9
:1002000060E070E080EA91E40F9485190E94DAA31F
:1002100017FD22C020E030E046E153E46091D217A0
:100220007091D3178091D4179091D5170F94B8B5CA
:100230006093D2177093D3178093D4179093D517E8
:1002400065E575E585E591E40E943E948AE69FE1C7
:100250000E94AFC80E94EC9F81E00E94B3A282E09E
:100260000E94EF990F3FBFEF1B0731F48DE29FE132
:100270000E94AFC810E049C00E3FEFEF1E0781F4A7
:10028000AD96FFADAD97FF2329F0F23031F086EE49
:100290009DE1EECF8BE69EE1EBCF8BE29EE1E8CFD6
:1002A000AD962FADAD97211106C00330110598F022
:1002B0008BE69EE117C0AD963FADAD97323019F495
:1002C00088EE9EE102C08EE99EE10E94AFC8101642
:1002D00011065CF309C0F801EE0FFF1FEA53FD4F52
:1002E000808191810E94AFC80F3F1F4F19F286EEA7
:1002F0000E94FE698FE59FE00F941DB5813021F0CB
:100300008FE89FE10E94AFC811E00F94D15CEBC46D
:100310008FED93E20E94AFC810E0E5C481E0E9816F
:10032000FA81882309F482C00091DE161091DF164D
:100330002091E0163091E1164091DA165091DB16CB
:100340006091DC167091DD168091D6169091D716CB
:10035000A091D816B091D916FF93EF931F930F93E6
:100360005F934F939F938F9386E992E29F938F932E
:100370000F9437AF4091DE165091DF166091E01672
:100380007091E1164854510900E028EC30E0AD9638
:100390006FADAD97AE967FADAE97C2010E9484F46B
:1003A0008091D6169091D716A091D816B091D916F3
:1003B000C058DF4F88839983AA83BB83C058D0403D
:1003C000C058DF4F28803980C058D0408091DA165D
:1003D0009091DB16A091DC16B091DD16C457DF4F6B
:1003E00088839983AA83BB83CC58D0408091DE1642
:1003F0009091DF16A091E016B091E116C057DF4F43
:1004000088839983AA83BB83C059D040C057DF4FEC
:1004100068807980C059D040A5EFB3E10FB6F89459
:10042000DEBF0FBECDBF80E090E006C0F0E98F1ABE
:10043000F1E09F0A0C94CE72FC01E85BFC4D259123
:1004400034912D933D93FC01E05DFC4D2591349159
:1004500057963C932E93569702968831910561F7F3
:1004600080E197E263969FAF8EAF639780EE92E252
:100470009F938F930F9437AF0F900F90A0E4B0E04D
:10048000AA96BFAFAEAFAA97412C512CC457DF4FED
:10049000E881F981CC58D040E05EF340C857DF4F87
:1004A000F983E883C858D040C201880F991FC85704
:1004B000DF4FA881B981C858D040A80FB91FCC56CA
:1004C000DF4FB983A883C459D040AA96EEADFFADE3
:1004D000AA97AE96FFAFEEAFAE97912C9101205E3A
:1004E0003340CC57DF4F39832883C458D040C101F3
:1004F00080529C4FEA969FAF8EAFEA97D201AC5ED6
:10050000BF4EC856DF4FB983A883C859D040C090AA
:10051000DE16D090DF16E090E016F090E1169920FC
:1005200029F0EA966EAD7FADEA9706C0CC57DF4F53
:1005300068817981C458D0408091D6169091D716A1
:10054000A091D816B091D916681B790BCB01770F03
:10055000AA0BBB0B8C019D01B7FF07C00027112719
:100560009801081B190B2A0B3B0B011511052105DE
:10057000310561F0BC01CD01662797FD63957727B2
:1005800088279927A80181E00F9481778091DA1656
:100590009091DB16A091DC16B091DD16CC56DF4FA2
:1005A00028813981C459D040281B390BC901092E33
:1005B000000CAA0BBB0BAC01BD01B7FF07C0442761
:1005C0005527BA01481B590B6A0B7B0B8827B7FDCF
:1005D00083959927AA27BB27880F411551056105E7
:1005E000710521F0682F82E00F9481778091DE16EB
:1005F0009091DF16A091E016B091E116C81AD90AC1
:100600000D2C000CEE08FF08B701A601F7FE07C08D
:1006100044275527BA014C195D096E097F09CC247E
:10062000F7FCC394DD24EE24FF24CC0CCC0C411544
:1006300051056105710521F06C2D84E00F948177DF
:100640004091DE165091DF166091E0167091E11630
:10065000992039F0E9968FADE997EA969FADEA9730
:100660000AC0CC57DF4F8881C458D040CB57DF4FEA
:100670009881C558D04000E028EC30E0CC56DF4FE0
:1006800068817981C459D0400E9484F431E080911E
:100690000B01931202C0816001C08E7F80930B0119
:1006A0000000AE966FADAE976F93AD968FADAD97E0
:1006B0008F938CED92E29F938F930F9437AFDE016F
:1006C0001196E696BFAFAEAFE697C856DF4FE8810A
:1006D000F981C859D040E296FFAFEEAFE2976E01C4
:1006E000FFE3CF0ED11C0F900F900F900F90F0EE04
:1006F000AF2EF3E0BF2E20E137E263963FAF2EAF7F
:100700006397911003C08FEF9FEF02C081E090E0EC
:100710004091D6165091D7166091D8167091D9167F
:100720008A9D80018B9D100D9A9D100D1124020D44
:10073000131D041B150B17FF03C01195019511091B
:10074000C80195958795CC55DF4F99838883C45A06
:10075000D0401C9903C08824839402C075E0872E82
:10076000692D882D0E94FDF3E12CF12CCC55DF4F33
:10077000A881B981C45AD040EA16FB0691F028EC52
:1007800030E0AE014F5A5F4F68EE73E0882D0E9453
:10079000E4F2692D882D0E941EF49FEFE91AF90AF0
:1007A000E5CF0E191F0967961FAF0EAF6797692D2A
:1007B000882D0E94FDF39E012B5A3F4FAE014F5AE8
:1007C0005F4F68EE73E0882D0E9489F3882329F03B
:1007D000692D882D0E941EF4EECF80910B018B7F36
:1007E00080930B010000E0E1F7E26396FFAFEEAF0C
:1007F00063970091DE161091DF162091E01630917C
:10080000E116005A164F17FF02C00F5F1F4F1595D4
:1008100007958091DE169091DF16A091E016B091B9
:10082000E1168017910704F51C9B1EC028EC30E0F0
:10083000AE014F5A5F4F68EE73E084E00E94E4F22D
:100840008091DE169091DF16A091E016B091E1162E
:100850000196A11DB11D8093DE169093DF16A09323
:10086000E016B093E116D5CF1C99B7C060E084E0E4
:100870000E94FDF363962EAD3FAD6397203167E292
:10088000360768F4AE014F5A5F4F68E17CEF84E0B1
:100890000E94E4F260E084E00E941EF4EBCF8091BD
:1008A0000B01846080930B01000080E197E2639666
:1008B0009FAF8EAF63970091DE161091DF162091E7
:1008C000E0163091E116060D171D17FF02C00F5FED
:1008D0001F4F159507958091DE169091DF16A09118
:1008E000E016B091E1160817190704F51C99B7C076
:1008F00028EC30E0AE014F5A5F4F68EE73E084E0C1
:100900000E94E4F28091DE169091DF16A091E0162D
:10091000B091E1160197A109B1098093DE16909379
:10092000DF16A093E016B093E116D5CF83011C9992
:1009300026C09EC063968EAD9FAD6397803197426F
:1009400008F0DDC028EC30E0AE014F5A5F4F68E19F
:100950007CEF84E00E94E4F28091DE169091DF1635
:10096000A091E016B091E1160197A109B109809319
:10097000DE169093DF16A093E016B093E1168091F7
:10098000DE169091DF16A091E016B091E116681680
:1009900079060CF0B4C0CECF89819A8180349B4017
:1009A00098F49E012F5F3F4F790104EB10E02CE794
:1009B0003CEFA4014C5251406B2D7A2D8D2D9C2D76
:1009C0000F94D977811102C080E0A9CC29813A81A6
:1009D0002059374F3A832983A2CC8091DE1690911B
:1009E000DF16A091E016B091E116E0E6F9E0E81B11
:1009F000F90BCF01F7FF02C080E090E023969FAF94
:100A00008EAF23971C9B32CF8091DE169091DF161C
:100A1000A091E016B091E116803699400CF026CFF7
:100A20009E012F5B3F4FAE014F5A5F4F68EE73E060
:100A300084E00E9489F38091DE169091DF16A091E8
:100A4000E016B091E1160196A11DB11D8093DE164E
:100A50009093DF16A093E016B093E116D3CF0091E8
:100A6000DE161091DF162091E0163091E1165FCF6F
:100A70008091DE169091DF16A091E016B091E116FC
:100A80008619970997FF02C080E090E023969FAFF8
:100A90008EAF23971C992AC08091DE169091DF16A5
:100AA000A091E016B091E11668167906FCF49E015B
:100AB0002F5B3F4FAE014F5A5F4F68EE73E084E00B
:100AC0000E9489F38091DE169091DF16A091E016C6
:100AD000B091E1160197A109B1098093DE169093B8
:100AE000DF16A093E016B093E116D4CF0091DE1686
:100AF0001091DF162091E0163091E11640CF0619D3
:100B00001709911007C0E696EEADFFADE697118389
:100B100000831AC0012E000C220B330BD6018D91DD
:100B20009C91080F191F211D311D3695279517958A
:100B300007950F3F11052105310508F00FEFE296EB
:100B4000EEADFFADE2970083E6962EAD3FADE697A2
:100B50002E5F3F4FE6963FAF2EAFE697E2968EAD03
:100B60009FADE2970197E2969FAF8EAFE29792E03A
:100B7000C91AD108A0E4AA1AB108B0EEAB16BBEFAF
:100B8000BB0609F0B8CDAE96EEADFFADAE9731978E
:100B9000AE96FFAFEEAFAE97F1E09F1611F40C9456
:100BA000777399249394B3CC8F3F11F00C94D8733E
:100BB0002F5F3F4F0C94D8734333510514F40C94BA
:100BC000E4732333310514F40C94E47380E094E06F
:100BD000841B950B821B930B8417950714F00C94C0
:100BE000E4738217930714F00C94E4730DEF1FEF76
:100BF0000C9449750FEF0C94FF738FEF22966FAD35
:100C000022971981082F0C94197420E030E040EAF3
:100C100050E469817A818B819C810F94B7B59F9351
:100C20008F937F936F93A501940125966CAD7DAD55
:100C30008EAD9FAD25970F94B7B59F938F937F93FC
:100C40006F93FF92EF92DF92CF9284E193E29F93B2
:100C50008F930F9437AF65964CAE5DAE6EAE7FAEA0
:100C6000659725968CAE9DAEAEAEBFAE25970FB6FE
:100C7000F894DEBF0FBECDBF0C9498740FEF1FEF3A
:100C80000C944175F2012581368147815085EC969F
:100C90006CAD7DAD8EAD9FADEC970C94CC77F20131
:100CA0002581368147815085EC966CAD7DAD8EAD4A
:100CB0009FADEC970C94E57760E070E080E89FE3EF
:100CC0000C94E777112311F40C94F577812C912C77
:100CD00070E8A72E7FE3B72E0C94D07701110C9407
:100CE000BB770C94F57781E00E94B3A280E00F946B
:100CF000593980E0DBD6812FC353DF4F0FB6F8940C
:100D0000DEBF0FBECDBFDF91CF911F910F91FF903E
:100D1000EF90DF90CF90BF90AF909F908F907F909B
:100D20006F905F904F903F902F90089584FF02C086
:100D30008D9A01C08D9885FF02C0A49A01C0A49825
:100D40002FB786FF05C0F89490910201906804C007
:100D5000F894909102019F77909302012FBF87FF33
:100D600002C0A39A01C0A3988F9A85E08A95F1F7F3
:100D700000008F980895CF93AC012091A509309180
:100D8000A6098091B3079091B4072817390739F461
:100D9000E091B607F091B7071E161F06A4F1C62F03
:100DA000FA01E80FF91FBF0163597F4F82179307BC
:100DB00028F481E02617370738F525C06E3E7140CC
:100DC00000F13496EE3EF14018F429363105C8F4AE
:100DD00043595F4F24173507B0F04DEE51E0481BE3
:100DE000590B60E070E08854984F0F94DBBACC2325
:100DF00009F0F8941092B4071092B307CC2309F0CD
:100E0000789481E001C080E0CF910895FF920F9324
:100E10001F93CF93DF931F92CDB7DEB7F82E8A01D1
:100E200060FF02C05D9A01C05D988AE18A95F1F782
:100E300000C08F2D69837ADF698161FD0AC08FE868
:100E400091E00197F1F700C000008F2D8295807F1F
:100E50006DDFC8010F90DF91CF911F910F91FF902F
:100E60000C94D9F28A3069F48091A505843018F089
:100E70008FEF8093A5056091A5056F5F80E00C94CE
:100E8000109C44E650E061E0C1CFCF92DF92EF9238
:100E9000FF926B017C016093A1057093A205809382
:100EA000A3059093A40580919505823009F04DC06B
:100EB00020E030E040E950E4C701B6010F942DB0C6
:100EC00087FF0EC08091361790913717A091381781
:100ED000B0913917803D9740A105B105A0F435C008
:100EE0002AE939E949E95EE3C701B6010F942DB05B
:100EF00087FF23C020E030E048E351E4C701B6019A
:100F00000F9496A918C02AE939E949E95EE3C701B7
:100F1000B6010F942DB087FDEDCF20E030E040E822
:100F20005EE3C701B6010F9496A920E030E048E5E2
:100F300050E40F94B8B56B017C0185E495E20E9402
:100F4000C36AC701B6010F942463C701B601FF90BD
:100F5000EF90DF90CF900895CF92DF92EF92FF92C3
:100F6000CF9390919505891709F442C0C82FC0907E
:100F7000A105D090A205E090A305F090A40520E083
:100F800030E0A901C701B6010F942DB0882341F0CC
:100F9000C0925A17D0925B17E0925C17F0925D17DF
:100FA00088E295E20E94C36AC13049F028F0C2305D
:100FB00061F488E195E205C080E295E202C08CE12F
:100FC00095E20E94C36A0E94E46BC093950560910C
:100FD0005A1770915B1780915C1790915D1755DFE0
:100FE00060935A1770935B1780935C1790935D170B
:100FF000CF91FF90EF90DF90CF9008951F920F92C6
:101000000FB60F9211240BB60F922F938F939F93CD
:10101000AF93BF93EF93FF938091A00590E088304A
:10102000910508F089C0FC018827EE58FF4F8F4FCB
:101030000D94A5BA8091D51681117EC080911E06AF
:10104000880F80939F05882309F476C081E00BC048
:1010500080919E058F5F80939E0590919F059817C4
:1010600008F46AC082E08093A00566C083E08093A4
:10107000A0058FE080939D058FEF86BD81E085BD43
:1010800084B58F7E39C080919D058295807F819542
:1010900088BD80919D0581113BC084E08093A005AF
:1010A0008FEF88BD8EEF86BD47C085E08093A00599
:1010B0008FEF88BD86BD3EC02FEF28BD8091D5162D
:1010C00081113AC080919E058F5F80939E0590911B
:1010D0009F05891788F180911E0690E08F37910552
:1010E0005CF586E08093A0058FE080939D0526BD8A
:1010F00081E085BD84B5806184BD1EC080919D0561
:101100008295807F819588BD80919D05882321F0FF
:10111000815080939D0510C087E08093A00580E8F2
:1011200086BD8FEF88BD08C01092A00580E886BDFF
:101130008FEF88BD82E085BDFF91EF91BF91AF91A8
:101140009F918F912F910F900BBE0F900FBE0F901C
:101150001F9018958091B4069091B5069C012E526F
:1011600033412033334118F487EE94E20BC02091D1
:10117000FC06213059F4835D9A438E31954030F45A
:1011800086EB94E20F945FAF80E0089581E00895CC
:10119000809161028823B1F080911302882391F03D
:1011A00080914005882371F08091060180FF05C081
:1011B00081E080939C0580E0089580919C058111D9
:1011C00010929C050895CF93C82FC4DF811108C0E9
:1011D0001092610281E0809343051092120209C0CF
:1011E00091E0909361021092430590931202CC23F8
:1011F00031F06091120287E69FE00F943EB5809136
:101200006102CF9108958091FC06882341F08130DE
:1012100019F48CEC96E208958EEB96E208958AED2F
:1012200096E208958DE994E20F945FAF20E030E0FC
:10123000A901CA01B9010F94783D60E070E0CB01CB
:101240000D94983B0F931F93CF93C82F8B0182303F
:1012500018F460E774E20CC0843018F469E674E2B4
:1012600007C0863018F462E674E202C06BE574E2EF
:10127000C8010F94EFADC170CF5CF801C68317822F
:10128000CF911F910F9108952BE0829FC0011124EF
:10129000805B924F0F942AB521E0019609F420E07B
:1012A000822F0895CF93DF93C82FD8E0CF5FC83047
:1012B0000CF0C0E08C2FE8DF811104C0D150B1F7F1
:1012C0008FEF01C08C2FDF91CF91089581EA9DE0CF
:1012D0000F941DB5E7DF87FD05C0682F81EA9DE00B
:1012E0000D943EB50895FC012081318137FF07C080
:1012F0008DE28093EB0631952195310914C0243697
:10130000310574F0C90164E670E00F9476BACB0140
:101310006AE070E00F9476BA805D8093EB0606C0B9
:1013200080E28093EB062A30310564F0EAE0F0E0D9
:10133000C901BF010F9476BACB01BF010F9476BAF1
:10134000805D01C080E28093EC06C9016AE070E034
:101350000F9476BA805D8093ED061092EE068BEEC8
:1013600096E008958F929F92AF92BF92CF92DF92B4
:10137000EF92FF92CF9320E030E048EC52E4FC0182
:1013800060817181828193810F9496A90F9417B720
:101390004B015C0197FD12C020E137E240E050E0D4
:1013A0000F9489BACA01B9012AE030E040E050E068
:1013B0000F9489BA605D6093EB0603C08DE2809361
:1013C000EB06640197FE04C0CC24DD24C818D908BC
:1013D0000D2C000CEE08FF08C701B60128EE33E023
:1013E00040E050E00F9489BA8AE0882E912CA12C1D
:1013F000B12CCA01B901A50194010F9489BA605DAD
:101400006093EC06C701B60124E630E040E050E00E
:101410000F9489BACA01B901A50194010F9489BA40
:10142000605D6093ED068EE28093EE06C701B60123
:10143000A50194010F9489BAC62FCA01B901A5016B
:1014400094010F9489BA605D6093EF06C05DC0930C
:10145000F0061092F1068BEE96E0CF91FF90EF90A0
:10146000DF90CF90BF90AF909F908F900895CF93D3
:10147000DF931F921F92CDB7DEB7FC0160817181AF
:10148000828193810F9417B77A836983CE01019685
:101490002ADF0F900F90DF91CF9108952091B6072A
:1014A0003091B70721153105A1F18091A5099091DF
:1014B000A60940E050E0FC01E854F84FA081A230BA
:1014C00021F461817281460F571F2150310921F1AA
:1014D0000396FC01E854F84FE0810196E111F9CF41
:1014E0008D3EE1E09E0740F4FC01E854F84FE081B6
:1014F000E111E1CF0196F4CF8D3EE1E09E07D9F6F0
:10150000E8EBF7E0CF01885B9740A191AA23D1F3E4
:10151000D2CF80E090E00895CA010895FF920F9322
:101520001F93CF93DF938C01F62E662339F00F942F
:10153000F6ADEC018036910560F082C0EC010990B7
:101540000020E9F72197C81BD90BC036D10508F058
:1015500061C060E0CE010FDC882309F44DC08091AA
:10156000B3079091B407FC01E854F84F23E02083BF
:101570000396B8018854984FFF2019F00F94EFADEF
:1015800002C00F9414BB8FE594E60E94C36A8EE5F7
:1015900095E20E94C36A8091B3079091B407855485
:1015A000984F0E94E66B88E294E20E94C36A0E9410
:1015B000E46B8091B3079091B4070496C80FD91FCC
:1015C000CD3E81E0D80729F0D093B407C093B3078C
:1015D00004C01092B4071092B3078091B60790919F
:1015E000B70701969093B7078093B607DF91CF9125
:1015F0001F910F91FF9008958DE394E60E94C36AB6
:101600008EE595E20E94C36AFF2061F0C8010E9446
:10161000C36A0BC08DE394E60E94C36A8EE595E22F
:101620000E94C36AC8010E94E66B81E194E20E94B5
:10163000C36ADF91CF911F910F91FF900C94E46BDF
:101640008DE394E60E94C36A8EE595E20E94C36A28
:10165000DDCF2F923F924F925F926F927F928F9247
:101660009F92AF92BF92CF92DF92EF92FF920F9331
:101670001F93CF93DF9300D0CDB7DEB78A839B83D0
:10168000062F10E08FE3B82EBF9296E2892E8F923C
:1016900022EE922E9F9234EDA32EAF92B801012E2E
:1016A000000C880B990B0F9433B02DEC3CEC4CECF8
:1016B0005EE30F9496A99B01AC010F94B8B59B0112
:1016C000AC0160E070E08CE092E40F94B7B59F93BA
:1016D0008F937F936F931F9286E48F9348E8C42E75
:1016E00044E2D42EDF92CF928B818F939A819F9385
:1016F0000F9490AF60E08A819B8110DFB801660F84
:10170000771F6F5F7F4F072E000C880B990B0F948C
:1017100033B02DEC3CEC4CEC5EE30F9496A99B01AE
:10172000AC0160E070E08CE092E40F94B7B5462E17
:10173000382E292E6CE3562E5F92E9E56E2E6F92BD
:10174000F9EF7F2E7F92BF929F938F937F934F925B
:10175000A7E7EA2EA4E2FA2EFF92EF928B818F93F5
:101760009A819F9379830F9490AF60E08A819B81E7
:10177000D5DEBF928F929F92AF922F923F92798146
:101780007F934F921F9282E38F93DF92CF928B8150
:101790008F939A819F930F9490AF0FB6F894DEBF0A
:1017A0000FBECDBF60E08A819B81B8DE5F926F92F1
:1017B0007F92BF92B8016F5F7F4F072E000C880B9E
:1017C000990B0F9433B02DEC3CEC4CEC5EE30F9492
:1017D00096A99B01AC010F94B8B59B01AC0160E0E8
:1017E00070E08CE092E40F94B7B59F938F937F9352
:1017F0006F93FF92EF929B819F938A818F930F94B7
:1018000090AF0FB6F894DEBF0FBECDBF60E08A8107
:101810009B810F900F900F90DF91CF911F910F91AF
:10182000FF90EF90DF90CF90BF90AF909F908F9000
:101830007F906F905F904F903F902F906FCE8091F0
:10184000B6079091B707181619060CF048C0019713
:101850009093B7078093B607892B79F48091B107ED
:101860009091B207892B21F41092B4071092B3071C
:101870008091B3079091B4072CC0E091A509F09135
:10188000A609E554F84FCF01885B974021912111BB
:10189000FACF01968D3E21E0920740F09093A60981
:1018A0008093A5098D3E914061F017C0AC014F5F58
:1018B0005F4FFC01E854F84F208121110AC0CA0192
:1018C000E9CFE8EBF7E0CF01885B97402191222335
:1018D000D1F39093A6098093A50981E0089580E053
:1018E00008958091B6079091B707892B21F00F9446
:1018F000C87DA5DFF6CF1092A6091092A509109217
:10190000B4071092B30781E08093B5070895FC01F6
:1019100020E03EE2DB014C91403241F0283011F4EE
:1019200030833196DB014C91408331962F5F6F5F9E
:101930007F4F2B3079F71082089560915F0484E324
:101940009DE00F943EB560915D0483E39DE00F94AC
:101950003EB56091080282E39DE00F943EB5609130
:1019600006027091070280E39DE00D9458B5FF9246
:101970000F931F93CF93DF93FC01F080F11002C00F
:10198000F12C19C0EB018C010E94556FF8014181C7
:1019900052819E01240F351F2417350720F062174E
:1019A000730738F403C06217730750F364177507A1
:1019B00038F7F80110828F2DDF91CF911F910F9191
:1019C000FF900895CF93DF93EC010E94556F7A83C7
:1019D000698381E08883DF91CF9108957F92CF92D0
:1019E000DF92EF92FF920F931F93CF93DF93FC014F
:1019F0007080711002C0712C23C06A017B01EC0160
:101A00000E94556F09811A812B813C81C00ED11E25
:101A1000E21EF31EC016D106E206F30630F06C1586
:101A20007D058E059F0558F405C06C157D058E0556
:101A30009F0508F36017710782079307E0F6188285
:101A4000872DDF91CF911F910F91FF90EF90DF9045
:101A5000CF907F90089580916104882331F1809127
:101A600008028230A1F4A0910602B091070228EE8C
:101A700033E00F94B3BAAB01BC018AEA9CE0AEDF5D
:101A8000811107C08091AA0C882379F007C08111C9
:101A900005C060915D0470915E0404C060915F04B4
:101AA0007091600485E00C9412F20895882361F02F
:101AB00081E08093080280915F04909160044E97CA
:101AC00094F48EE190E00BC082E39DE00F941DB58D
:101AD0008093080284E39DE00F941DB590E09093FD
:101AE000600480935F04B7CFCF93DF93EC010E9433
:101AF000556F69837A838B839C8381E08883DF9130
:101B0000CF9108954F925F926F927F928F929F92A2
:101B1000AF92BF92CF92DF92EF92FF920F931F93FB
:101B2000CF93DF93CDB7DEB76E970FB6F894DEBFD5
:101B30000FBECDBF61E08FE590E01DD9882309F489
:101B4000B7C30E94E7698F37910571F48091F9045A
:101B50009091FA049093F8048093F7048CE494E253
:101B60000E94C36A0E94E46B94E2F92E0E94E76926
:101B7000181619060CF077C180911107882329F0F7
:101B800080915F05882309F46EC180912607811139
:101B90006AC10E94076A182F85EA9CE0A5DF17FD3D
:101BA000E5CF2091B1073091B2071A3031F01D30E6
:101BB00021F02F3531050CF43BC12115310519F405
:101BC00010929B0575C3C090B307D090B4078601EF
:101BD0000D5F1F4F2854384FF901E00FF11F10829D
:101BE00080919B05811112C1109297051092980562
:101BF0001092990510929A050854184F68EC73E0FA
:101C0000C8010F9438BB892B09F06AC0F8018081A4
